:100000000C94CE000C94ED000C94ED000C94ED00DB
:100010000C94ED000C94ED000C94ED000C94ED00AC
:100020000C94ED000C94ED000C94ED000C94ED009C
:100030000C94ED000C943D010C94ED000C94ED003B
:100040000C94ED000C94ED000C94ED000C94ED007C
:100050000C94ED000C94ED000C94ED000C94ED006C
:100060000C94ED000C94ED000C94ED000C94ED005C
:100070000C94ED000C94ED000C94ED000C94ED004C
:100080000C942C080C94ED000C94ED001B69706925
:100090006B696669A768A768A768A76861695C69F2
:1000A000A768A768A768A76854694F694A6945693E
:1000B000A768A768A768A768A768A768A768A768C8
:1000C000A768A768A768A768A768A768A768A768B8
:1000D000A768A768A768A768A768A768A768A768A8
:1000E000A768A768A768A768A768A768A768A76898
:1000F000A768A768A768A768A768A768A768A76888
:10010000A768A768A768A768A768A768A768A76877
:10011000A768A768A768A768A768A768A768A76867
:10012000A768A768A768A768A768A768A768A76857
:10013000A768A768A768A768A768A768A768A76847
:10014000A768A768A768A768A768A768A768A76837
:10015000A768A768A768A768A768A768A768A76827
:10016000A768A768A768A768A768A768A768A76817
:10017000A768A768A768A768A768A768A768A76807
:10018000A768A768A768A768A768A76840693B69C8
:10019000366931692C6927692069146911241FBEE9
:1001A000CFEFD0E4DEBFCDBF15E0A0E0B1E0EEE1DF
:1001B000F7ED00E00BBF02C007900D92A038B10729
:1001C000D9F71BE3A0E8B5E001C01D92A53CB1073B
:1001D000E1F70E9439090C948D6B0C94000040915A
:1001E0000001442309F455C295B19F7370E460E89F
:1001F00058E095B987FD73B963B9880F4E99839517
:100200005A9563B9B1F70895372F3F7030637295EF
:100210008295482F7F70407F472B8F7080639FB7F8
:10022000F89442B985B94F9A000062B935B91C9A61
:100230000000000086B100001C9A4F9A9FBF0895ED
:10024000372F3F70306172958295582F7F70507FA5
:10025000572B8F7080632FEF9FB7F89427B952B94F
:1002600085B94F9A48B91D9A62B935B91C9A1D9A39
:100270001C9A4F9A17B89FBF08959F938F937F93AF
:100280007FB7992780EF1C9A4F9A93951C9A4F9AA3
:10029000D1F78395C1F77FBF7F918F919F9118957B
:1002A000A0E3B0E0E6E5F1E00C94566BA8E04E0167
:1002B0000894811C911CF401BA2F1192BA95E9F7A8
:1002C00029833A834B835C836D837E838F839887F6
:1002D000CE010996FC011192AA95E9F7A986BA8682
:1002E000CB86DC86ED86FE860F87188B29813A81C6
:1002F0004B815C812DA73EA74FA758AB79018A019E
:100300008FEF9FEFA0E0B0E0E822F9220A231B2341
:100310001A014424552429853A854B855C8529A7F3
:100320003AA74BA75CA759016A01A822B922CA22A1
:10033000DB223A0188249924C601B501A80197015E
:100340000E94156B6DA37EA38FA398A7C401B30170
:100350000E94156B69A37AA38BA39CA3C601B50168
:10036000A20191010E94156B7B018C01C401B301B4
:100370000E94156B5B016C0189A19AA1ABA1BCA184
:100380008E0D9F1DA01FB11F89A39AA3ABA3BCA371
:100390002DA13EA14FA158A5CA01AA27BB2729A17B
:1003A0003AA14BA15CA1280F391F4A1F5B1F29A34B
:1003B0003AA34BA35CA32E153F054007510740F419
:1003C00080E090E0A1E0B0E0A80EB91ECA1EDB1EDE
:1003D00089A19AA1ABA1BCA19D01442755272A0D53
:1003E0003B1D4C1D5D1D2D8F3E8F4F8F58A36C0103
:1003F000BB24AA248DA19EA1AFA1B8A5A070B07006
:10040000A80EB91ECA1EDB1EA98EBA8ECB8EDC8E3C
:100410009A8C8B8C7C8C9E8D6F8D78A1FE01719651
:1004200088E0DF011D928A95E9F72D8B9E8B6F8BFB
:10043000788F2D853E854F8558896DA57EA58FA522
:1004400098A90E94156B7B018C012D813E814F8103
:10045000588569A57AA58BA59CA50E94156BE60E0B
:10046000F71E081F191F6D897E898F89988D6E0D63
:100470007F1D801F911F6D8B7E8B8F8B988FEE89D8
:100480002A2D392D482D572D7E2F8F89988DE09656
:10049000E2E10C94726BEF92FF920F93DF93CF9394
:1004A000CDB7DEB760970FB6F894DEBF0FBECDBFF5
:1004B000A82F002309F461C07E010894E11CF11CFF
:1004C00088E0F70111928A95E9F729833A834B83F3
:1004D0005C836D837E83AF83988780E2801BE82FE7
:1004E000FF27E7FDF0954D815E816F8178851816B5
:1004F00084F01D861E861F86188A882799278E1BE2
:100500009F0B04C076956795579547958A95D2F7C6
:1005100028C0202F332727FD3095DB01CA01022E8A
:1005200004C0B695A795979587950A94D2F78D87BD
:100530009E87AF87B88B04C0440F551F661F771F77
:10054000EA95D2F789819A81AB81BC8104C0B695C6
:10055000A795979587952A95D2F7482B592B6A2B03
:100560007B2B49875A876B877C8729853A854B8502
:100570005C856D857E85AF8598898A2F60960FB6DC
:10058000F894DEBF0FBECDBFCF91DF910F91FF90EA
:10059000EF900895EF92FF920F93DF93CF93CDB733
:1005A000DEB760970FB6F894DEBF0FBECDBFA82FA1
:1005B000002309F461C07E010894E11CF11C88E06D
:1005C000F70111928A95E9F729833A834B835C837B
:1005D0006D837E83AF83988780E2801BE82FFF279F
:1005E000E7FDF09549815A816B817C81181684F072
:1005F00019861A861B861C86882799278E1B9F0BB7
:1006000004C0440F551F661F771F8A95D2F728C074
:10061000202F332727FD3095DB01CA01022E04C0AD
:10062000880F991FAA1FBB1F0A94D2F789879A8740
:10063000AB87BC8704C07695679557954795EA9533
:10064000D2F78D819E81AF81B88504C0880F991F34
:10065000AA1FBB1F2A95D2F7482B592B6A2B7B2B3D
:100660004D875E876F87788B29853A854B855C85BA
:100670006D857E85AF8598898A2F60960FB6F89430
:10068000DEBF0FBECDBFCF91DF910F91FF90EF90F6
:100690000895DF93CF9300D0CDB7DEB7282F30E099
:1006A0002DC02E981A82198289819A8101969A8387
:1006B000898389819A8101979A8389832F9A1A82E3
:1006C000198289819A8101969A83898389819A8185
:1006D00001979A838983220F4E992F5F2F981A8250
:1006E000198289819A8101969A83898389819A8165
:1006F00001979A8389833F5F383021F027FFD1CF5C
:100700002E9AD0CF2E98822F0F900F90CF91DF91FD
:1007100008952F923F924F925F926F927F928F92A5
:100720009F92AF92BF92CF92DF92EF92FF920F9380
:100730001F93DF93CF9300D000D0CDB7DEB71C015D
:100740004A015B01C982DA82EB82FC82880C991C27
:10075000AA1CBB1C880C991CAA1CBB1C880C991CCD
:10076000AA1CBB1C089481089108A108B108801A32
:10077000910AA20AB30A8701760144245524320162
:10078000D501C40123E0B695A795979587952A953D
:10079000D1F7F101E80FF91F808190E0A5019401E4
:1007A0002095309540955095277002C09595879576
:1007B0002A95E2F78170907029813A812E193F09BC
:1007C00002C0880F991F2A95E2F7AA2797FDA095E6
:1007D000BA2F482A592A6A2A7B2A0894E108F10884
:1007E00001091109089481089108A108B108E114D0
:1007F000F1040105110521F6B201C3010F900F901C
:100800000F900F90CF91DF911F910F91FF90EF907C
:10081000DF90CF90BF90AF909F908F907F906F9020
:100820005F904F903F902F900895FC01848181FF4D
:1008300007C02081318142815381B901CA010895E5
:1008400020E030E040E050E0B901CA010895DF92B5
:10085000EF92FF920F931F93DF93CF9300D000D0BE
:1008600000D0CDB7DEB7222309F03FC08064898372
:10087000872F9927AA27BB278A83CB01AA27BB27C3
:100880008B83BB27A72F962F852F8C834D8380E0EA
:1008900015E0D12E7E010894E11CF11C8E838701A6
:1008A000F80181918F010E94EF00802F8E198D1524
:1008B000B8F38FEF0E94EF008F3F49F411E08FEF04
:1008C0000E94EF001F5F113811F08F3FC1F3269691
:1008D0000FB6F894DEBF0FBECDBFCF91DF911F9151
:1008E0000F91FF90EF90DF90089580648983872FA8
:1008F0009927AA27BB278A83CB01AA27BB278B83EB
:10090000BB27A72F962F852F8C834D837E010894BC
:10091000E11CF11CF70130E0BE016A5F7F4F49E046
:10092000208190E001C0220F330F832F822787FDA3
:1009300034279F5F9830B9F73196E617F70781F7AC
:10094000832F880F8160B6E0DB2EA8CFBF92CF92B5
:10095000DF92EF92FF920F931F93CF93DF93C82EF6
:10096000B62E662309F050C0EE24FF248701DD2453
:10097000D394C0E0D0E01EC087E340E050E060E0E8
:1009800070E021E00E94270487FD02C082FF35C08D
:1009900090E087FD1AC0DD2019F1BB2039F5E12C6C
:1009A000F12C30E2032F112D2196DD2487E2C03196
:1009B000D80759F0CC2001F781E0B801A70121E068
:1009C0000E94270490E087FFE6CF80E0DF91CF917F
:1009D0001F910F91FF90EF90DF90CF90BF900895FF
:1009E00081709070892B01F781E0F0CFE12CF12C20
:1009F00020E2022F20E4122FD7CF89E2B801A7010D
:100A000021E00E942704C4CFE12CF12C012D40E409
:100A1000142FADCF2F923F924F925F926F927F92A1
:100A20008F929F92AF92BF92CF92DF92EF92FF92FE
:100A30000F931F93CF93DF935C017A018B0188E0C2
:100A400089B9D5011496EC91E1FF56C0B901A8010E
:100A50009701F9E0220F331F441F551FFA95D1F774
:100A60006B01922E832E742E652E5E2C4F2C302E11
:100A7000212EE12C5AE0F52EE60EF71EE0FF37C0DE
:100A8000452D542D632D722D88E120E00E9427040E
:100A900087FD32C08FEF0E94EF008EEF0E94EF00C3
:100AA0008601C0E0D0E0F80181918F010E94EF0043
:100AB0002196F2E0C030DF07B1F780E092E0C80E87
:100AC000D91E8FEF0E94EF00182F8F3FD1F38FEFC9
:100AD0000E94EF008F3FD9F71F71153031F1CE140E
:100AE000DF04F9F0D5011496EC91E0FDC9CF492D52
:100AF000582D672D762DC8CF90E0892FDF91CF91AB
:100B00001F910F91FF90EF90DF90CF90BF90AF902B
:100B10009F908F907F906F905F904F903F902F901D
:100B2000089590E088E089B9E8CF91E0FBCFEF929B
:100B3000FF921F93CF93DF937C01EB0118EC04C06D
:100B40009E3F79F0115019F18FEF0E94EF00982F1E
:100B5000807FB1F7892FDF91CF911F91FF90EF90A8
:100B600008951123A1F0F7019083209741F08FEFB2
:100B70000E94EF00F70181937F012197C1F790E078
:100B8000892FDF91CF911F91FF90EF9008959FEFF4
:100B9000892FDF91CF911F91FF90EF9008957F9261
:100BA0008F929F92AF92BF92CF92DF92EF92FF927D
:100BB0000F931F93CF93DF93EC01790184E089B900
:100BC0002C8121FF30C0DB01CA0119E0880F991F79
:100BD000AA1FBB1F1A95D1F710E0782E892E9A2EE6
:100BE000AB2EB42EC52ED62E072F20FF17C04B2DAF
:100BF0005C2D6D2D702F81E120E00E94270487FD80
:100C000012C0C70160E072E00E9497058823F9F0E6
:100C10001F5F1530C1F02C8120FDE9CF472D582DE5
:100C2000692D7A2DE8CF90E0892FDF91CF911F9128
:100C30000F91FF90EF90DF90CF90BF90AF909F907B
:100C40008F907F90089590E084E089B9EDCF91E096
:100C5000FBCF2F923F924F925F926F927F928F9233
:100C60009F92AF92BF92CF92DF92EF92FF920F933B
:100C70001F93DF93CF93CDB7DEB766970FB6F89487
:100C8000DEBF0FBECDBF1C01DC0114968C91149702
:100C9000897F14968C931092000110E08FEF0E94D0
:100CA000EF001F5F1A30D1F700E010E01A821982BE
:100CB00089819A8101969A83898389819A81019792
:100CC0009A8389832E9A1A82198289819A81019640
:100CD0009A83898389819A8101979A8389832F9A3C
:100CE0001A82198289819A8101969A8389838981DE
:100CF0009A8101979A8389832F981A821982898110
:100D00009A8101969A83898389819A8101979A832E
:100D1000898380E040E050E060E070E021E00E94E4
:100D200027040F5F1F4FB2E009351B0709F45DC0B0
:100D3000813009F0BBCF88E04AEA51E060E070E022
:100D400021E00E94270487FD50C090E0969587958A
:100D50009695879501E010E0802791278170F10139
:100D600024812E7F282B248387E340E050E060E03D
:100D700070E021E00E94270487FD37C090E096953F
:100D8000879596958795802791278170880F880F82
:100D9000D10114962C9114972B7F282B14962C9309
:100DA00022FD3DC080E061E00E94A604882309F492
:100DB00044C08BE340E050E060E070E021E00E943E
:100DC000270487FD12C089E040E050E060E070E059
:100DD00020E00E94270487FD08C0CE01039660E151
:100DE00070E00E949705882379F180E066960FB63F
:100DF000F894DEBF0FBECDBFCF91DF911F910F9151
:100E0000FF90EF90DF90CF90BF90AF909F908F902A
:100E10007F906F905F904F903F902F90089581E06A
:100E200061E00E94A604882321F681E060E00E9430
:100E3000A604882309F0BDCFD8CF60E00E94A604A5
:100E4000882309F0B6CFD1CFF1018480CE0103967B
:100E500040E150E060E070E00EE710E020E030E0BC
:100E6000B2E0CB2ED12CE12CF12C0E94890361152C
:100E700071058105910541F082FC9BC063307105CD
:100E80008105910508F095C0CE01039640E150E040
:100E900060E070E00EE310E020E030E0ACE0CA2E4D
:100EA000D12CE12CF12C0E9489034B015C01CE0175
:100EB000039640E150E060E070E00FE210E020E0D7
:100EC00030E0F3E0CF2ED12CE12CF12C0E948903ED
:100ED0002B013C01CE01039640E150E060E070E060
:100EE00000E510E020E030E0E4E0CE2ED12CE12C53
:100EF000F12C0E94890381E090E0A0E0B0E004C002
:100F0000880F991FAA1FBB1F6A95D2F78B8B9C8BEA
:100F1000AD8BBE8B750164010894C11CD11CE11C12
:100F2000F11CA2E0B0E04A0E5B1E04C0CC0CDD1C3C
:100F3000EE1CFF1C4A94D2F709E010E020E030E0FC
:100F40008B899C8981709070892B09F03CC08B89BA
:100F50009C89AD89BE89B695A795979587958B8B0A
:100F60009C8BAD8BBE8B015010402040304041F730
:100F700000E010E0C701B6012B893C894D895E89EC
:100F80000E94156B04C096958795779567950A958D
:100F9000D2F7D1016D937D938D939C931397149603
:100FA0008C911497826014968C9381E08093000159
:100FB0001DCF6130710581059105F9F060E070E0A9
:100FC00080E090E0E6CF011511052105310581F2A1
:100FD000C60181709070892B31F0CCCFC601817031
:100FE0009070892B39F6F694E794D794C794015002
:100FF00010402040304091F7BBCFCE01039640E136
:1010000050E060E070E000E310E020E030E0E6E176
:10101000CE2ED12CE12CF12C0E9489030AE0660F20
:10102000771F881F991F0A95D1F7B3CF8091C00011
:1010300087FD04C02EEF3FEFC90108958091C600DF
:10104000282F30E0C9010895982F8091C00085FFB6
:10105000FCCF9093C60008951F920F920FB60F9287
:1010600011242F938F939F93AF93BF93209180056B
:10107000222399F08091C13B9091C23BA091C33B48
:10108000B091C43B0196A11DB11D8093C13B9093CB
:10109000C23BA093C33BB093C43B81E0282720937D
:1010A0008005BF91AF919F918F912F910F900FBEAF
:1010B0000F901F901895FC019081992371F08091F9
:1010C000C00085FFFCCF892F992787FD90958093DD
:1010D000C60091813196992391F708952091C13BE3
:1010E0003091C23B4091C33B5091C43B8091C13B86
:1010F0009091C23BA091C33BB091C43B28173907E4
:101100004A075B0759F7B901CA0108959F92AF9248
:10111000BF92CF92DF92EF92FF920F931F93CF93E4
:10112000DF935A016B01922EE701002301F599200C
:1011300079F481E0DF91CF911F910F91FF90EF90B3
:10114000DF90CF90BF90AF909F90089557016801B6
:10115000860175010894E11CF11C011D111DC601D9
:10116000B5010E94040189939A9481F7E2CF9920F6
:1011700019F4DFCF57016801860175010894E11C5D
:10118000F11C011D111D4991C601B5010E942001EC
:101190009A9481F7CECF1F93F894F894A89598E18C
:1011A0000FB6F89490936000109260000FBE85B760
:1011B000806885BF85BF1092C5003CE03093C400B5
:1011C0001092C00086E08093C2009093C10082ED2F
:1011D0009AE59093890080938800109280008BE0BC
:1011E0008093810022E020936F008FEF81B984B15A
:1011F0008F6384B9579A17B812B885B1807F85B9C3
:1012000085B1806385B95F9A18B884E197E7A6E64F
:10121000BFE48093C13B9093C23BA093C33BB09388
:10122000C43B8BE197EB90939900809398001092C8
:10123000900030939100209371008AB18C608AB93C
:10124000569884B1806C84B98BB1837F8BB985B19A
:101250008F7385B954985C9A80EB94E00197F1F70D
:1012600010E00E943D011F5F1830D9F778941F915C
:1012700008952F923F924F925F926F927F928F923A
:101280009F92AF92BF92CF92DF92EF92FF920F9315
:101290001F93DF93CF9300D000D00F92CDB7DEB76E
:1012A0000E94CB081E010894211C311CC1010E9420
:1012B0002906882391F493E7E5E2F1E08091C000EC
:1012C00085FFFCCF892F992787FD90958093C600D5
:1012D0009081992311F03196F1CF81E895E06BEA86
:1012E00073E546E858E026E138E004E218E0B8ED9E
:1012F000EB2EB9E0FB2E61010E94CF514C994FC0FB
:10130000812C912CA0EEAA2EA0EABA2E40E250E049
:101310006CE070E02A013B010894411C511C611CE7
:10132000711CC10129E835E00E94CF05F9E8CF2EF4
:10133000F5E0DF2EC501B4017B018C010894E11CAE
:10134000F11C011D111DD6014D916D010E9420015E
:10135000C801B701B9E8CB16B7E0DB0669F780E052
:1013600092E0A0E0B0E0880E991EAA1EBB1E90E29B
:10137000491690E159069CE0690690E0790619F05B
:10138000B301A201C7CF80E092E0A0EEB0EA809363
:10139000D9079093DA07A093DB07B093DC0781E8C5
:1013A00095E040E050E060E070E00E94C850FFCF60
:1013B0000F93CF93DF93E9010130D9F0013048F06A
:1013C000023009F120E030E0C901DF91CF910F91A7
:1013D00008954115510561057105F9F4009769F10A
:1013E0000E941504688379838A839B8321E030E01F
:1013F000EBCF9E010E94CF05282F30E0C901DF917D
:10140000CF910F9108959E010E940A05282F30E088
:10141000C901DF91CF910F910895413051056105C8
:10142000710581F680E092E0A0E0B0E088839983C6
:10143000AA83BB8321E030E0C7CF188219821A82C9
:101440001B8221E030E0C0CF6115710529F0FC015D
:10145000119261507040E1F70895EF92FF920F935F
:101460001F93CF93DF93EC0179018A012115310598
:1014700041055105E9F020E030E040E050E0EE2782
:10148000FF27E21BF30BDE01AE0FBF1FE60FF71FB6
:1014900080818C932150304040405040DA01C90196
:1014A0008E0D9F1DA01FB11F0097A105B10539F733
:1014B000DF91CF911F910F91FF90EF900895AF9220
:1014C000BF92CF92DF92EF92FF920F931F93DF9321
:1014D000CF93CDB7DEB760970FB6F894DEBF0FBEDF
:1014E000CDBF6B017C01188A8FE0A82EB12CAC0E09
:1014F000BD1E00E0C701B6012AE030E040E050E048
:101500000E94346B162F105DC701B6012AE030E04F
:1015100040E050E00E94346BC901DA016C017D01AA
:10152000F5011083C114D104E104F10431F00F5F1F
:101530000894A108B1080F30E9F62EE030E0201B36
:101540003109CE010196820F931F0E945B086096BD
:101550000FB6F894DEBF0FBECDBFCF91DF911F91C4
:101560000F91FF90EF90DF90CF90BF90AF900895D4
:10157000DF93CF93CDB7DEB729970FB6F894DEBFD0
:101580000FBECDBF1986FE01389606C0295C2083A8
:101590003197EC17FD0789F0262F2F7034E09695D0
:1015A0008795779567953A95D1F72A3078F7205D3A
:1015B00020833197EC17FD0779F7CE0101960E9441
:1015C0005B0829960FB6F894DEBF0FBECDBFCF9152
:1015D000DF910895DC01603188F46F30D1F0E62F9F
:1015E000F0E0EE0FFF1FEE0FFF1FEA0FFB1F208141
:1015F000318142815381B901CA010895603151F1AD
:10160000613189F120E030E040E050E0B901CA01E9
:101610000895A05CBF4F2D913D914D915C91139722
:10162000A054B04095E056954795379527959A95E3
:10163000D1F72170307040705070DC968D919D9183
:101640000D90BC91A02D280F391F4A1F5B1FB901B7
:10165000CA010895A05CBF4F2D913D914D915C91C1
:10166000B901CA010895AC5BBF4F2D913D914D91D9
:101670005C91B901CA010895EF92FF920F931F93F5
:10168000CF93DF93EC0179018A016F3099F0E62F57
:10169000F0E0EE0FFF1FEE0FFF1FE80FF91FE082D3
:1016A000F18202831383DF91CF911F910F91FF90FD
:1016B000EF900895DA01C9018E7F8CAF9DAFAEAF78
:1016C000BFAFFE01E05CFF4F208131814281538139
:1016D0002F7D2083318342835383C70181709070B3
:1016E000892B69F4E1FEDFCFC05BDE4FE881F98131
:1016F000C055D140CE0163E371E00995D4CF20629B
:101700002083318342835383DF91CF911F910F91C7
:10171000FF90EF900895DC016331B1F16431A8F0DE
:101720006B3141F16F31E1F06731F9F0A05BBE4FF1
:10173000ED91FC911197A055B140CD0165E671E0A6
:101740000995E0E0F0E0CF0108956131C1F0623128
:1017500028F0FC01E858FF4FCF010895603131F7C0
:10176000FD01E85BFF4FCF010895FC01E05AFF4FF8
:10177000CF010895FC01E459FF4FCF010895FC010A
:10178000EC57FF4FCF010895FC01EC5AFF4FCF01FA
:101790000895DF92EF92FF920F931F93CF93DF9301
:1017A0008C01D62E30E4E32EF12CE80EF91EE70171
:1017B00068816F716D1509F45FC0613109F464C00F
:1017C000E1E1DE1609F460C0C8010E948B0BEC0158
:1017D000C8016D2D0E948B0B9C01C817D90709F415
:1017E0004BC0F80184A995A9A6A9B7A988839983B4
:1017F000AA83BB8380AD91ADA2ADB3AD8C839D8335
:10180000AE83BF83EC5BFF4F80819181A281B38166
:1018100088879987AA87BB87E90188819981AA81EE
:10182000BB81E8018CAB9DABAEABBFABE9018C815A
:101830009D81AE81BF81E80188AF99AFAAAFBBAFF0
:10184000E90188859985AA85BB8580839183A283D8
:10185000B3832D2D30E040E050E0F701808191818D
:10186000A281B381807E282B392B4A2B5B2BE70189
:10187000288339834A835B83DF91CF911F910F9136
:10188000FF90EF90DF900895E801C057DF4FF80117
:1018900070E0288139814A815B8180A191A1A2A158
:1018A000B3A189939993A993B99320A331A342A398
:1018B00053A37F5F3496753061F786CF2F923F92A6
:1018C0004F925F926F927F928F929F92AF92BF9250
:1018D000CF92DF92EF92FF920F931F93DF93CF93FC
:1018E000CDB7DEB72A970FB6F894DEBF0FBECDBFD7
:1018F0008C5A9E4FDC01ED91FC911197A455B1409B
:10190000BA87A987309719F0CD012C2D0995EE20C3
:1019100009F090C0E985FA85E65BFE4F20803180B2
:1019200042805380EA54F140FA87E98784AD95AD4F
:10193000A6ADB7AD89839A83AB83BC83E05CFF4FD0
:10194000F887EF83A080B180C280D380A5FC6CC0F3
:1019500064E0662E712C812C912C40E6E42E4FEF32
:10196000F42E4FEF042F4FEF142FEA20FB200C2111
:101970001D2187E990E0A0E0B0E0E82AF92A0A2BCF
:101980001B2B6E2D6F7189859A850E94C90BAF81C3
:10199000B885ED92FD920D931C931397E985FA8516
:1019A000EC5BFF4FDF01A082B182C282D382A454DC
:1019B000B040BA87A98789819A81AB81BC81680EC2
:1019C000791E8A1E9B1EA985BA85D8966D927D9236
:1019D0008D929C92DB9780E190E0A0E0B0E0280E31
:1019E000391E4A1E5B1EA985BA85DC962D923D9252
:1019F0004D925C92DF972A960FB6F894DEBF0FBE29
:101A0000CDBFCF91DF911F910F91FF90EF90DF90AD
:101A1000CF90BF90AF909F908F907F906F905F908E
:101A20004F903F902F90089556E0652E712C812C99
:101A3000912C93CFE985FA85E65BFE4F608071803B
:101A400082809380EA54F140FA87E9878CE090E045
:101A5000A0E0B0E0680E791E8A1E9B1EA4ACB5AC57
:101A6000C6ACD7AC84E090E0A0E0B0E0A80EB91E10
:101A7000CA1EDB1EE05CFF4FFE83ED8320803180B9
:101A80004280538070E6E72E7FEFF72E7FEF072F1F
:101A90007FEF172FE220F3200421152187E990E042
:101AA000A0E0B0E0E82AF92A0A2B1B2B6E2D6F71FB
:101AB00089859A850E94C90BAD81BE81ED92FD9208
:101AC0000D931C931397E985FA85EC5BFF4FDF01BB
:101AD0002082318242825382A454B040BA87A987BF
:101AE000FD01A0AEB1AEC2AED3AEDC966D927D92DA
:101AF0008D929C92DF977FCFDC01662369F04423AF
:101B000049F5FC01EA55FF4F80819181009759F119
:101B10000197918380830895442399F4FC01EC5547
:101B2000FF4F80819181009799F7A05BBE4FED91A7
:101B3000FC911197A055B140CD016CEB71E0099576
:101B40000895FC01EC55FF4F8081918101969183AE
:101B500080830895FC01EA55FF4F808191810196B1
:101B6000918380830895A05BBE4FED91FC91119706
:101B7000A055B140CD0168E971E009950895262F7F
:101B800030E0F901EE0FFF1FEE0FFF1FEE0FFF1FFA
:101B9000220F331FE20FF31FE80FF91FE655FF4F27
:101BA000DA018AE00D9001928150E1F70895FC017D
:101BB000E65BFE4F40835183628373830895FC018B
:101BC000E855FF4F808191810895FC01E855FF4F52
:101BD0007183608308958A5A9E4F0E94D05508955C
:101BE0008A5A9E4F0E945E5508952F923F924F92BF
:101BF0005F926F927F928F929F92AF92BF92CF929D
:101C0000DF92EF92FF920F931F93DF93CF93CDB7A5
:101C1000DEB7C557D0400FB6F894DEBF0FBECDBFBC
:101C200062969FAF8EAF629766964CAF5DAF6EAF18
:101C30007FAF66976A960CAF1DAF2EAF3FAF6A9726
:101C40006B96EFAE6B976C96CFAE6C976D96AFAE12
:101C50006D97805C9F4FE0969FAF8EAFE097DC0161
:101C6000AD90BD90CD90DC90D601C5018F71907084
:101C7000A070B07080319105A105B10509F473C160
:101C80001EAA4F97A105B10509F46AC166968CADED
:101C90009DADAEADBFAD66977DE1B695A795979525
:101CA00087957A95D1F783309105A105B10509F49F
:101CB0009FC784309105A105B10508F433C1853073
:101CC0009105A105B10509F4A9C785309105A105C4
:101CD000B10508F44BC186309105A105B10509F4A1
:101CE000C7C70797A105B10509F4ADC766960CAD46
:101CF0001DAD2EAD3FAD6697007010702070307135
:101D000040E080E0011511052105310539F044233B
:101D100029F490E0882309F491E0892F882309F4BD
:101D2000E6C066964CAC5DAC6EAC7FAC6697872D1A
:101D30009927AA27BB278F709070A070B070883049
:101D40009105A105B10508F06AC286309105A1058B
:101D5000B10508F4D9C463963FAC639734FE35C12E
:101D600066960CAD1DAD2EAD3FAD66970B5B1B4B64
:101D70002B4B374FE1F46C965FAD6C975523B9F060
:101D800062966EAD7FAD62976E5A7E4FDB01ED912C
:101D9000FC911197A255B1406296BFAFAEAF62976A
:101DA000309729F0CD010995882309F0A0C080EE75
:101DB00091E00E945B0866966CAD7DAD8EAD9FADE7
:101DC00066970E94B80A81EF91E00E945B086A96CC
:101DD0006CAD7DAD8EAD9FAD6A970E94B80A8DEF58
:101DE00091E00E945B08E096EEADFFADE097608168
:101DF0007181828193810E94B80A87E092E00E94FB
:101E00005B0862960EAD1FAD6297065B1E4FD80150
:101E10002D903D904D905C901397AA54B1406296DE
:101E2000BFAFAEAF62976B96BFAD6B97BB2309F0A8
:101E3000AFC2B4E06B2E712C812C912CE096EEADEC
:101E4000FFADE097E080F18002811381F0E6AF2ED4
:101E5000FFEFBF2EFFEFCF2EFFEFDF2EAE20BF2014
:101E6000C022D1222BE930E040E050E0A22AB32A80
:101E7000C42AD52A6A2D6F7162968EAD9FAD629786
:101E80000E94C90BE096AEADBFADE097AD92BD929A
:101E9000CD92DC9213976296EEADFFAD6297EC5B4C
:101EA000FF4FDF01E082F18202831383A454B0402C
:101EB0006A96ACACBDACCEACDFAC6A976A0C7B1C4E
:101EC0008C1C9D1CD8966D927D928D929C92DB9776
:101ED000E4E06E2E712C812C912C260C371C481CB2
:101EE000591CDC962D923D924D925C92DF9780E0DA
:101EF000CB58DF4F0FB6F894DEBF0FBECDBFCF91EA
:101F0000DF911F910F91FF90EF90DF90CF90BF90E6
:101F1000AF909F908F907F906F905F904F903F9089
:101F20002F90089581309105A105B10509F44AC6A5
:101F30000297A105B10598F1D601C5018827B7FD23
:101F400083959927AA27BB2766960CAD1DAD2EADAC
:101F50003FAD6697007010702070307140E0D2CEB7
:101F6000E1E0EEAB93CEB1E0BEAB90CED5FE28C69D
:101F7000D601C5012EE1B695A795979587952A9527
:101F8000D1F78095817066960CAD1DAD2EAD3FAD3D
:101F90006697007010702070307140E0B3CED601AB
:101FA000C5016EE1B695A795979587956A95D1F786
:101FB000817066960CAD1DAD2EAD3FAD669700707D
:101FC00010702070307140E09DCE442311F00C94CD
:101FD000741866962CAD3DAD4EAD5FAD6697CA01E7
:101FE000AA27BB27BFE0FB2EF82251FF02C00C94AA
:101FF000221939014A014FEF5FE060E070E064228E
:1020000075228622972266960CAD1DAD2EAD3FAD92
:10201000669726FD02C010E1F12A66962CAD3DAD13
:102020004EAD5FAD669744FF02C030E2F32A66967C
:102030004CAD5DAD6EAD7FAD669767FD08C0909409
:10204000809470946094611C711C811C911C669634
:102050006CAD7DAD8EAD9FAD669790FF02C00C94C8
:1020600014191B821C821D821E8285FF02C070E42F
:10207000F72A2B813C814D815E81F7FC71CE1F2DAB
:10208000F6FE03C06C961FAE6C9714FF02C00C9452
:102090005F1ADD24D3949F2D9F709BA3A92FB0E0DE
:1020A000AA0FBB1FAA0FBB1FAC96BFAFAEAFAC97BA
:1020B0006296EEADFFAD6297EA0FFB1F2080318084
:1020C000428053809F3011F40C94801B6B96FFADBF
:1020D0006B97FF2369F06D96AFAC6D97AA2041F026
:1020E0006CEF7FEF8FEF9FEF262237224822592295
:1020F00015FF02C00C94901B6114710481049104BB
:1021000011F00C94721B1DA61EA61FA618AA320160
:102110002101420E531E641E751E81E0D81611F473
:102120000C943B1F66960CAD1DAD2EAD3FAD669772
:102130004CE036952795179507954A95D1F7669601
:102140000CAF1DAF2EAF3FAF669763968FAD639711
:102150008F70E82FF0E0EE0FFF1FEE0FFF1F62966B
:102160002EAD3FAD6297E20FF31F20813181428196
:1021700053818F3011F40C9404206B967FAD6B97D4
:10218000772329F06D968FAD6D9781112C7F2B836E
:102190003C834D835E8303E0802E912C8C0E9D1E2C
:1021A0006296AEADBFAD6297A25BBE4FED91FC9162
:1021B0001197AE54B1406296BFAFAEAF6297CD01FA
:1021C000B401A30192010D2DEE24E3946C96CFACE3
:1021D0006C975E010894A11CB11C0995882311F429
:1021E0000C948C1FF7FE83CE8F2D8F708F3011F4DF
:1021F0000C94AC29E82FF0E0EE0FFF1FEE0FFF1F4D
:1022000062962EAD3FAD6297E20FF31F4DA55EA51E
:102210006FA578A9408351836283738368CE8C3025
:102220009105A105B10508F0B9C00A97A105B1054E
:1022300008F40BC666968CAD9DADAEADBFAD66978E
:10224000B07066962CAC3DAC4EAC5FAC669747FC6C
:10225000BF6F6B963FAC6B97332009F058C78C016A
:102260009D01000F111F221F331F000F111F221F7E
:10227000331F88E090E0A0E0B0E078018901E80E2B
:10228000F91E0A1F1B1F6A964CAC5DAC6EAC7FAC8E
:102290006A97E40CF51C061D171D442309F46BC74F
:1022A00066966CAC7DAC8EAC9FAC669790FE09C018
:1022B00082E0882E912CA12CB12CE80CF91C0A1D6F
:1022C0001B1D6B969FAC6B97992011F00C94DA1A3A
:1022D00084E090E0A0E0B0E06A96ACACBDACCEACDF
:1022E000DFAC6A978A0D9B1DAC1DBD1D6296EEADDD
:1022F000FFAD629780AF91AFA2AFB3AFE096AEAD46
:10230000BFADE0978C9185FD09C0B1E02B2E312C3B
:10231000412C512CE228F32804291529D801C701A2
:102320008E7F6296EEADFFAD629784AF95AFA6AF9C
:10233000B7AFE096AEADBFADE0972D913D914D9119
:102340005C9113972F7DFD0120833183428353835A
:10235000C70181709070892B09F005C7E1FEC7CDD8
:102360006296EEADFFAD6297E05BFE4F6296FFAF07
:10237000EEAF62970190F081E02D62960EAD1FAD39
:10238000629700551140C80163E371E00995AFCD34
:10239000A2E06A2E712C812C912C50CD8E309105AB
:1023A000A105B10509F490C48E309105A105B105D0
:1023B00008F478C00F97A105B10509F0D1CC4423EA
:1023C00009F0CECC62960EAD1FAD6297065B1E4F34
:1023D000D8012D903D904D905C901397AA54B14038
:1023E0006296BFAFAEAF62976B96BFAD6B97BB23E4
:1023F00011F00C94ED1A24E0622E712C812C912C9A
:1024000080E6E82E8FEFF82E8FEF082F8FEF182F32
:10241000EA20FB200C211D2123E930E040E050E0C0
:10242000E22AF32A042B152B6E2D6F7162968EAD66
:102430009FAD62970E94C90BE096AEADBFADE0972D
:10244000ED92FD920D931C9313976296EEADFFAD46
:102450006297EC5BFF4FDF01A082B182C282D38220
:10246000A454B0406A96ACACBDACCEACDFAC6A97BD
:102470006A0C7B1C8C1C9D1CD8966D927D928D9253
:102480009C92DB9718E0612E712C812C912C260CEC
:10249000371C481C591CDC962D923D924D925C9243
:1024A000DF9725CD66960CAD1DAD2EAD3FAD669781
:1024B00010702070307066962CAC3DAC4EAC5FACAA
:1024C0006697C201AA27BB27FFE09F2E982250FEE5
:1024D00031C6592D50616696ACACBDACCEACDFAC0C
:1024E0006697C5FE02C0592D5063252E3324E0E4C3
:1024F000AE2EB12CA220B32056FD17C0000F111F25
:10250000221F331F000F111F221F331F6696CCACF2
:10251000DDACEEACFFAC6697E7FC07C030952095CC
:10252000109501951F4F2F4F3F4F0B831C832D8319
:102530003E8366964CAC5DAC6EAC7FAC6697BB27B9
:10254000A72D962D852D682F6F706E3008F442C62A
:102550006C965FAC6C97552009F402CC57FF02C013
:102560000C94F31D0A835F70598F452E5524440C3B
:10257000551C440C551CA8965FAE4EAEA8976296AB
:10258000EEADFFAD6297E40DF51DC080D180E28015
:10259000F3805F3011F40C947C1F6B967FAC6B97CB
:1025A000772069F06D968FAC6D97882041F08CEFA5
:1025B0009FEFAFEFBFEFC822D922EA22FB22862F7E
:1025C00090E0FC01EE0FFF1FEE0FFF1FEE0FFF1F4D
:1025D000880F991FE80FF91F6296AEADBFAD6297E5
:1025E000EA0FFB1FE255FF4F408051802C965FAEF3
:1025F0004EAE2C97452809F4B3CB26013701400E87
:10260000511E621E731E862F90E0FC01EE0FFF1F0D
:10261000EE0FFF1FEE0FFF1F880F991FE80FF91F26
:10262000EA0FFB1FEE54FF4F6081718124FE02C050
:102630000C94EB1DFC2D6E96DFAE6E975E2DEF2D8C
:10264000AB2811F00C94E71DA0E0B0E066960CAD4D
:102650001DAD2EAD3FAD669786E136952795179552
:1026600007958A95D1F701706696CCACDDACEEACDF
:10267000FFAC669794E1F694E794D794C7949A9543
:10268000D1F7C09488248394C82066968CAC9DAC06
:10269000AEACBFAC66978CE0B694A7949794879441
:1026A0008A95D1F71FE0D12E8D2062968EAD9FAD19
:1026B0006297202F0C2DE82CAF2E6E96BFAC6E9734
:1026C000C52EDE2E4D012C96AEADBFAD2C97FD0173
:1026D0000995882309F444CB25FE09CCB98DBF3078
:1026E00011F40C940F2A62962EAD3FAD6297A89616
:1026F0004EAD5FADA897240F351FD9014D925D9265
:102700006D927C921397F3CB84309105A105B105AE
:1027100008F05BCC0297A105B10508F478C1442309
:1027200009F01ECB66968CAD9DADAEADBFAD669784
:1027300080709070A079B17080509040A040B140FE
:1027400011F40C94161D66968CAD9DADAEADBFAD6B
:10275000669764E1B695A795979587956A95D1F7A1
:10276000782F717022967FAF2297D601C5015CE168
:10277000B695A795979587955A95D1F7E82FE1706B
:102780002396EFAF2397D601C5014DE1B695A795E6
:10279000979587954A95D1F7182F117066962CACAE
:1027A0003DAC4EAC5FAC669751FEB5C5D201C101E0
:1027B00037E0B695A795979587953A95D1F7282F45
:1027C0002E71420131014FEF50E060E070E0642271
:1027D000752286229722222309F46DC630E0B401C7
:1027E000A301022E04C076956795579547950A94E4
:1027F000D2F780E290E0821B930B04C0660C771C3A
:10280000881C991C8A95D2F7642A752A862A972AE9
:10281000D401C3018827B7FD83959927AA27BB2731
:1028200024968FAF249766964CAD5DAD6EAD7FADAF
:102830006697CB01AA27BB27682F6F7066962CADD1
:102840003DAD4EAD5FAD669705E156954795379521
:1028500027950A95D1F72F7030704070507027304F
:1028600031054105510511F40C94C227283031057A
:102870004105510508F0B8C6233031054105510521
:1028800011F40C94D328243031054105510510F082
:102890000C947D22213031054105510511F40C9431
:1028A0000C29223031054105510510F40C944627BE
:1028B000E62FF0E0EE0FFF1FEE0FFF1F6296EEAC6B
:1028C000FFAC6297EE0DFF1DE080F1800281138165
:1028D0006F3011F40C9464316B963FAD6B973323DA
:1028E00069F06D964FAD6D97442341F06CEF7FEF2B
:1028F0008FEF9FEFE622F722082319231701280103
:10290000261837084808590822967FAD2297772362
:1029100011F40C940E2FD201C1018E259F25A02702
:10292000B127A80197012625372548255925822357
:102930009323A423B5238827B7FD83959927AA2736
:10294000BB2723968FAF239724961FAE2497E614B8
:10295000F7040805190520F081E024968FAF24972D
:1029600081E06696ECACFDAC0EAD1FAD66974CE019
:1029700016950795F794E7944A95D1F76696ECAECD
:10298000FDAE0EAF1FAF669763960FAD63970F70E6
:10299000420131014EA8442021F40F3011F40C946F
:1029A000D523A60195015F7061147104810491041F
:1029B00011F00C94251F50642496FFAD2497F1115B
:1029C000506223962FAC239721105061E096AEAD54
:1029D000BFADE0972D933D934D935C931397882360
:1029E00009F485CA0F3011F40C949D1FE02FF0E01C
:1029F000EE0FFF1FEE0FFF1F62962EAC3FAC6297EB
:102A0000E20DF31D608271828282938270CA442338
:102A100009F0A6C966962CAD3DAD4EAD5FAD66978B
:102A200020793070407050702039310541055105D2
:102A300009F4FCC666968CAD9DADAEADBFAD669794
:102A400080709070A079B17080509040A040B140EB
:102A500009F079CE66968CAD9DADAEADBFAD6697F3
:102A600064E0B695A795979587956A95D1F78F708D
:102A70009070A070B07085309105A105B10511F47A
:102A80000C94862D86309105A105B10510F00C94AB
:102A9000F92581309105A105B10561F081309105DD
:102AA000A105B10510F40C94252D0397A105B105DE
:102AB00009F056C966962CAC3DAC4EAC5FAC66973F
:102AC00046FC02C00C946032D201C101807F9F702D
:102AD000BF7080519F40AF46B14009F041C9639635
:102AE0008FAD63978F70E82FF0E0EE0FFF1FEE0FB2
:102AF000FF1F62962EAD3FAD6297E20FF31FE0809D
:102B0000F180028113818F3011F40C94773B6B9626
:102B10004FAD6B97442369F06D965FAD6D9755236C
:102B200041F06CEF7FEF8FEF9FEFE622F722082353
:102B3000192320E030E040E050E860E007C06F5F1C
:102B4000603271F05695479537952795DA01C9019E
:102B50008E219F21A023B1230097A105B10579F310
:102B600066968CAD9DADAEADBFAD66973CE0B695BB
:102B7000A795979587953A95D1F766968CAF9DAFB7
:102B8000AEAFBFAF669763960FAD63970F70C62E5B
:102B9000DD24EE24FF240F3011F40C94FB2BE02FE6
:102BA000F0E0EE0FFF1FEE0FFF1F62962EAD3FAD60
:102BB0006297E20FF31FC082D182E282F38297C94B
:102BC00080E0E1C9D601C5015DE1B695A79597956D
:102BD00087955A95D1F7817066960CAD1DAD2EADD7
:102BE0003FAD6697007010702070307140E08AC869
:102BF000D601C5013CE1B695A795979587953A957D
:102C0000D1F7817066960CAD1DAD2EAD3FAD6697C8
:102C1000007010702070307140E074C8A6019501FA
:102C2000222757FD2395332744275527D601C50171
:102C30001CE1B695A795979587951A95D1F780953C
:102C400081708227A0C940E066960CAD1DAD2EAD07
:102C50003FAD6697007010702070307166962CAC96
:102C60003DAC4EAC5FAC669754FC41E081E04AC895
:102C7000A6019501222757FD239533274427552781
:102C8000D601C501FCE1B695A79597958795FA956C
:102C9000D1F741E050E060E070E084279527A62757
:102CA000B7278170821709F48BCFD601C501EEE1F9
:102CB000B695A79597958795EA95D1F78427952797
:102CC000A627B72781705FC966962CAC3DAC4EAC89
:102CD0005FAC6697BB27A52D942D832D282F2F70D1
:102CE0002E3008F01FC262960EAD1FAD62970855D8
:102CF0001F4FD8018D919C911197A85AB0406296B0
:102D0000BFAFAEAF6297A0E0B0E0022E04C0B695B0
:102D1000A795979587950A94D2F781709070892B23
:102D200009F41EC86396BFAD6397B4FFCCC3822F6E
:102D300090E0FC01EE0FFF1FEE0FFF1FEE0FFF1FD5
:102D4000880F991FE80FF91F62962EAC3FAC62976F
:102D5000E20DF31DE655FF4F408051802A965FAE8D
:102D60004EAE2A97452811F40C94B00E822F90E0B5
:102D7000FC01EE0FFF1FEE0FFF1FEE0FFF1F880F6E
:102D8000991FE80FF91FE20DF31DEE54FF4F60810C
:102D9000718166968CAD9DADAEADBFAD669724E1F9
:102DA000B695A795979587952A95D1F7282F2170E5
:102DB0006696ECACFDAC0EAD1FAD669785E1169541
:102DC0000795F794E7948A95D1F717E0512EE520FF
:102DD00066962CAC3DAC4EAC5FAC6697BCE05694AE
:102DE000479437942794BA95D1F7AFE06A2E2620FE
:102DF00066968CAD9DADAEADBFAD66975D01CC2442
:102E0000DD24A62063963FAD63973F703C014D01E2
:102E1000E5E09694879477946794EA95D1F797E0E4
:102E2000692262968EAD9FAD62970E2DE22CCA2C60
:102E3000A32E862C2A96AEADBFAD2A97FD0109952B
:102E4000882311F40C94B00E52C8442311F00C9452
:102E5000B00E66962CAC3DAC4EAC5FAC6697C20132
:102E6000AA27BB27AFE0FA2EF82246FE03C0F0E8FF
:102E70003F2EF32866964CAC5DAC6EAC7FAC66978B
:102E800065FE03C0E0E45E2EF52866966CAC7DAC72
:102E90008EAC9FAC669787FE03C070E1772EF72853
:102EA00066968CAC9DACAEACBFAC6697B0FE03C072
:102EB00060E2962EF928F7FC05C766968CAD9DADAD
:102EC000AEADBFAD669754E1B695A795979587953A
:102ED0005A95D1F7DD24D394D8220F2D0F700E8F81
:102EE000202F30E0220F331F220F331FAA963FAF4F
:102EF0002EAFAA976296EEADFFAD6297E20FF31F79
:102F00004081518162817381498B5A8B6B8B7C8BA1
:102F10000F3009F47BC76B963FAC6B97332071F091
:102F20006D964FAC6D97442049F009891A892B8919
:102F30003C890C7F098B1A8B2B8B3C8B64962EADB6
:102F40003FAD649738AF2FABDD2011F0F7FCF7C031
:102F50001DAA1A828F2D90E09CAB8BAB8071907074
:102F6000988B8F87AFA9B8AD1D0144245524629674
:102F7000EEADFFAD6297E85BFF4FFD8FEC8F629681
:102F80000EAD1FAD6297045B1F4F1B8F0A8F6988C0
:102F90007A888B889C8820E04BA95CA9407250708D
:102FA000E4965FAF4EAFE49762966EAD7FAD6297E9
:102FB000625B7E4FE6967FAF6EAFE6974BC0F7FC45
:102FC0002AC1E4960EAD1FADE497012B69F02F8561
:102FD0003889232B09F0BDC08CEF9FEFAFEFBFEF17
:102FE000680E791E8A1E9B1E10E0DD2009F411E098
:102FF000E696AEADBFADE697ED91FC9162968EADD3
:103000009FAD6297A401930104E0E12E6C96CFACD2
:103010006C975E010894A11CB11C0995882309F4E2
:103020008CC6E496EEADFFADE497EF2B69F4AF8468
:10303000B888AB2809F092C08CEF9FEFAFEFBFEFDD
:10304000680E791E8A1E9B1E2A812F5F2A832031DB
:1030500008F0E5C18F859889892B19F49FE0921BB0
:10306000292FD201C101022E04C0B695A7959795CC
:1030700087950A94D2F781709070892B29F3422F9B
:1030800050E0BA01660F771F660F771F6296AEADEC
:10309000BFAD62976A0F7B1FDD2009F090CFF7FE6E
:1030A00090CFBEA8BB2009F08CCF822F88508530EE
:1030B00090F4E096EEADFFADE09780819181A28122
:1030C000B3818F719070A070B0704197A105B10568
:1030D00011F40C94FD222D3009F42CC72E3009F088
:1030E00070CF6A8D7B8D6DCF66968CAD9DADAEAD8C
:1030F000BFAD66978070907FA077BD708050904F75
:10310000A045B54011F00C94B00E0C94770F8C01D3
:103110009D01000F111F221F331F84E090E0A0E0EB
:10312000B0E0ABC86C963FAC6C97332011F40C94B4
:10313000B00EF8CD45FE44C2592D5062D6C937FFB6
:1031400007CF1DAA5EA9552309F003CF61E06DAB3F
:1031500000CF84E090E0A0E0B0E042CF84E090E0D7
:10316000A0E0B0E06DCF20622D933D934D935C9332
:1031700013970C94770F66964CAC5DAC6EAC7FAC3D
:10318000669770FE24C06B965FAC6B97552009F074
:1031900054C684E090E0A0E0B0E06A966CAC7DACF0
:1031A0008EAC9FAC6A97860D971DA81DB91D6296BF
:1031B000EEADFFAD629780AF91AFA2AFB3AFE09637
:1031C000AEADBFADE097AD90BD90CD90DC90A5FECB
:1031D000A5C89BC862968EAD9FAD629788559F4FDC
:1031E000DC018D919C911197A85AB0406296BFAFB7
:1031F000AEAF6297A0E0B0E0062E04C0B695A795EA
:10320000979587950A94D2F781709070892B11F465
:103210000C94B00EA3C9EFA9F8ADF7FDD2CEFEA96C
:10322000FF2309F0CECE41CF66968CAD9DADAEADFD
:10323000BFAD6697A5FF4DC26B827C828D829E8258
:103240000C94391063965FAD639754FF02C060E839
:10325000F62A63968FAD63978F70E82FF0E0EE0F3C
:10326000FF1FEE0FFF1F6296AEADBFAD6297EA0F74
:10327000FB1F60807180828093808F3009F4ECC5E1
:103280006B96EFAD6B97EE2389F06D96FFAD6D9762
:10329000FF2361F0ECEF2E2EEFEF3E2EEFEF4E2EE0
:1032A000EFEF5E2E622073208420952066968CAD11
:1032B0009DADAEADBFAD669777E0B695A7959795F6
:1032C00087957A95D1F78F7166962CAD3DAD4EAD51
:1032D0005FAD669765E056954795379527956A9552
:1032E000D1F72370307040705070213031054105A6
:1032F000510511F40C947522213031054105510519
:1033000008F057C504C0660C771C881C991C8A9568
:10331000D2F70C94031066968CAD9DADAEADBFADEB
:10332000669705E0B695A795979587950A95D1F785
:10333000382F337063968FAD63978F70E82FF0E06E
:10334000EE0FFF1FEE0FFF1F62966EAD7FAD62970F
:10335000E60FF71F60807180828093808F3009F4C0
:1033600023C66B968FAD6B97882389F06D969FADC2
:103370006D97992361F0FCEF2F2EFFEF3F2EFFEFAB
:103380004F2EFFEF5F2E62207320842095206396DE
:103390003FAC639734FE9CC466964CAD5DAD6EAD9C
:1033A0007FAD6697BB27A72F962F852F8F70E82FAD
:1033B000F0E0EE0FFF1FEE0FFF1F62966EAD7FADC8
:1033C0006297E60FF71F40815181628173818F30D0
:1033D00011F40C943E236B969FAD6B97992329F0C3
:1033E0006D96AFAD6D97A1114C7F242F442309F446
:1033F00062C0313011F40C940730313010F00C946D
:10340000AF2A403208F47DC4403211F40C940C38D9
:1034100024961FAE249766247724430104CABBA8D0
:10342000B6FE15C00E8D0F3011F40C945D2362961C
:103430002EAD3FAD6297AA964EAD5FADAA97240F11
:10344000351FD9016D927D928D929C921397BDA9E3
:10345000BB2309F0BDC52FA838AC37FC02C00C94C3
:10346000770FF7FE02C00C94770F6296AEADBFAD3A
:103470006297DC962D913D914D915C91DF97C9014A
:1034800081709070892B11F40C94672A2E7FFD01B6
:1034900024AF35AF46AF57AFE096EEADFFADE09746
:1034A00080819181A281B381806280839183A28394
:1034B000B3830C94770F24961FAF2497B4C984E08C
:1034C000D82E0C944B10822F90E0FC01EE0FFF1FC2
:1034D000EE0FFF1FEE0FFF1F880F991FE80FF91F58
:1034E00062962EAC3FAC6297E20DF31DE455FF4FA0
:1034F000A081B181109711F40C94B00E822F90E04E
:10350000FC01EE0FFF1FEE0FFF1FEE0FFF1F880FD6
:10351000991FE80FF91FE20DF31DEE54FF4F608174
:10352000718166960CAD1DAD2EAD3FAD669794E1F1
:1035300036952795179507959A95D1F70F7066964A
:103540004CAC5DAC6EAC7FAC66978CE076946794C7
:10355000579447948A95D1F71FE0312E4320669601
:103560006CAC7DAC8EAC9FAC66976401EE24FF24FE
:10357000C32063965FAD63975F7054014301E5E03C
:10358000B694A79497948794EA95D1F737E0732E71
:10359000872062968EAD9FAD6297202F042DEC2C74
:1035A000C52EA82CFD010995882311F40C94B00EAA
:1035B0000C94770F82E090E0A0E0B0E00C946C11E6
:1035C00066964CAC5DAC6EAC7FAC669767FE3AC459
:1035D000892D582F50640C94751292E0692E712C2D
:1035E000812C912C0C9400122B3031054105510592
:1035F00011F40C9477282C3031054105510508F061
:1036000041C7293031054105510511F40C94432877
:103610002A3031054105510510F40C9415282296E5
:103620000FAD2297002311F40C94B00EE62FF0E0BA
:10363000EE0FFF1FEE0FFF1F62962EAD3FAD62979C
:10364000E20FF31FE080F180028113816F3011F4EB
:103650000C9447346B964FAD6B97442369F06D968D
:103660005FAD6D97552341F06CEF7FEF8FEF9FEFCC
:10367000E622F72208231923170128012618370804
:1036800048085908D201C1018E259F25A027B127DE
:10369000A8019701262537254825592582239323FC
:1036A000A423B5238827B7FD83959927AA27BB278D
:1036B00023968FAF239724961FAE2497E614F70422
:1036C0000805190520F071E024967FAF249780E06B
:1036D00048C96B827C828D829E8266247724430156
:1036E0000C943910C201B101660D771D881D991D1A
:1036F0006DA77EA78FA798AB70E8F72A0C94871068
:103700006B96EFAD6B97EE2309F05DC484E090E01B
:10371000A0E0B0E0280E391E4A1E5B1E0C94661015
:10372000D201C101820F931FA41FB51F8F8F98A3D1
:10373000A9A3BAA36296AEADBFAD6297A25BBE4F1E
:10374000ED91FC911197AE54B1406296BFAFAEAF10
:103750006297CD01BE016D5F7F4F2F8D38A149A1CA
:103760005AA10D2DEE246C96CFAC6C975E01089497
:10377000A11CB11C0995882309F490C7B1E0DB16A0
:1037800011F40C943C27CB80DC80ED80FE806696A3
:103790000CAD1DAD2EAD3FAD6697BCE036952795BF
:1037A00017950795BA95D1F766960CAF1DAF2EAF5A
:1037B0003FAF669763960FAD63970F700F3011F4AC
:1037C0000C941427E02FF0E0EE0FFF1FEE0FFF1F09
:1037D00062962EAD3FAD6297E20FF31FC082D18299
:1037E000E282F382611471048104910411F40C9457
:1037F000770FB201A101460D571D681D791D3BA130
:103800003F3011F40C94E82A62962EAD3FAD6297DA
:10381000AC968EAD9FADAC97280F391FD9014D9353
:103820005D936D937C9313970C94770F66968CAD94
:103830009DADAEADBFAD669780769070A070B07054
:103840000097A105B10509F0EFC366966CAC7DAC9D
:103850008EAC9FAC669790FC02C00C944A24D401B5
:10386000C30134E1B695A795979587953A95D1F719
:103870008F709070A070B0700097A105B10511F025
:103880000C943D2B66968CAC9DACAEACBFAC6697F1
:10389000C501AA27BB278F70E82FF0E0EE0FFF1FAE
:1038A000EE0FFF1F6296AEACBFAC6297EA0DFB1D38
:1038B00040805180628073808F3011F40C947A3490
:1038C0006B96CFAC6B97CC2089F06D96DFAC6D9783
:1038D000DD2061F08CEFE82E8FEFF82E8FEF082FB0
:1038E0008FEF182F4E205F206022712262960EAD5E
:1038F0001FAD6297025B1E4FE2961FAF0EAFE297BD
:10390000B3E08B2E912C8C0E9D1ED801ED91FC9175
:1039100062968EAD9FAD6297B401A301920104E05F
:10392000EE246C96CFAC6C971E010894211C311CC0
:1039300051010995882311F40C949235AB80BC8019
:10394000CD80DE80A8A6B9A6CAA6DBA663968FADF9
:1039500063978F70E82FF0E0EE0FFF1FEE0FFF1F51
:103960006296CEACDFAC6297EC0DFD1D20813181FB
:10397000428153818F3011F40C9482356B96EFACF9
:103980006B97EE2029F06D96FFAC6D97F1102C7FB0
:103990002B833C834D835E83E296AEADBFADE29751
:1039A000ED91FC9162968EAD9FAD6297B401A3013B
:1039B000920104E0EE24E3946C96CFAC6C97510135
:1039C0000995882311F40C944C3766962CAC3DACC9
:1039D0004EAC5FAC66977CE056944794379427943E
:1039E0007A95D1F766962CAE3DAE4EAE5FAE669739
:1039F00063960FAD63970F700F3011F40C9421375D
:103A0000E02FF0E0EE0FFF1FEE0FFF1F62962EADCE
:103A10003FAD6297E20FF31F48A559A56AA57BA5A4
:103A200040835183628373830C94770F66962CAC2A
:103A30003DAC4EAC5FAC669745FE92C4D201C1016D
:103A400080709070AF74B0700097A105B10511F44B
:103A50000C94B00E82017101FFEF4F2E512C612C9E
:103A6000712CE420F5200621172166966CAC7DAC04
:103A70008EAC9FAC6697BB27A92D982D872D8F7094
:103A80009070A070B070880F991FAA1FBB1F882369
:103A9000D1F090E0B801A701082E04C07695679593
:103AA000579547950A94D2F720E230E0281B390B4E
:103AB00004C0EE0CFF1C001F111F2A95D2F7E42A48
:103AC000F52A062B172B66962CAD3DAD4EAD5FAD9E
:103AD000669746FF02C00C94A12A66962CAC3DACBA
:103AE0004EAC5FAC6697C201AA27BB27282F2F7068
:103AF0006C963FAC6C97332011F40C94062F222E59
:103B000020FF18C06E2D6F7162968EAD9FAD6297CB
:103B10000E94C90BD601C50180705FEFA52EB12CA4
:103B2000C12CD12CAE20BF20C022D122A82AB92A74
:103B3000CA2ADB2A21FE14C04FEF442E512C4FEF2E
:103B4000642E4FEF742EA420B520C620D720D801B4
:103B5000C7018070A070B070A82AB92ACA2ADB2ACF
:103B600022FE14C03FEF632E3FEF732E812C3FEFF8
:103B7000932EA620B720C820D920D801C701807075
:103B80009070B070A82AB92ACA2ADB2A23FE14C072
:103B90002FEF3FEF4FEF50E0A222B322C422D522F5
:103BA00040E050E060E07FEFE422F5220623172397
:103BB000AE28BF28C02AD12AE096AEADBFADE097AF
:103BC000AD92BD92CD92DC9213970C94770FDE01EB
:103BD00012960C942613F42D6E965FAE6E97562DAA
:103BE000E72D0C942013862F90E0FC01EE0FFF1FB1
:103BF000EE0FFF1FEE0FFF1F880F991FE80FF91F31
:103C000062962EAC3FAC6297E20DF31DE055FF4F7C
:103C1000A081B181109711F40C94B00E862F90E022
:103C2000FC01EE0FFF1FEE0FFF1FEE0FFF1F880FAF
:103C3000991FE80FF91FE20DF31DEE54FF4F60814D
:103C4000718166962CAD3DAD4EAD5FAD669784E15A
:103C500056954795379527958A95D1F721706696A1
:103C6000ACACBDACCEACDFAC669704E0D694C794E8
:103C7000B794A7940A95D1F71FE0312EA32066963A
:103C8000ECACFDAC0EAD1FAD6697FCE0169507954C
:103C9000F794E794FA95D1F7E3206396EFAD639735
:103CA000EF7062968EAD9FAD6297422F2A2D0E2D3A
:103CB000E92CCE2EFD010995882311F40C94B00E49
:103CC0000C94770FAEA8AA2011F00C94B00EF5C892
:103CD00066968CAD9DADAEADBFAD669747E0B6952F
:103CE000A795979587954A95D1F7282F2F71313051
:103CF00011F40C94FE29313008F098C4222309F401
:103D0000DACB30E080E290E0821B930B13012401B8
:103D100004C056944794379427948A95D2F7022D7D
:103D2000017024960FAF249704C0660C771C881C82
:103D3000991C2A95D2F70C94131462968EAD9FAD00
:103D40006297B401A30124E0012FEE24C9800E94F0
:103D50005E0CEBA9FCA9EF70F070FCABEBAB0BA811
:103D600004C056944794379427940A94D2F7C1011B
:103D700081709070892B11F40C94770FFE8DFF30B9
:103D800011F40C94762A62962EAD3FAD6297AA96F6
:103D90004EAD5FADAA97240F351FD90169897A8985
:103DA0008B899C896D937D938D939C9313970C9431
:103DB000770F223031054105510509F457C32330EF
:103DC00031054105510511F00C940310882311F4BD
:103DD0000C94022890E0B401A301082E04C076954B
:103DE0006795579547950A94D2F720E230E0281B53
:103DF000390B04C0660C771C881C991C2A95D2F7D5
:103E0000642A752A862A972A0C9403106B965FAD54
:103E10006B97552309F0ECC384E090E0A0E0B0E09C
:103E200029883A884B885C88280E391E4A1E5B1EFA
:103E3000298A3A8A4B8A5C8A6EC882E090E0A0E0C8
:103E4000B0E0ABC9892D8068C4CB97FC02C00C944C
:103E5000DC1450680C94DC146B96BFAD6B97BB23DD
:103E600009F0DAC384E090E0A0E0B0E0680E791ECB
:103E70008A1E9B1E05CA1B821C821D821E8266969C
:103E80008CAC9DACAEACBFAC66977CE0B694A7940E
:103E9000979487947A95D1F766968CAE9DAEAEAE28
:103EA000BFAE669763968FAD63978F70E82FF0E093
:103EB000EE0FFF1FEE0FFF1F6296AEACBFAC629716
:103EC000EA0DFB1D20813181428153818F3011F435
:103ED0000C949C296B96CFAC6B97CC2029F06D96F7
:103EE000EFAC6D97E1102C7F53E0852E912C8C0E5A
:103EF0009D1E2B830C94D0106B966FAC6B97662035
:103F000009F08FC384E090E0A0E0B0E0C80ED91EB5
:103F1000EA1EFB1E0C94CD1262968EAD9FAD629789
:103F2000B301A2012D2D01E0EE24C9800E945E0C98
:103F30000C94770F6C8D7D8D44C8D401C3018E7FA6
:103F40006296EEADFFAD629784AF95AFA6AFB7AF07
:103F5000E096EEADFFADE09780819181A281B381C3
:103F60008F7D80839183A283B38361FE02C00C9412
:103F7000A934E096EEADFFADE0972081318142811A
:103F800053812F7D2083318342835383C30181700A
:103F90009070892B11F40C94770F20622083318369
:103FA000428353830C94770F6B967FAD6B97772387
:103FB00009F05FC384E090E0A0E0B0E0680E791EF5
:103FC0008A1E9B1ECEC982E090E0A0E0B0E0A2CBAA
:103FD0006296EEADFFAD6297EC5BFF4F1081018101
:103FE000F280E380612F6F7162968EAD9FAD629714
:103FF0000E94C90BE096EEADFFADE0971083018300
:10400000F282E3820C94770F6B966FAD6B97662309
:1040100009F0EAC584E090E0A0E0B0E0280F391F85
:104020004A1F5B1F0C94BD10DE011796EAE6F2E012
:1040300088E001900D928150E1F766962CAC3DAC82
:104040004EAC5FAC6697C201AA27BB27182F1F7022
:1040500046FED8C34201310174E096948794779468
:1040600067947A95D1F760EFA62EB12CC12CD12C94
:104070006A207B208C209D20D201C1018F7090701E
:10408000A070B070682A792A8A2A9B2A66968CAD1D
:104090009DADAEADBFAD669744E1B695A79597953A
:1040A00087954A95D1F7282F217066968CAD9DADE6
:1040B000AEADBFAD669735E0B695A7959795879558
:1040C0003A95D1F7817063963FAD639736FDD6C3BD
:1040D000882309F41068222309F0DAC366964CADF0
:1040E0005DAD6EAD7FAD669767FD08C0909480941E
:1040F00070946094611C711C811C911C66966CAD5F
:104100007DAD8EAD9FAD669790FDFFC21B821C8278
:104110001D821E8285FD10682B803C804D805E8054
:104120002CA23DA24EA25FA217FF02C00C94B00EBB
:104130000FE0202E2122422C5524440C551C440C07
:10414000551CAE965FAE4EAEAE976296EEADFFAD2D
:104150006297E40DF51DA080B180C280D380AD8A46
:10416000BE8ACF8AD88EAFE0BA2E2B1411F40C94ED
:10417000442F6B963FAD6B97332371F06D964FAD27
:104180006D97442349F06D897E898F89988D6C7F66
:104190006D8B7E8B8F8B988F812F90E0F0E34F2E6D
:1041A000512C4822592270E14716510459F0A1E1DF
:1041B0004A16510414F00C94222C4114510411F0AD
:1041C0000C942B2CE2E03E2E86FF02C00C945C2F58
:1041D000611471048104910411F00C94C42C28968C
:1041E0001CAE1DAE1EAE1FAE2897BB24B3943B146D
:1041F00011F40C94F93172E0371611F40C94D932A1
:1042000066964CAC5DAC6EAC7FAC66975CE0769429
:104210006794579447945A95D1F766964CAE5DAE25
:104220006EAE7FAE669763960FAD63970F70E02F0B
:10423000F0E0EE0FFF1FEE0FFF1F62966EAC7FAC3B
:104240006297E60DF71D80819181A281B3810F30C5
:1042500011F40C9427336B968FAC6B97882029F060
:104260006D969FAC6D9791108C7F8F839887A987EF
:10427000BA87802F8F5FE82FF0E0EE0FFF1FEE0F61
:10428000FF1F6296AEACBFAC6297EA0DFB1D2081AA
:104290003181428153818F3011F40C9417336B9626
:1042A000CFAC6B97CC2029F06D96DFAC6D97D11019
:1042B0002C7F2B873C874D875E876D887E888F8813
:1042C000988C2CA13DA14EA15FA1620E731E841E8D
:1042D000951E62964EAD5FAD6297425B5E4FDA010E
:1042E000ED91FC911197AE54B1406296BFAFAEAF65
:1042F0006297CD01BE01695F7F4FA4019301032D39
:10430000EE24E3946C96CFAC6C975E010894A11CEC
:10431000B11C0995882311F40C94743117FD02C067
:104320000C94770F812F8F708F3011F40C949F3580
:10433000E82FF0E0EE0FFF1FEE0FFF1F62962EAD8D
:104340003FAD6297E20FF31F28964CAD5DAD6EADA9
:104350007FAD289740835183628373830C94770FDA
:1043600066962CAC3DAC4EAC5FAC669746FEDCC1AD
:10437000D201C1012CE0B695A795979587952A950E
:10438000D1F70FE0D02ED8226D2D70E0660F771F89
:10439000660F771F6296EEADFFAD6297E60FF71FCF
:1043A000E080F18002811381BFE03B2ED31411F431
:1043B0000C94D9316B965FAC6B97552089F06D9654
:1043C0006FAC6D97662061F0ACEF8A2EAFEF9A2E3E
:1043D000AFEFAA2EAFEFBA2EE820F9200A211B2159
:1043E0002FEF3FEF40E050E0E222F32204231523B9
:1043F00066962CAD3DAD4EAD5FAD669720703070CA
:104400004F705070FCE0220F331F441F551FFA9568
:10441000D1F766968CAD9DADAEADBFAD66979F7082
:10442000A070B07066968CAF9DAFAEAFBFAF669711
:10443000DC0199278827282B392B4A2B5B2B2E2927
:104440003F29402B512B9FE0D91611F40C94362AAA
:1044500062968EAD9FAD6297680F791FDB012D9339
:104460003D934D935C9313970C94770F882309F435
:1044700038C604C095948794779467948A95D2F748
:104480000C9403102E3031054105510509F4A5C4E3
:104490002F3031054105510509F49AC42C303105FE
:1044A0004105510509F471C466962CAC3DAC4EAC87
:1044B0005FAC66978CE056944794379427948A951E
:1044C000D1F766962CAE3DAE4EAE5FAE6697639664
:1044D0000FAD63970F7022963FAC2297332011F4F3
:1044E0000C94F21481E00C94CA14882309F01BC7C1
:1044F0006624772443010C940310253031054105CF
:10450000510509F4ACC6263031054105510508F4C2
:10451000DFC4E62FF0E0EE0FFF1FEE0FFF1F6296E5
:104520004EAC5FAC6297E40DF51D20813181428174
:1045300053816F3011F40C9440326B96EFAC6B9753
:10454000EE2029F06D96FFAC6D97F1102C7F1123B2
:1045500011F40C94922E79018A01E618F7080809E3
:10456000190922966FAD2297662339F124961FAE62
:104570002497261537054805590520F071E0249643
:104580007FAF2497D801C70182279327A427B52797
:10459000262537254825592582239323A423B5238F
:1045A0008827B7FD83959927AA27BB2723968FAF26
:1045B0002397170128010C94B0143701480166961F
:1045C000ACACBDACCEACDFAC66975CE0D694C79427
:1045D000B794A7945A95D1F76696ACAEBDAECEAE61
:1045E000DFAE669763960FAD63970F700C94F2146D
:1045F00082E090E0A0E0B0E013CCBA01645E7F4FAF
:10460000660F771F660F771F6296AEACBFAC6297DE
:104610006A0D7B1D0C94E11782E090E0A0E0B0E011
:1046200025CC82E090E0A0E0B0E070CC323009F41C
:10463000BEC6333011F00C945B1A222311F00C9497
:104640002E30862D817024968FAF24979694879470
:1046500077946794112311F40C941314212C312CAA
:10466000412C90E8592E62287328842895280C94B0
:10467000131482E090E0A0E0B0E0A0CC6B968FAD88
:104680006B97882309F083C784E090E0A0E0B0E056
:10469000480F591F6A1F7B1F0C94EB1962968EAD51
:1046A0009FAD62974F8D58A169A17AA12D2D00E091
:1046B000C9800E945E0C0C94770FD401C3018E7FD9
:1046C0006296EEADFFAD629784AF95AFA6AFB7AF80
:1046D000E096AEADBFADE0972D913D914D915C91CF
:1046E00013972F7DFD012083318342835383C301C0
:1046F00081709070892B09F49FC720622D933D93A0
:104700004D935C9313970C94271A66968CAD9DADD0
:10471000AEADBFAD6697A5FD02C00C94DC2E6B82DA
:104720007C828D829E82F8CC66968CAD9DADAEADBE
:10473000BFAD66971CE0B695A795979587951A9596
:10474000D1F7E82FEF7066962CAD3DAD4EAD5FAD65
:104750006697A4E05695479537952795AA95D1F782
:104760002070307F4070507066966CAD7DAD8EAD20
:104770009FAD66977F7080709070262B372B482BEB
:10478000592BEF3009F472C6F0E0EE0FFF1FEE0F69
:10479000FF1F62966EAD7FAD6297E60FF71F208315
:1047A0003183428353830C94770F882311F40C9444
:1047B000D1146296EEADFFAD6297EC5BFF4F1081B6
:1047C0000181F280E380612F6F7162968EAD9FADA3
:1047D00062970E94C90BE096AEADBFADE0971C9307
:1047E00011960C9311971296FC9212971396EC92D5
:1047F0006296EEADFFAD629764AE75AE86AE97AED3
:104800000C94770F66968CAD9DADAEADBFAD66973F
:1048100080709F70A070B0700097A105B10509F07D
:10482000106863968FAD63978F70E82FF0E0EE0FFE
:10483000FF1FEE0FFF1F6296CEACDFAC6297EC0D50
:10484000FD1D60807180828093808F3011F40C9404
:10485000E9316B96EFAC6B97EE2009F417CC6D96AF
:10486000FFAC6D97FF2009F411CC2CEF3FEF4FEF19
:104870005FEF622273228422952208CC882309F4F8
:10488000BBC51061222321F41063882309F026CCD4
:10489000106424CC66968CAD9DADAEADBFAD669771
:1048A00014E1B695A795979587951A95D1F78F70CE
:1048B0009070A070B0708A309105A105B10508F024
:1048C000D1C788309105A105B10510F40C94613071
:1048D00066964CAD5DAD6EAD7FAD6697CB01AA27F8
:1048E000BB27582F5F705AAB66968CAD9DADAEADB1
:1048F000BFAD6697ECE0B695A79597958795EA9535
:10490000D1F7682F6F7069AB6F961FAE6F97A09647
:104910001FAEA097A1961FAEA197A2961FAEA29719
:10492000A3961FAEA397A4961FAEA497A5961FAEFD
:10493000A597A6961FAEA69766962CAC3DAC4EAC3E
:104940005FAC6697BB27A52D942D832D8F70E82F24
:10495000F0E0EE0FFF1FEE0FFF1F62964EAC5FAC54
:104960006297E40DF51D20803180428053808F30A6
:1049700011F40C9428346B967FAC6B97772089F0F8
:104980006D968FAC6D97882061F02CEFA22E2FEFE3
:10499000B22E2FEFC22E2FEFD22E2A203B204C20FA
:1049A0005D2063968FAD63978F70E82FF0E0EE0F78
:1049B000FF1FEE0FFF1F6296CEACDFAC6297EC0DCF
:1049C000FD1DA080B180C280D3808F3011F40C9483
:1049D000FD336B96FFAC6B97FF2069F06D960FADC2
:1049E0006D97002341F02CEF3FEF4FEF5FEFA222D6
:1049F000B322C422D52266964CAD5DAD6EAD7FADBF
:104A0000669766FD02C00C94CB3286017501110FCA
:104A1000EE08FE2C870142013101990C6608762CC4
:104A200043019501A6016E2D7E2D8E2D9E2D5101E7
:104A30006201E62CF62C062D162D0E945001A32FA4
:104A4000B42F152F062FF72EE82ED92E6F962FACE8
:104A50006F97220EF1E0221608F0F0E0A0963FAD2D
:104A6000A0973A0FE1E03A1708F0E0E08F2E830EAE
:104A700021E0831608F020E0E22BA1964FADA1972C
:104A80004B0F31E04B1708F030E07E2E740E21E022
:104A9000741608F020E0322BA2965FADA297510F5A
:104AA00041E0511708F040E0632E650E21E06516E5
:104AB00008F020E0422BA3966FADA397600F31E082
:104AC000601708F030E0542E560E21E0561608F01C
:104AD00020E0322BA4967FADA4977F0D41E07F1597
:104AE00008F040E0432E470E21E0471608F020E092
:104AF000422BA5968FADA5978E0D21E08E1508F05F
:104B000020E0342E380E91E0381608F090E0922E16
:104B1000992AA6965FADA697D50E9D0C222D382D0D
:104B2000472D562D652D742D832D992D00E20E9461
:104B30004B0259016A01222D382D472D562D69A9A6
:104B40006F3011F40C947A3319A9E12FF0E0EE0FD5
:104B5000FF1FEE0FFF1F62966EAD7FAD6297E60FEF
:104B6000F71F20833183428353837AA97F3011F466
:104B70000C94B0331AA9E12FF0E0EE0FFF1FEE0FF7
:104B8000FF1F62962EAD3FAD6297E20FF31FA0822A
:104B9000B182C282D38266964CAD5DAD6EAD7FAD03
:104BA000669764FD02C00C94770FE096AEADBFAD82
:104BB000E0974D915D916D917C917F73822D882955
:104BC00087298629852984298329892909F47064FC
:104BD000D7FC7068E096EEADFFADE097408351835F
:104BE000628373830C94770F82E090E0A0E0B0E0E2
:104BF00015CA87309105A105B10509F4D6C60797F6
:104C0000A105B10510F40C94B00E20383105410512
:104C1000510511F00C94B00E63968FAD63978F70B1
:104C2000E82FF0E0EE0FFF1FEE0FFF1F62962EAC95
:104C30003FAC6297E20DF31D2080318042805380AB
:104C40008F3011F40C9469376B967FAC6B9777209B
:104C500089F06D968FAC6D97882061F09CEFA92E3E
:104C60009FEFB92E9FEFC92E9FEFD92E2A203B2010
:104C70004C205D206696CCACDDACEEACFFAC66970C
:104C8000BB27AF2D9E2D8D2D8F70E82FF0E0EE0FFE
:104C9000FF1FEE0FFF1F6296EEACFFAC6297EE0DAA
:104CA000FF1D20813181428153818F3011F40C949A
:104CB0005A376B960FAD6B97002329F06D961FAD99
:104CC0006D9711112C7F66968CAD9DADAEADBFADCD
:104CD000669715E1B695A795979587951A95D1F79B
:104CE00083709070A070B07081309105A105B105FE
:104CF00011F40C94F83981309105A105B10510F437
:104D00000C94693982309105A105B10511F40C9418
:104D100096380397A105B10511F40C9452386696A4
:104D20002CAD3DAD4EAD5FAD6697CA01AA27BB273E
:104D3000082F0F7088249924540110E00F3011F4CB
:104D40000C941836E02FF0E0EE0FFF1FEE0FFF1F60
:104D500062964EAD5FAD6297E40FF51F808291823F
:104D6000A282B382112311F40C94770FE096EEAD7A
:104D7000FFADE09780819181A281B381B86080838B
:104D80009183A283B3830C94770FE62FF0E0EE0FAC
:104D9000FF1FEE0FFF1F62964EAD5FAD6297E40FEF
:104DA000F51F20813181428153816F3011F40C94C1
:104DB00030326B967FAD6B97772329F06D968FAD70
:104DC0006D9781112C7F622A732A842A952A6CCBD5
:104DD000609470948094909467CBE62FF0E0EE0F8F
:104DE000FF1FEE0FFF1F6296AEADBFAD6297EA0FD9
:104DF000FB1F20813181428153816F3011F40C946B
:104E000054316B96EFAD6B97EE2329F06D96FFADA5
:104E10006D97F1112C7F609470948094909462222D
:104E200073228422952240CBD701C6018E7F6296E1
:104E3000EEADFFAD629784AF95AFA6AFB7AFE0968A
:104E4000AEADBFADE0972D913D914D915C91139723
:104E50002F7DFD012083318342835383C6018170FE
:104E60009070892B09F4B1C720622D933D934D9327
:104E70005C9313970C94F21B8B8190E0A0E0B0E060
:104E80008B839C83AD83BE830C94C31BE62FF0E021
:104E9000EE0FFF1FEE0FFF1F62968EAD9FAD629764
:104EA000E80FF91F20813181428153816F3011F465
:104EB0000C9450326B96AFAD6B97AA2309F4AFCF29
:104EC0006D96BFAD6D97BB2309F4A9CF2C7FA7CFFB
:104ED000E62FF0E0EE0FFF1FEE0FFF1F62964EADC4
:104EE0005FAD6297E40FF51F2081318142815381CC
:104EF0006F3011F40C9492316B967FAD6B977723E2
:104F000029F06D968FAD6D9781112C7F79018A0103
:104F1000E60CF71C081D191D22969FAD22979923B8
:104F200009F44BCBD801C70182279327A427B527C3
:104F3000212C312C412CF0E85F2E620C731C841C58
:104F4000951C622673268426952686219721A82102
:104F5000B9218827B7FD83959927AA27BB272396D0
:104F60008FAF239724961FAE2497E216F30604070B
:104F7000150720F421E024962FAF2497170128016C
:104F80000C94B014E62FF0E0EE0FFF1FEE0FFF1FA2
:104F90006296AEADBFAD6297EA0FFB1F20813181F3
:104FA000428153816F3011F40C9444316B96EFAD14
:104FB0006B97EE2329F06D96FFAD6D97F1112C7F65
:104FC000112309F48AC684017301E21AF30A040B5F
:104FD000150B22962FAC2297222009F4EECA2496B4
:104FE0001FAE2497621673068406950620F061E0D2
:104FF00024966FAF2497D801C70186259725A82549
:10500000B925C6CA9694879477946794D5FC02C054
:105010000C940310A12CB12CC12C90E8D92E6A2835
:105020007B288C289D280C94031022969FAD2297F4
:10503000992311F40C94B00EE62FF0E0EE0FFF1F51
:10504000EE0FFF1F6296AEADBFAD6297EA0FFB1F7A
:1050500080819181A281B3816F3011F40C946B3403
:105060006B96FFAD6B97FF2329F06D962FAC6D9774
:1050700021108C7F1C012D0126203720482059202B
:1050800080E00C94B11422963FAC2297332011F4A7
:105090000C94B00EE62FF0E0EE0FFF1FEE0FFF1F97
:1050A00062964EAC5FAC6297E40DF51D80819181F4
:1050B000A281B3816F3011F40C94ED336B96EFAC99
:1050C0006B97EE2029F06D96FFAC6D97F1108C7FF9
:1050D0001C012D01262437244824592480E00C94F7
:1050E000B114990C6608762C43010C940310229697
:1050F0008FAD2297882311F40C94B00EE62FF0E0C8
:10510000EE0FFF1FEE0FFF1F6296AEADBFAD6297B1
:10511000EA0FFB1F20813181428153816F3011F4EE
:105120000C94DD336B96EFAD6B97EE2329F06D9603
:10513000FFAD6D97F1112C7F79018A01E60CF71C08
:10514000081D191DD801C70182279327A427B52759
:10515000212C312C412C70E8572E620C731C841CBE
:10516000951C622673268426952686219721A821E0
:10517000B9218827B7FD83959927AA27BB272396AE
:105180008FAF239724961FAE2497E216F3060407E9
:10519000150720F421E024962FAF2497170128014A
:1051A00080E00C94B114E62FF0E0EE0FFF1FEE0F3D
:1051B000FF1F6296AEADBFAD6297EA0FFB1FE080A6
:1051C000F180028113816F3011F40C9482316B965F
:1051D000EFAD6B97EE2389F06D96FFAD6D97FF23D2
:1051E00061F03CEF232E3FEF332E3FEF432E3FEF96
:1051F000532EE220F32004211521130124012E183F
:105200003F08400A510A22962FAD2297222309F027
:10521000AAC542013101D3C9E62FF0E0EE0FFF1F0E
:10522000EE0FFF1F62962EAC3FAC6297E20DF31DAE
:1052300020813181428153816F3011F40C94C93146
:105240006B964FAC6B97442029F06D965FAC6D97D1
:1052500051102C7F622673268426952625C9E62FB9
:10526000F0E0EE0FFF1FEE0FFF1F62964EAD5FAD39
:105270006297E40FF51F20813181428153816F30A5
:1052800011F40C94A9316B967FAD6B97772329F0BD
:105290006D968FAD6D9781112C7F112309F4D9C5BF
:1052A0000894611C711C811C911C84017301E20E25
:1052B000F31E041F151F08946108710881089108E6
:1052C00022969FAD2297992309F477C924961FAEA1
:1052D00024972E153F054007510720F0A1E02496A2
:1052E000AFAF2497D801C70182279327A427B527FA
:1052F000212C312C412C60E8562E620C731C841C2E
:10530000951C262537254825592582239323A42338
:10531000B5238827B7FD83959927AA27BB2723960E
:105320008FAF23972BCE04C096948794779467947D
:105330008A95D2F70C9403106B96BFAC6B97BB2089
:1053400009F067C584E090E0A0E0B0E0280F391FC5
:105350004A1F5B1F0C946A1F8DA59EA5AFA5B8A917
:105360008E7F6296EEADFFAD629784AF95AFA6AF2C
:10537000B7AFE096AEADBFADE0972D913D914D91A9
:105380005C9113972F7DFD012083318342835383EA
:105390008DA59EA581709070892B11F00C94B31887
:1053A000BDA5B1FD02C00C94770F0C94B01122235F
:1053B00009F434C1422F50E041505040D401C301A0
:1053C000042E04C0B695A795979587950A94D2F7B1
:1053D0004F5F5F4F782F717024967FAF249797FEB1
:1053E00002C00C94DA3404C096948794779467943E
:1053F0004A95D2F70C941314106244CA222309F080
:10540000CBC0662497FC639477248824992424963F
:105410006FAE24976624772443010C941314D301B0
:10542000C2018E7F6296EEADFFAD629784AF95AFFD
:10543000A6AFB7AFE096AEADBFADE0972D913D9171
:105440004D915C9113972F7DFD0120833183428321
:105450005383C20181709070892B11F00C94B318A2
:1054600041FC02C00C94770F0C94B011DA01C90111
:105470008E7F6296EEADFFAD629784AF95AFA6AF1B
:10548000B7AFE096AEADBFADE097ED90FD900D915A
:105490001C911397FFED2F2EFFEF3F2EFFEF4F2EA6
:1054A000FFEF5F2EE220F32004211521ED92FD9203
:1054B0000D931C931397C90181709070892B09F08B
:1054C00058C721FD02C00C94770F0C94B011E096E0
:1054D000EEADFFADE09780819181A281B3818F7D98
:1054E00080839183A283B3830C94770F89899A89EF
:1054F000AB89BC898E7F6296EEADFFAD629784AFBB
:1055000095AFA6AFB7AFE096AEADBFADE0972D912A
:105510003D914D915C9113972F7DFD012083318347
:105520004283538389899A8981709070892B11F005
:105530000C94B318B989B1FD02C00C94770F0C9488
:10554000B01162964EAD5FAD62974C5B5F4FDA0172
:10555000ED92FD920D931C9313970C94770F3230BC
:1055600009F45DC5333011F00C945B1A2F7111F002
:105570000C949434D401C3018827B7FD83959927EF
:10558000AA27BB2724968FAF24970C94131482E08C
:1055900090E0A0E0B0E07CC8822F90E00197A401E9
:1055A0009301082E04C056954795379527950A9480
:1055B000D2F70196622F617024966FAF249704C0D2
:1055C00096948794779467948A95D2F70C941314E1
:1055D000DB01CA018E7F6296EEADFFAD629784AFAC
:1055E00095AFA6AFB7AFE096AEADBFADE0970D916A
:1055F0001D912D913C9113970F7DFD010083118327
:1056000022833383CA0181709070892B09F0A8C767
:1056100041FD02C00C94770F0C94B01197FC02C0AE
:105620000C94081A21E024962FAF249766246A94DC
:10563000762C43010C94131461FC02C00C94271ABD
:105640006296EEADFFAD6297E05BFE4F6296FFAFF4
:10565000EEAF62970190F081E02D62960EAD1FAD26
:1056600062970055114062961FAF0EAF6297C80156
:1056700063E371E009950C94271A0497A105B1051D
:1056800011F00C94B00E66962CAC3DAC4EAC5FACF9
:105690006697C201AA27BB278F70E82FF0E0EE0FB4
:1056A000FF1FEE0FFF1F62964EAC5FAC6297E40DDA
:1056B000F51D60807180828093808F3011F40C948E
:1056C000C8346B96AFAC6B97AA2089F06D96BFACCF
:1056D0006D97BB2061F03CEFC32E3FEFD32E3FEF21
:1056E000E32E3FEFF32E6C207D208E209F206296CC
:1056F0000EAD1FAD6297025B1E4FE2961FAF0EAF5D
:10570000E29722E0422E512C4C0E5D1ED801ED9105
:10571000FC9162968EAD9FAD6297B201A401930198
:1057200001E0EE246C96CFAC6C971E010894211C0E
:10573000311C51010995882311F40C94BB341A8152
:1057400063968FAD63978F70E82FF0E0EE0FFF1F29
:10575000EE0FFF1F6296AEACBFAC6297EA0DFB1D69
:1057600020813181428153818F3011F40C94F734C0
:105770006B96CFAC6B97CC2029F06D96DFAC6D9714
:10578000D1102C7F2A83E296AEADBFADE297ED91AA
:10579000FC9162968EAD9FAD6297B201A401930118
:1057A00001E0EE24E3946C96CFAC6C97510109951F
:1057B000882311F40C94A73A66962CAC3DAC4EAC01
:1057C0005FAC66970CE056944794379427940A95FB
:1057D000D1F766962CAE3DAE4EAE5FAE6697639641
:1057E0000FAD63970F70C12EDD24EE24FF240F3020
:1057F00011F00C94CF15D701C6018E7F6296EEADE5
:10580000FFAD629784AF95AFA6AFB7AFE096AEADF0
:10581000BFADE0972D913D914D915C9113972F7DF8
:10582000FD012083318342835383C60181709070D0
:10583000892B11F00C94B318C1FC02C00C94770FA3
:105840000C94B011B0E24B16510409F436C4E0E3F5
:105850004E16510419F033240C94E42078E0372ECE
:105860000C94E4208E309105A105B10508F46AC5B9
:1058700066962CAC3DAC4EAC5FAC6697C201AA27D5
:10588000BB27082F0F700AABE02FF0E0EE0FFF1FD1
:10589000EE0FFF1F62962EAD3FAD6297E20FF31F32
:1058A000E080F180028113813AA93F3011F40C9419
:1058B00082376B965FAD6B97552369F06D966FAD30
:1058C0006D97662341F08CEF9FEFAFEFBFEFE822BB
:1058D000F9220A231B2366968CAD9DADAEADBFADFC
:1058E00066976CE0B695A795979587956A95D1F7D9
:1058F000E82FEF70E9ABF0E0EE0FFF1FEE0FFF1F98
:1059000062962EAC3FAC6297E20DF31D208131818F
:105910004281538169A96F3011F40C9416386B964B
:105920008FAD6B97882329F06D969FAD6D97911180
:105930002C7F19012A01570168019701A60160E037
:1059400070E080E090E000E20E94CA0222296F9697
:105950002FAF6F973329A0963FAFA0974429A19608
:105960004FAFA1975529A2965FAFA297A3966FAFAD
:10597000A397A4967FAFA497A5968FAFA597A69659
:105980009FAFA6970C949C24AD88BE88CF88D88CF6
:10599000A60CB71CC81CD91C2896ACAEBDAECEAEAA
:1059A000DFAE289710680C94F52062960EAD1FADFF
:1059B0006297065B1E4FD801ED90FD900D911C91F2
:1059C0001397AA54B1406296BFAFAEAF62973CE066
:1059D000232E312C412C512CE20CF31C041D151DDF
:1059E000CD0167E10E94C90B87E990E0A0E0B0E03B
:1059F000E096EEADFFADE09780839183A283B38301
:105A000062962EAD3FAD62972C5B3F4FD901AD92B0
:105A1000BD92CD92DC921397A454B0406A962CADFF
:105A20003DAD4EAD5FAD6A972C5F3F4F4F4F5F4F1F
:105A3000D8962D933D934D935C93DB97FD01E4AE97
:105A4000F5AE06AF17AF0C94770F66968CAD9DAD93
:105A5000AEADBFAD66979F70AF7BB0708050904089
:105A6000AF40B04009F404C666968CAD9DADAEADB6
:105A7000BFAD6697807FA07BB0708050904FA042F2
:105A8000B04011F00C94B00E63968FAD63978F7099
:105A9000E82FF0E0EE0FFF1FEE0FFF1F62964EADF6
:105AA0005FAD6297E40FF51FE080F1800281138102
:105AB0008F3011F40C944A3B6B966FAD6B97662355
:105AC00069F06D967FAD6D97772341F08CEF9FEF76
:105AD000AFEFBFEFE822F9220A231B2366962CAC16
:105AE0003DAC4EAC5FAC669746FC02C00C946D1D9D
:105AF00062962EAD3FAD62972C5B3F4FD901ED9280
:105B0000FD920D931C9313970C94770F66968CADB2
:105B10009DADAEADBFAD669780709F70A070B07048
:105B20000097A105B10511F00C94B00E63968FADEE
:105B300063978F70E82FF0E0EE0FFF1FEE0FFF1F4F
:105B400062962EAD3FAD6297E20FF31F60807180C9
:105B5000828093808F3011F40C9434386B964FAD63
:105B60006B97442369F06D965FAD6D97552341F0B7
:105B70006CEF7FEF8FEF9FEF6622772288229922CA
:105B800066962CAC3DAC4EAC5FAC6697C201AA27C2
:105B9000BB278F70E82FF0E0EE0FFF1FEE0FFF1F07
:105BA00062964EAC5FAC6297E40DF51DE080F1802B
:105BB000028113818F3011F40C9425386B96AFACB1
:105BC0006B97AA2069F06D96BFAC6D97BB2041F032
:105BD0002CEF3FEF4FEF5FEFE222F3220423152378
:105BE00066968CAD9DADAEADBFAD6697E5E1B69561
:105BF000A79597958795EA95D1F783709070A070D7
:105C0000B07081309105A105B10511F40C94DF3716
:105C100081309105A105B10508F0C2C7570168019F
:105C2000A60CB71CC81CD91CD601C5018E259F2502
:105C3000A027B12740E050E060E070E8640E751ED8
:105C4000861E971E6E247F2480269126862197210A
:105C5000A821B9218827B7FD83959927AA27BB27B3
:105C60008CA7882349F017FF02C00C94C536AA24DC
:105C7000BB24650151E05CA766968CAD9DADAEADD1
:105C8000BFAD66975CE0B695A795979587955A95B1
:105C9000D1F766968CAF9DAFAEAFBFAF66976396F8
:105CA0000FAD63970F700F3011F40C94C33AE02FCF
:105CB000F0E0EE0FFF1FEE0FFF1F62962EAD3FAD1F
:105CC0006297E20FF31FA082B182C282D3823CA509
:105CD000332311F40C94770F49C8089461087108B4
:105CE0008108910884017301E21AF30A040B150B71
:105CF0000894611C711C811C911C22967FAD229717
:105D0000772311F40C94DD2224961FAE24972615D8
:105D100037054805590508F06EC981E024968FAF14
:105D2000249769C984017301E094F094009510955B
:105D3000E20EF31E041F151F22968FAD22978823B3
:105D400011F40C94DD2224961FAE2497621673067C
:105D50008406950610F00C94C22291E024969FAF21
:105D600024970C94C222D201C10186259725A8252B
:105D7000B925A801970126253725482559258223CD
:105D80009323A423B5238827B7FD83959927AA27B2
:105D9000BB2723968FAF239724961FAE24976E14AC
:105DA0007F048006910610F40C94B01431E0249620
:105DB0003FAF24970C94B0146B827C828D829E82BC
:105DC0006624772443010C948C20C1FC02C00C94FF
:105DD000F21B6296EEADFFAD6297E05BFE4F6296FE
:105DE000FFAFEEAF62970190F081E02D62960EADAD
:105DF0001FAD62970055114062961FAF0EAF6297BC
:105E0000C80163E371E009950C94F21B222E0C94F7
:105E1000C61D82E090E0A0E0B0E098CA66966CAC47
:105E20007DAC8EAC9FAC66977CE09694879477941B
:105E300067947A95D1F766966CAE7DAE8EAE9FAEC6
:105E4000669763960FAD63970F70420131010C9412
:105E5000F21479018A01E60CF71C081D191D22961F
:105E6000BFAD2297BB2311F40C94DD2224961FAE04
:105E70002497E216F3060407150708F033CAE1E099
:105E80002496EFAF24972ECA6B96CFAC6B97CC209D
:105E900009F06EC384E090E0A0E0B0E02D893E8977
:105EA0004F89588D280F391F4A1F5B1F2D8B3E8B42
:105EB0004F8B588F0C94B920AD88BE88CF88D88C72
:105EC000ECA0FDA00EA11FA1AE0CBF1CC01ED11ED8
:105ED0006096ACAEBDAECEAEDFAE609762960EAD54
:105EE0001FAD6297025B1E4FD801ED91FC91119797
:105EF000AE54B1406296BFAFAEAF6297CD01BE0166
:105F0000695F7F4FA6019501032DEE246C96CFACFF
:105F10006C975E010894A11CB11C0995882309F4B3
:105F20007CC4B1E03B1609F4AEC532E0331611F47F
:105F30000C947B3A66964CAD5DAD6EAD7FAD6697C9
:105F40009CE076956795579547959A95D1F7669613
:105F50004CAF5DAF6EAF7FAF669763960FAD639743
:105F60000F70CF80D884E984FA840F3011F40C9438
:105F70004D3AE02FF0E0EE0FFF1FEE0FFF1F62968D
:105F80002EAD3FAD6297E20FF31FC082D182E28255
:105F9000F3820F5FCB84DC84ED84FE840F3009F440
:105FA00079C6E02FF0E0EE0FFF1FEE0FFF1F6296A5
:105FB0002EAD3FAD6297E20FF31FC082D182E28225
:105FC000F382611471048104910411F40C94770F2D
:105FD000ED88FE880F89188DE60CF71C081D191D29
:105FE0003FE0231611F40C948E1162962EAD3FAD56
:105FF0006297AE964EAD5FADAE97240F351FD901B7
:10600000ED92FD920D931C9313970C94770F4032F1
:1060100008F4C2CA403211F00C94081AF2C9403296
:1060200008F0FCCA842F90E00197A4019301082E88
:1060300004C056954795379527950A94D2F701964F
:10604000722F717024967FAF249704C09594879423
:10605000779467948A95D2F70C94131430E021500A
:106060003040D401C301022E04C0B695A795979580
:1060700087950A94D2F72F5F3F4F082F017024961F
:106080000FAF2497B401A301022E04C07695679543
:10609000579547950A94D2F780E290E0821B930BC4
:1060A00004C0660C771C881C991C8A95D2F7642A58
:1060B000752A862A972A0C941314332433940C944B
:1060C000E42082309105A105B10508F456C2049779
:1060D000A105B10510F00C94B00E66968CAD9DAD87
:1060E000AEADBFAD66977CE0B695A79597958795C1
:1060F0007A95D1F78F70E82FF0E0EE0FFF1FEE0FCB
:10610000FF1F6296AEADBFAD6297EA0FFB1F6080C6
:106110007180828093808F3011F40C94B43A6B9626
:10612000EFAD6B97EE2389F06D96FFAD6D97FF2372
:1061300061F05CEF252E5FEF352E5FEF452E5FEFB0
:10614000552E62207320842095206696ACACBDACA1
:10615000CEACDFAC6697BB27AD2D9C2D8B2D8F7001
:10616000E82FF0E0EE0FFF1FEE0FFF1F6296CEACA0
:10617000DFAC6297EC0DFD1DA080B180C280D380A2
:106180008F3009F43BC56B96FFAC6B97FF2069F02D
:106190006D960FAD6D97002341F02CEF3FEF4FEF61
:1061A0005FEFA222B322C422D52263968FAD6397FC
:1061B0008F70E82FF0E0EE0FFF1FEE0FFF1F6296CB
:1061C0004EAD5FAD6297E40FF51F208131814281B2
:1061D00053818F3009F403C56B967FAD6B9777239E
:1061E00029F06D968FAD6D9781112C7FCA01B90191
:1061F000A60195010E94156B7B018C01E60CF71C32
:10620000081D191D66962CAC3DAC4EAC5FAC669774
:10621000C201AA27BB278F708F3009F407C4E82F6B
:10622000F0E0EE0FFF1FEE0FFF1F62964EAD5FAD69
:106230006297E40FF51FE082F18202831383669672
:106240006CAD7DAD8EAD9FAD669784FD02C00C94A4
:10625000770FE096EEADFFADE09780819181A2814E
:10626000B381BF73E114F1040105110509F4A0C362
:1062700017FDB068E096EEADFFADE09780839183A7
:10628000A283B3830C94770F6B96BFAD6B97BB2340
:1062900009F0D9C284E090E0A0E0B0E0280F391FF7
:1062A0004A1F5B1F0C94D6276B96BFAD6B97BB2321
:1062B00009F0E8C284E090E0A0E0B0E0280F391FC8
:1062C0004A1F5B1F0C9401276B962FAD6B972223FF
:1062D00009F06EC284E090E0A0E0B0E0E80EF91EA4
:1062E0000A1F1B1F0C946C1462968EAD9FAD6297B3
:1062F000B401A301232D01E0EE24C9800E945E0CAD
:106300000C94770F6B96BFAD6B97BB2309F0CFC290
:1063100084E090E0A0E0B0E0E80EF91E0A1F1B1F29
:106320000C94E7286B966FAD6B97662309F0DDC17F
:1063300084E090E0A0E0B0E0280F391F4A1F5B1F07
:106340000C947C270C97A105B10508F491CA0C9414
:1063500068246B966FAD6B97662309F08EC284E05C
:1063600090E0A0E0B0E0280F391F4A1F5B1F0C949B
:106370004329E0E22E2E312C412C512CE228F32827
:1063800004291529ED92FD920D931C9313970C94FB
:10639000770F6B963FAC6B97332009F069C284E0AE
:1063A00090E0A0E0B0E0280F391F4A1F5B1F0C945B
:1063B00020296B964FAC6B97442009F03FC284E0D4
:1063C00090E0A0E0B0E0E80EF91E0A1F1B1F0C943D
:1063D000DA216B96DFAC6B97DD2009F023C184E0F6
:1063E00090E0A0E0B0E0680E791E8A1E9B1E0C941F
:1063F00029246696CCACDDACEEACFFAC6697BCE075
:10640000F694E794D794C794BA95D1F76696CCAE34
:10641000DDAEEEAEFFAE669763968FAD63978F707D
:10642000E82FF0E0EE0FFF1FEE0FFF1F6296EEACBD
:10643000FFAC6297EE0DFF1D2081318142815381B7
:106440008F3009F4E4C26B960FAD6B97002329F0EF
:106450006D966FAD6D9761112C7F2F830C945D212C
:106460006B966FAD6B97662309F02BC284E090E0CA
:10647000A0E0B0E0280F391F4A1F5B1F0C94D926FB
:106480006B965FAC6B97552009F020C284E090E0DA
:10649000A0E0B0E0280F391F4A1F5B1F0C949D221B
:1064A0006B969FAD6B97992309F006C284E090E04C
:1064B000A0E0B0E0280F391F4A1F5B1F0C945A2739
:1064C00066968CAD9DADAEADBFAD66978070BF706A
:1064D00080509F4FAF42B14011F00C94B00E6696C1
:1064E0008CAD9DADAEADBFAD669780739070A07062
:1064F000B070C097A105B10511F40C94FC3C6396F3
:106500008FAD63978F70E82FF0E0EE0FFF1FEE0F57
:10651000FF1F62962EAC3FAC6297E20DF31DC08068
:10652000D180E280F3808F3011F40C94ED3C6B96B7
:106530004FAC6B97442009F45EC96D965FAC6D97C4
:10654000552009F458C90CEF602E0FEF702E0FEF95
:10655000802E0FEF902EC620D720E820F9204BC9BF
:1065600000620D931D932D933C9313970C94770F1A
:1065700082E090E0A0E0B0E091CC64968EAD9FAD5B
:1065800064978070907F892B11F00C94B00E662474
:1065900077244301DACD9501A60160E070E080E048
:1065A00090E051016201EE24FF2400E010E00C9421
:1065B0001D2566968CAD9DADAEADBFAD66977CE0FA
:1065C000B695A795979587957A95D1F766968CAFEE
:1065D0009DAFAEAFBFAF669763968FAD63978F7079
:1065E000E82FF0E0EE0FFF1FEE0FFF1F6296AEAD3B
:1065F000BFAD6297EA0FFB1F208131814281538139
:106600008F3011F40C94593B6B96EFAD6B97EE23E2
:1066100029F06D96FFAD6D97F1112C7F38872F8390
:106620000C945D2182E090E0A0E0B0E0DCCE6B96BF
:10663000BFAC6B97BB2009F0F0C284E090E0A0E013
:10664000B0E0280F391F4A1F5B1F0C944F216B9637
:106650007FAC6B97772009F010C234E0C32ED12CA9
:10666000E12CF12C8C0D9D1DAE1DBF1D0C942B211A
:1066700066968CAD9DADAEADBFAD66970CE0B695A0
:10668000A795979587950A95D1F78F7066962CAC4C
:106690003DAC4EAC5FAC669746FE12C062960EAD46
:1066A0001FAD62970C5B1F4FD801AD90BD90CD9090
:1066B000DC901397A454B0406296BFAFAEAF629720
:1066C0008F3009F42EC4E82FF0E0EE0FFF1FEE0F1D
:1066D000FF1F62962EAD3FAD6297E20FF31FA082BF
:1066E000B182C282D3820C94770F82E090E0A0E066
:1066F000B0E022CEDA01C9018E7F6296EEADFFAD29
:10670000629784AF95AFA6AFB7AFE096AEADBFAD21
:10671000E097ED90FD900D911C9113976FED7FEF39
:106720008FEF9FEFE622F72208231923ED92FD92C7
:106730000D931C931397C90181709070892B09F4F4
:1067400088C720E230E040E050E0E22AF32A042B40
:10675000152BED92FD920D931C9313970C94B52578
:10676000D601C5018E7F6296EEADFFAD629784AF14
:1067700095AFA6AFB7AFE096AEADBFADE0972D91A8
:106780003D914D915C9113972F7DFD0120833183C5
:1067900042835383C50181709070892B09F4F2C341
:1067A00020622D933D934D935C9313970C94CB25CE
:1067B00082E090E0A0E0B0E091CD6B96BFAD6B972A
:1067C000BB2309F002C284E090E0A0E0B0E0280F13
:1067D000391F4A1F5B1F0C9492286B965FAC6B9716
:1067E000552009F0F7C124E030E040E050E0820F8E
:1067F000931FA41FB51F0C945E286B96EFAC6B978C
:10680000EE2009F07AC184E090E0A0E0B0E0A80EAC
:10681000B91ECA1EDB1E0C94E92462968EAD9FAD94
:10682000629760964CAD5DAD6EAD7FAD6097232DE8
:1068300000E0C9800E945E0C0C94770F82E090E02B
:10684000A0E0B0E0C0CD82E090E0A0E0B0E026CDD6
:106850006B966FAC6B97662009F05CC084E090E0AB
:10686000A0E0B0E0280E391E4A1E5B1E0C94BB242B
:1068700082E090E0A0E0B0E096CD82E090E0A0E081
:10688000B0E071CD82E090E0A0E0B0E017CD6B9673
:106890003FAD6B97332309F093C184E090E0A0E013
:1068A000B0E0E80EF91E0A1F1B1F0C942A1B82E0A1
:1068B00090E0A0E0B0E030CD82E090E0A0E0B0E079
:1068C000F9CD82E090E0A0E0B0E0D4CD82E090E0AD
:1068D000A0E0B0E0DFCD6B96EFAD6B97EE23F9F45F
:1068E00024E030E040E050E0820F931FA41FB51F6A
:1068F0000C9430286B96BFAC6B97BB2009F0C5C1D8
:1069000084E090E0A0E0B0E0480E591E6A1E7B1EB5
:106910000C94601C82E090E0A0E0B0E0A3CF22E005
:1069200030E040E050E0E0CF30E021503040D40192
:10693000C301022E04C0B695A795979587950A9432
:10694000D2F72F5F3F4FE82FE1702496EFAF2497E7
:1069500099CB62960EAD1FAD6297005B1E4FD801BA
:10696000ED91FC911197A055B140CD0163E371E029
:1069700009950C94B91F62968EAD9FAD6297B401D4
:10698000A30121E000E0C9800E945E0C0C94770F07
:106990006B965FAC6B97552009F0A0C184E090E046
:1069A000A0E0B0E0680E791E8A1E9B1E0C94612B3D
:1069B000B06460CC042E04C0969487947794679456
:1069C0000A94D2F720E230E0241B350B8FEF9FEFC3
:1069D000AFEFBFEF04C0880F991FAA1FBB1F2A95F6
:1069E000D2F7682A792A8A2A9B2A0C9413146B9668
:1069F000BFAC6B97BB2009F043C184E090E0A0E0FE
:106A0000B0E0280F391F4A1F5B1F0C94B82B6B9600
:106A1000FFAC6B97FF2009F066C184E090E0A0E036
:106A2000B0E0280F391F4A1F5B1F0DCDD801C701E9
:106A30008E7F6296EEADFFAD629784AF95AFA6AF45
:106A4000B7AFE096AEADBFADE0972D913D914D91C2
:106A50005C9113972F7DFD01208331834283538303
:106A6000C70181709070892B09F4D6C520622D93DF
:106A70003D934D935C931397E2CB22E0C22ED12C31
:106A8000E12CF12CEFCD8F81C82EDD24EE24FF24E4
:106A900087FF08C000E01FEF2FEF3FEFC02AD12A89
:106AA000E22AF32A66962CAD3DAD4EAD5FAD6697FA
:106AB0006CE056954795379527956A95D1F7669678
:106AC0002CAF3DAF4EAF5FAF669763960FAD639748
:106AD0000F700F3009F433C5E02FF0E0EE0FFF1F09
:106AE000EE0FFF1F62962EAD3FAD6297E20FF31FD0
:106AF000C082D182E282F38264CA82E090E0A0E0A8
:106B0000B0E085CE6B96DFAC6B97DD2009F035C227
:106B100084E090E0A0E0B0E0280F391F4A1F5B1F1F
:106B20000C94BE1C62968EAD9FAD6297B301A2011C
:106B300024E000E0C9800E945E0C0C94770F289638
:106B40008CAD9DADAEADBFAD28978E7F6296EEAD9C
:106B5000FFAD629784AF95AFA6AFB7AFE096AEAD8D
:106B6000BFADE0972D913D914D915C9113972F7D95
:106B7000FD01208331834283538326968EAD9FADE2
:106B8000269781709070892B11F00C94B31825967C
:106B9000BFAD2597B1FD02C00C94770F0C94B011D6
:106BA00082309105A105B10509F4F7C00397A1054D
:106BB000B10509F49DC0AA24BB2465011CA65CC8CC
:106BC00082E090E0A0E0B0E06CCE82E090E0A0E057
:106BD000B0E0FDCD22E030E040E050E008CE6B9622
:106BE0006FAD6B976623F1F494E0E92EF12C012D43
:106BF000112D2E0D3F1D401F511FEECA6B96EFAC9D
:106C00006B97EE2009F064C584E090E0A0E0B0E06E
:106C1000A80EB91ECA1EDB1EB6CA82E090E0A0E034
:106C2000B0E00FCD82E0E82EF12C012D112DE1CF47
:106C3000D501C4018E7F6296EEADFFAD629784AF41
:106C400095AFA6AFB7AFE096AEADBFADE0972D91D3
:106C50003D914D915C9113972F7DFD0120833183F0
:106C600042835383C40181709070892B09F477C6E5
:106C700020622D933D934D935C9313970C94B22611
:106C800082E090E0A0E0B0E0BCCE82E090E0A0E046
:106C9000B0E03ACED701C6018E7FF90184AF95AF3F
:106CA000A6AFB7AFE096AEADBFADE0972D913D91E9
:106CB0004D915C9113972F7DFD0120833183428399
:106CC0005383C60181709070892B09F465C62062D8
:106CD0002D933D934D935C93139773C982E090E09D
:106CE000A0E0B0E05FCE82E090E0A0E0B0E099CE1E
:106CF00017012801220C331C441C551CA4019301CC
:106D0000205030404040504829AF3AAF4BAF5CAFC5
:106D1000D201C1018E259F25A027B1272E253F2511
:106D20004027512782239323A423B5238827B7FD27
:106D300083959927AA27BB278CA7882331F01701B1
:106D40002801550C2208322C210162015101A60CA8
:106D5000B71CC81CD91CD601C50182259325A425C2
:106D6000B52549AD5AAD6BAD7CAD422553256425A3
:106D7000752584239523A623B723B7FD02C00C9461
:106D80003C2E57FC02C00C94372EAA24AA94BA2C8D
:106D9000650161E06CA70C943C2E17012801220CC0
:106DA000331C441C551CD401C30180509040A040AA
:106DB000B04821968CAF9DAFAEAFBFAF2197D20147
:106DC000C1018E259F25A027B12721962CAD3DAD71
:106DD0004EAD5FAD21972E253F25402751278223B9
:106DE0009323A423B5238827B7FD83959927AA2742
:106DF000BB278CA7882331F017012801550C2208E6
:106E0000322C210162015101A60CB71CC81CD91CEF
:106E1000D601C50182259325A425B52521966CAC04
:106E20007DAC8EAC9FAC219762247324842495247E
:106E300086219721A821B921B7FD02C00C943C2ED0
:106E4000A0CF88A599A5AAA5BBA58E7F6296EEAD19
:106E5000FFAD629784AF95AFA6AFB7AFE096AEAD8A
:106E6000BFADE0972D913D914D915C9113972F7D92
:106E7000FD01208331834283538388A599A58170C6
:106E80009070892B11F00C94B318B8A5B1FD02C015
:106E90000C94770F0C94B01162968EAD9FAD6297F3
:106EA000B301A20124E001E0EE24C9800E945E0C3F
:106EB0000C94770F6B96FFAC6B97FF20C9F484E0BE
:106EC00090E0A0E0B0E0280F391F4A1F5B1F0C9430
:106ED00059266B966FAC6B97662079F484E090E04E
:106EE000A0E0B0E0280E391E4A1E5B1E0C9424263A
:106EF00082E090E0A0E0B0E0E6CF82E090E0A0E0A9
:106F0000B0E0F0CF6B964FAD6B97442389F584E0EA
:106F100090E0A0E0B0E0E80EF91E0A1F1B1F0C94E1
:106F2000592CD601C5018E7F6296EEADFFAD6297FA
:106F300084AF95AFA6AFB7AFE096AEADBFADE0976B
:106F40002D913D914D915C9113972F7DFD012083F3
:106F5000318342835383C50181709070892B11F076
:106F60000C94B318A1FC02C00C94770F0C94B011D0
:106F700082E090E0A0E0B0E0CECF82E090E0A0E040
:106F8000B0E0CACDA1FC02C00C94CB256296EEAD58
:106F9000FFAD6297E05BFE4F6296FFAFEEAF629788
:106FA0000190F081E02D62960EAD1FAD6297005505
:106FB0001140C80163E371E009950C94CB2564018D
:106FC0005301AE18BF08C00AD10AA60195012625B3
:106FD000372548255925D401C30180509040A04051
:106FE000B0488E259F25A027B127282339234A237F
:106FF0005B23222757FD23953327442755272CA7AA
:10700000222311F40C943C2E64015301DD0CAA08D8
:10701000BA2C65010C943C2E262D217024962FAF9E
:1070200024976624772443010C9413146B967FAD48
:107030006B97772341F584E090E0A0E0B0E0280F63
:10704000391F4A1F5B1F0C948F2C6B965FAC6B979C
:107050005520F1F484E090E0A0E0B0E0E80EF91EE5
:107060000A1F1B1F0C94DE2D6B963FAD6B973323CD
:10707000A1F484E090E0A0E0B0E0680E791E8A1EE2
:107080009B1E0C94AE2D82E090E0A0E0B0E0D7CF44
:1070900082E090E0A0E0B0E0E1CF82E090E0A0E00C
:1070A000B0E0EBCF64968EAD9FAD64978070907F1B
:1070B000892B11F00C94B00E63966FAD639765FF4A
:1070C000E1C36201EE24FF24C60180709078892B11
:1070D00041F080E090E0AFEFBFEFC82AD92AEA2A5A
:1070E000FB2A63969FAD639796FF70C39A0144276E
:1070F0005527C90180709078892B11F04F6F5F6F11
:10710000CA01B901A70196010E94156B4B015C01F0
:1071100066962CAC3DAC4EAC5FAC6697C201AA271C
:10712000BB27082F0F7010E00C949E2663966FAC5F
:10713000639765FE40C36201EE24FF24C6018070A0
:107140009078892B51F0812C912C9FEFA92E9FEFE5
:10715000B92EC828D928EA28FB2863969FAC6397E4
:1071600096FE21C39A0144275527C9018070907863
:10717000892B11F04F6F5F6FCA01B901A70196010A
:107180000E94156BAB01BC01DB01CA018827B7FD6A
:1071900083959927AA27BB27782E66968CAD9DAD3F
:1071A000AEADBFAD66971CE0B695A7959795879550
:1071B0001A95D1F7BFE0DB2ED8222D2D30E0220F1B
:1071C000331F220F331F6296EEADFFAD6297E20FC1
:1071D000F31FE080F18002811381FFE0AF2EDA140B
:1071E00009F4D3C26B96CFAC6B97CC2089F06D9627
:1071F0008FAD6D97882361F0ECEF2E2EEFEF3E2ED2
:10720000EFEF4E2EEFEF5E2EE220F320042115214A
:10721000DB01CA018E0D9F1DA01FB11F8E159F059A
:10722000A007B10718F462E0362E73285FE0452E00
:10723000D41409F4DDC262964EAD5FAD6297240F9F
:10724000351FD901ED92FD920D931C93139766960D
:107250002CAC3DAC4EAC5FAC6697C201AA27BB27F5
:10726000082F0F70E02FF0E0EE0FFF1FEE0FFF1F53
:1072700062964EAC5FAC6297E40DF51D8080918004
:10728000A280B3800F3009F4A4C26B966FAC6B97E9
:10729000662069F06D96CFAC6D97CC2041F02CEF55
:1072A0003FEF4FEF5FEF82229322A422B522872D7A
:1072B00071FE05C00894811C911CA11CB11C80FFAB
:1072C00032CF089481089108A108B10810E00C940D
:1072D0009E2663966FAD639765FFCBC36201EE2474
:1072E000FF24C60180709078892B41F080E090E007
:1072F000AFEFBFEFC82AD92AEA2AFB2A63969FADCF
:10730000639796FFAEC39A0144275527C901807041
:107310009078892B11F04F6F5F6FCA01B901A701F7
:1073200096010E94156B9B01AC0166968CAD9DADDC
:10733000AEADBFAD66976CE0B695A795979587956E
:107340006A95D1F78F70E82FF0E0EE0FFF1FEE0F78
:10735000FF1F6296AEADBFAD6297EA0FFB1FE080E4
:10736000F180028113818F3009F46DC36B96EFAD0C
:107370006B97EE2389F06D96FFAD6D97FF2361F05B
:107380008CEF282E8FEF382E8FEF482E8FEF582E50
:10739000E220F3200421152147015801820E931E9B
:1073A000A41EB51ED501C4018E259F25A027B12797
:1073B00020503040404050482E253F25402751273F
:1073C00082239323A423B5238827B7FD8395992788
:1073D000AA27BB27182F66964CAC5DAC6EAC7FAC71
:1073E0006697C301AA27BB27082F0F700C949E260F
:1073F00063966FAC639766FEA7C25A01CC24DD2466
:10740000C50180709078892B51F0E12CF12CFFEFB1
:107410000F2FFFEF1F2FAE28BF28C02AD12A8601C9
:107420007501110FEE08FE2C870142013101990C04
:107430006608762C43019501A6016E2D7E2D8E2DBA
:107440009E2D51016201E62CF62C062D162D0E9470
:10745000500100E10E944B0269017A0163960FAD71
:10746000639705FF1AC264968EAD9FAD64978070D6
:10747000907F892B11F00C94B00E66962CAD3DAD2B
:107480004EAD5FAD6697CA01AA27BB27082F0F70C4
:107490004601570110E00C949E26D701C6018E7F4D
:1074A0006296EEADFFAD629784AF95AFA6AFB7AF72
:1074B000E096AEADBFADE0972D913D914D915C91C1
:1074C00013972F7DFD012083318342835383C601AF
:1074D00081709070892B09F427C120622D933D9310
:1074E0004D935C931397CB84DC84ED84FE84E0E1C0
:1074F000F0E00C94D32F8F8198856C01EE24FF244B
:1075000040E14416510409F401C166968CAD9DAD6D
:10751000AEADBFAD66973CE0B695A79597958795BC
:107520003A95D1F766968CAF9DAFAEAFBFAF669779
:1075300063960FAD63970F700F3009F0CDCAD70176
:10754000C6018E7F6296EEADFFAD6297A7CB6296C5
:107550008EAD9FAD6297B401A30121E0EE24C980F6
:107560000E945E0C0C94770F6B96BFAD6B97BB239C
:1075700089F584E090E0A0E0B0E0680E791E8A1EF4
:107580009B1E0C948F30D601C5018E7F6296EEADA6
:10759000FFAD629784AF95AFA6AFB7AFE096AEAD43
:1075A000BFADE0972D913D914D915C9113972F7D4B
:1075B000FD012083318342835383C5018170907024
:1075C000892B69F020622D933D934D935C93139723
:1075D0000C94672E82E090E0A0E0B0E0CECFA1FC5A
:1075E00002C00C94672E6296EEADFFAD6297E05B31
:1075F000FE4F6296FFAFEEAF62970190F081E02DF3
:1076000062960EAD1FAD629700551140C80163E34D
:1076100071E009950C94672EE1FC02C00C941F31B7
:107620006296EEADFFAD6297E05BFE4F6296FFAFF4
:10763000EEAF62970190F081E02D62962EAD3FADE6
:10764000629720553140C90163E371E009950C94BC
:107650001F3121FC02C00C94B5256296EEADFFAD42
:107660006297E05BFE4F6296FFAFEEAF62970190CC
:10767000F081E02D62960EAD1FAD6297005511406E
:1076800062961FAF0EAF6297C80163E371E0099580
:107690000C94B5256B965FAD6B975523F1F484E0A0
:1076A00090E0A0E0B0E0E80EF91E0A1F1B1F0C944A
:1076B0005C2D6B96BFAD6B97BB23A1F484E090E08B
:1076C000A0E0B0E0280F391F4A1F5B1F0C94043361
:1076D00082E090E0A0E0B0E09BCA82E090E0A0E011
:1076E000B0E0E1CF82E090E0A0E0B0E0EBCF6B96BD
:1076F0003FAD6B97332309F584E090E0A0E0B0E064
:10770000E80EF91E0A1F1B1F0C94871580709078D5
:10771000892B09F4FACE60E070E08FEF9FEFC62A64
:10772000D72AE82AF92AF1CEC1FC0CC000E1CB84AB
:10773000DC84ED84FE840C94D12F82E090E0A0E004
:10774000B0E0DECF6296EEADFFAD6297E05BFE4F3C
:107750006296FFAFEEAF62970190F081E02D6296E6
:107760000EAD1FAD62970055114062961FAF0EAF70
:107770006297C80163E371E00995CB84DC84ED84F2
:10778000FE84E0E1F0E00C94D32F6B96BFAC6B97D6
:10779000BB2061F484E090E0A0E0B0E0E80EF91EC8
:1077A0000A1F1B1F1FCD40705070DFCC82E090E09D
:1077B000A0E0B0E0F3CF6FEFC62E6FEFD62EE12C36
:1077C000F12CC220D320E420F520B8CC40705070BA
:1077D00090CC6B965FAC6B97552081F524E0C22E60
:1077E000D12CE12CF12C8C0C9D1CAE1CBF1C4DCD62
:1077F000D801C7018E7F6296EEADFFAD629784AF70
:1078000095AFA6AFB7AFE096AEADBFADE0972D9107
:107810003D914D915C9113972F7DFD012083318324
:1078200042835383C70181709070892B69F0206275
:107830002D933D934D935C93139709CD92E0C92E00
:10784000D12CE12CF12CCFCFE1FE01CD6296EEAD33
:10785000FFAD6297E05BFE4F6296FFAFEEAF6297BF
:107860000190F081E02D62960EAD1FAD629700553C
:10787000114062961FAF0EAF6297C80163E371E0DB
:107880000995E5CC0FEFC02E0FEFD02EE12CF12C97
:10789000C220D320E420F52017CC66968CAD9DAD98
:1078A000AEADBFAD66972CE0B695A7959795879539
:1078B0002A95D1F78F70E82FF0E0EE0FFF1FEE0F43
:1078C000FF1F62964EAD5FAD6297E40FF51F2081FA
:1078D0003181428153818F3041F16B967FAD6B973F
:1078E000772329F06D968FAD6D9781112C7F49011B
:1078F0005A018C0C9D1CAE1CBF1CD501C4018C25EB
:107900009D25AE25BF25212C312C412C10E8512E70
:10791000C20CD31CE41CF51CC226D326E426F52693
:107920008C219D21AE21BF214FCD6B966FAD6B9702
:10793000662309F0A9C084E090E0A0E0B0E0280F41
:10794000391F4A1F5B1FC9CFAFEFAA2EAFEFBA2E68
:10795000C12CD12CA222B322C422D52251CD81FC2C
:1079600002C00C94B2266296EEADFFAD6297E05B6A
:10797000FE4F6296FFAFEEAF62970190F081E02D6F
:1079800062962EAD3FAD629720553140C90163E349
:1079900071E009950C94B226C1FC02C00C94E12F51
:1079A0006296EEADFFAD6297E05BFE4F6296FFAF71
:1079B000EEAF62970190F081E02D62960EAD1FADA3
:1079C00062970055114062961FAF0EAF6297C801D3
:1079D00063E371E009950C94E12F6B963FAC6B97D4
:1079E000332039F584E090E0A0E0B0E0C80ED91E65
:1079F000EA1EFB1E0C9497326B964FAD6B97442397
:107A0000E9F484E090E0A0E0B0E06A962CAC3DACF4
:107A10004EAC5FAC6A97820D931DA41DB51D629696
:107A2000EEADFFAD629780AF91AFA2AFB3AF0C9454
:107A30007F3282E090E0A0E0B0E0D8CF83E090E039
:107A4000A0E0B0E0E2CF6B96BFAD6B97BB2361F4D3
:107A500084E090E0A0E0B0E0E80EF91E0A1F1B1FD2
:107A600085CC4070507052CC82E090E0A0E0B0E055
:107A7000F3CFEFEFCE2EEFEFDE2EE12CF12CC22074
:107A8000D320E420F5202DCC82E090E0A0E0B0E00F
:107A900056CF2F923F924F925F926F927F928F922A
:107AA0009F92AF92BF92CF92DF92EF92FF920F938D
:107AB0001F93DF93CF93CDB7DEB72F970FB6F89410
:107AC000DEBF0FBECDBF8A559F4FDC018D919C91CB
:107AD0001197A65AB040BD87AC87892B09F075C0B5
:107AE000A05CBF4FBF87AE872C853D852C553F4F8F
:107AF000D9018D919C911197A45AB040BD87AC8754
:107B0000892B09F073C1EE85FF8580819181A28167
:107B1000B38185FDCCC077248F719070A070B07058
:107B20004097A105B10511F077247394AC85BD850C
:107B3000DC968D909D90AD90BC90DF97CD018A5AD8
:107B40009E4FB501A40124E0072D7E010894E11C9D
:107B5000F11CE4E0CE2ED12CCC0EDD1E0E9414567A
:107B6000882309F473C1EC85FD8584AD95ADA6AD80
:107B7000B7AD0496A11DB11D84AF95AFA6AFB7AF49
:107B80004C815D816E817F81CF0195018401EE245E
:107B9000C72CAA240E94F50D2F960FB6F894DEBFCD
:107BA0000FBECDBFCF91DF911F910F91FF90EF904E
:107BB000DF90CF90BF90AF909F908F907F906F900D
:107BC0005F904F903F902F900895EC85FD85E05C8D
:107BD000FF4FFF87EE87608071808280938066FC14
:107BE00083CFA0E2AA2EAFEFBA2EAFEFCA2EAFEF2F
:107BF000DA2EA620B720C820D92001ED10E020E021
:107C000030E0A02AB12AC22AD32A2C853D85265BE2
:107C10003E4FD9012D903D904D905C901397AA5402
:107C2000B140BD87AC870CE110E020E030E0200ED1
:107C3000311E421E531EAC85BD85DC96ED90FD9035
:107C40000D911C91DF9724E030E040E050E0E20E1F
:107C5000F31E041F151F6A2D6F71CD010E94C90B01
:107C6000AE85BF85AD92BD92CD92DC921397EC8527
:107C7000FD85EC5BFF4FDF0160827182828293821F
:107C8000A454B040BD87AC87FD01E0AEF1AE02AFB9
:107C900013AFDC962D923D924D925C92DF97EE856C
:107CA000FF8580819181A281B38185FF34CF7724C4
:107CB0008F719070A070B0704097A105B10511F060
:107CC00077247394AC85BD85DC968D909D90AD90A6
:107CD000BC90DF97CD018A5A9E4FB501A40122E0E6
:107CE000072D7E010894E11CF11CE2E0CE2ED12C80
:107CF000CC0EDD1E0E941456882309F4FAC0EC85D0
:107D0000FD85C4ACD5ACE6ACF7AC02E010E020E0F9
:107D100030E0C00ED11EE21EF31EC4AED5AEE6AEFC
:107D2000F7AE4A815B81CA01892F992782958F70AE
:107D30008730910509F4E0C28830910508F495C0B8
:107D40008B30910509F448C38C30910508F431C19A
:107D50008D30910509F4A2C20D9708F05BC28A012B
:107D600020E030E07FEFC72ED12CE12CF12CC02297
:107D7000D122E222F32280E090E0A0E8B8EEC82A07
:107D8000D92AEA2AFB2AD901C80180709770A0700D
:107D9000B070BA2FA92F982F8827C82AD92AEA2A83
:107DA000FB2A53FF08C080E090E0A0E1B0E0C82AC1
:107DB000D92AEA2AFB2A852F99278770907004C058
:107DC00036952795179507958A95D2F7C801817042
:107DD0009070892B09F0F8C100E010E020E230E05B
:107DE000C02AD12AE22AF32AE0E0D6C0EE85FF8538
:107DF000608071808280938067FC85CEF0E6AF2E34
:107E0000FFEFBF2EFFEFCF2EFFEFDF2EA620B72014
:107E1000C820D92002E910E020E030E0A02AB12AF1
:107E2000C22AD32AA65BBE4F2D903D904D905C9008
:107E30001397AA54B140BD87AC8728E130E040E0F9
:107E400050E0220E331E441E551EF5CEEC85FD85F6
:107E500044AD55AD66AD77ADCF0124E000E0EE2432
:107E6000E394C9800E945E0C97CE8430910508F09F
:107E70004CC0029708F4CDC08A0120E030E07FEFCB
:107E8000C72ED12CE12CF12CC022D122E222F322E8
:107E900080E090E0A0E0B0EEC82AD92AEA2AFB2AC6
:107EA000CA01892F9927869586958695837090704B
:107EB0008130910509F4C3C48130910508F039C3BC
:107EC0004070577042955295507F5427407F5427F9
:107ED000CA01A0E0B0E0C82AD92AEA2AFB2A00E0B9
:107EE00010E020EB33E0C02AD12AE22AF32AE0E0B6
:107EF00053C08C859D85B501A40122E000E0EE24ED
:107F0000E394C9800E945E0C47CE8530910509F448
:107F1000CDC0069708F45AC1CA0187709070982F97
:107F200088279295907F6C01EE24FF24CA01A0E07F
:107F3000B0E088739070A070B070EDE0880F991F6A
:107F4000AA1FBB1FEA95D1F7C82AD92AEA2AFB2A19
:107F500000E010E020E835EEC02AD12AE22AF32A18
:107F6000CA01929582958F7089279F708927A0E01A
:107F7000B0E08C779070A070B070C82AD92AEA2A35
:107F8000FB2A53FF21C120E030E040E150E0C22A4B
:107F9000D32AE42AF52AE0E08C859D85B701A60165
:107FA00095018401EE24E394C72CAE2E0E94F50DBA
:107FB000F3CD8930910509F4E3C10A9708F4BEC0F6
:107FC000CA018070977082959295907F9827807FE4
:107FD00098279A013070822B932BA0E0B0E0C12C3F
:107FE0000FE0D02E0DE8E02E02EEF02EC82AD92A9E
:107FF000EA2AFB2A53FD8FC2C12C1FE0D12E1FE8B5
:10800000E12E12EEF12EC82AD92AEA2AFB2AE0E054
:10801000C3CFCA01807098718050984109F4D4C2CE
:10802000CA0187709070982F88279295907F6C0175
:10803000EE24FF24CA019695879596958795969587
:108040008795A0E0B0E087709070A070B070C82AEB
:10805000D92AEA2AFB2A00E010E020EB31EEC02A00
:10806000D12AE22AF32ACA010024880F991F001C92
:10807000880F991F001C892F902DA0E0B0E080761A
:108080009070A070B070C82AD92AEA2AFB2A440F3F
:10809000551FCA01A0E0B0E080789F70A070B0705A
:1080A000C82AD92AEA2AFB2AE0E076CF6A01EE2420
:1080B000FF2408E310E020E030E0C022D122E222D9
:1080C000F3220DE0CC0CDD1CEE1CFF1C0A95D1F751
:1080D000FA01EE0FEF2FEE1FFF0BF195EC71F07030
:1080E000E65FFD4F80819181A281B381C82AD92AA0
:1080F000EA2AFB2A80E090E0A0E0B0EEC82AD92A64
:10810000EA2AFB2ACA0187709070982F88279295D7
:10811000907F0024440F551F001C440F551F001C66
:10812000452F502D47705070842B952BA0E0B0E068
:10813000C82AD92AEA2AFB2AE0E02ECFCA01877092
:108140009070982F88279295907F6C01EE24FF24E1
:10815000CA01A0E0B0E088739070A070B0701DE01C
:10816000880F991FAA1FBB1F1A95D1F7C82AD92AB1
:10817000EA2AFB2A80EB90E0A0ECB1EEC82AD92ACB
:10818000EA2AFB2ACA0196958795929582958F7067
:1081900089279F708927A0E0B0E08E709070A07052
:1081A000B070C82AD92AEA2AFB2ACA01969587956F
:1081B000A0E0B0E080709370A070B070C82AD92A97
:1081C000EA2AFB2A53FDD2C0E0E0E6CE53FF5DC1B0
:1081D000CA019070880F991F880F991F6C01EE24B7
:1081E000FF244070577042955295507F5427407F2E
:1081F0005427CA01A0E0B0E0C82AD92AEA2AFB2AFB
:1082000000E010E02FE935EEC02AD12AE22AF32A55
:10821000E1E0C2CEBA017770CA01892F992786950D
:1082200086958695837090708130910509F4D6C249
:108230008130910508F071C18B0120E030E0D90157
:10824000C801BA6E52FF05C0D901C801986FAF6F5F
:10825000BA6E53FDF2C06A01EE24FF240FEF17E05F
:1082600020E030E0C022D122E222F32200E010E040
:1082700020E03AE0C02AD12AE22AF32AC82AD92AE1
:10828000EA2AFB2A52FFA0CF20E038EF4FEF50E060
:10829000C22AD32AE42AF52AE0E07ECE852F8F7009
:1082A0008E3009F4CAC08F3009F48AC2C42EDD248E
:1082B000EE24FF2400E010E020E03AE0C02AD12ABA
:1082C000E22AF32A90E0A0E0B0E0FCE1880F991FD9
:1082D000AA1FBB1FFA95D1F7C82AD92AEA2AFB2A76
:1082E00047FF72CF20E03FEF4FEF50E0C22AD32A82
:1082F000E42AF52AE0E050CECA0187709070982FEA
:1083000088279295907F6C01EE24FF24CA01A0E09B
:10831000B0E088739070A070B0703DE0880F991F36
:10832000AA1FBB1F3A95D1F7C82AD92AEA2AFB2AE5
:1083300080E090E0A0ECB5EEC82AD92AEA2AFB2A10
:10834000CA010024880F991F001C880F991F001C68
:10835000892F902DA0E0B0E08F719070A070B07068
:10836000C82AD92AEA2AFB2A53FF2ECF00E010E0C0
:1083700020E130E0C02AD12AE22AF32AE0E00CCE44
:108380009A013070220F331F220F331FCA018070F1
:10839000977082959295907F9827807F9827282BB9
:1083A000392BC901A0E0B0E0C12CD12C6DE8E62E3C
:1083B00065EEF62EC82AD92AEA2AFB2A53FF04CFF3
:1083C000C12CD12C3DE9E32E35EEF32EC82AD92A53
:1083D000EA2AFB2AE0E0E0CDCA0180709670805066
:1083E000944009F4D2C050FD28C0CA01892F9927B2
:1083F000869587709070009709F08EC247FDCBC2BA
:1084000080E090E0A0E8B0E06A01EE24FF242FE7CE
:1084100030E040E050E0C222D322E422F52200E026
:108420001FED2DE032EEC02AD12AE22AF32AC82A13
:10843000D92AEA2AFB2AE0E0AFCD3BEB4B3B5307BE
:1084400009F413C16A01EE24FF248FEF90E0A0E04D
:10845000B0E0C822D922EA22FB2200EF10E020EF90
:1084600037EEC02AD12AE22AF32A407F429552955C
:10847000507F5427407F5427CA01A0E0B0E0C82AAB
:10848000D92AEA2AFB2AE0E087CD52FFF8C0CA01C8
:10849000929582958F7089279F708927282F287041
:1084A000842F8770282BCA01969587959695879576
:1084B00096958795E82FEF70052F112703701070A0
:1084C0000130110509F46CC20130110508F055C2E4
:1084D00030E040E050E0CE2EDD24EE24FF2480E0AA
:1084E00090E0A0E8B0EEC82AD92AEA2AFB2AD901EE
:1084F00099278827C82AD92AEA2AFB2AACE0220F22
:10850000331F441F551FAA95D1F7C22AD32AE42A44
:10851000F52AE0E041CDE1E03FCD8230910509F45C
:10852000CEC1039709F4A1C180E090E0A0E0B0EED5
:1085300090CE8230910509F4DBC1039709F044CE57
:108540004070577042955295507F5427407F542772
:10855000CA01A0E0B0E0C82AD92AEA2AFB2A80E0B2
:1085600090E0A0E5B2E0C82AD92AEA2AFB2A0070E6
:10857000177020703070B22FA12F902F8827C82A33
:10858000D92AEA2AFB2AE0E007CDCA01A0E0B0E040
:108590009070A070B0708C019D012D60306E53FF03
:1085A000D4C150FF05C08C019D0110682D60306E54
:1085B000C12CD12CA0EBEA2EA8E0FA2EC02AD12A99
:1085C000E22AF32AE0E0E8CC51FDD2C100E010E05D
:1085D00020E930E06A01EE24FF2488E390E0A0E087
:1085E000B0E0C822D922EA22FB22ADE0CC0CDD1C8F
:1085F000EE1CFF1CAA95D1F7CA0187709070982FC6
:1086000088279295907FA0E0B0E0C82AD92AEA2A6C
:10861000FB2A80E090E0A0E0B0EEC82AD92AEA2A3E
:10862000FB2ACA010024880F991F001C880F991F7C
:10863000001C892F902DA0E0B0E087709070A07092
:10864000B070C82AD92AEA2AFB2AC02AD12AE22AEB
:10865000F32A52FFB9CD00E010E020E032E0C02A5A
:10866000D12AE22AF32AE0E097CCABEBCA2EABEB9F
:10867000DA2EABEBEA2EA7EFFA2EE0E08DCC1886CF
:1086800019861A861B86842F87708A875695479588
:108690005695479556954795842F87708B875695A5
:1086A00047955695479556954795E42FEF702E2F91
:1086B000220FF0E0EE0FFF1FEE0FFF1FE65DFD4FF4
:1086C000C080D180E280F38080E090E0A0E0B0EE56
:1086D000C82AD92AEA2AFB2A8FEA9EEBA3EFBFEF2A
:1086E000022E04C0B695A795979587950A94D2F760
:1086F00083709070FE0138968E0F9F1FDC018C9165
:1087000090E0A0E0B0E0C82AD92AEA2AFB2A8AE051
:1087100098E2AEEABAE2022E04C0B695A795979504
:1087200087950A94D2F7837090708E0F9F1FDC019B
:108730008C9190E0A0E0B0E0DC0199278827C82A5E
:10874000D92AEA2AFB2A8AEA9AEAA8E0B2EA022EA1
:1087500004C0B695A795979587950A94D2F783702C
:1087600090708E0F9F1FDC018C9190E0A0E0B0E034
:108770003CE0880F991FAA1FBB1F3A95D1F7C82A62
:10878000D92AEA2AFB2A80EF93ECA0E0B8E004C0E3
:10879000B695A795979587952A95D2F7837090708F
:1087A000E80FF91F808190E0A0E0B0E0BA2FA92F78
:1087B000982F8827C82AD92AEA2AFB2AE0E0ECCB9E
:1087C000C42EDD24EE24FF2420E030E040E05FEE04
:1087D000C22AD32AE42AF52AE0E0DECBEC85FD8527
:1087E00080AD91ADA2ADB3AD0296A11DB11D9B01AF
:1087F00040E050E0220F331F441F551F820F931F8C
:10880000A41FB51F8C7F84AF95AFA6AFB7AF01E0B3
:1088100010E020E030E0C02AD12AE22AF32AC0AEDC
:10882000D1AEE2AEF3AEEE85FF8580819181A2816B
:10883000B3818F7D80839183A283B383ADC90070A0
:10884000177020703070B22FA12F902F8827C82A60
:10885000D92AEA2AFB2A20E030E040E553E0C22A88
:10886000D32AE42AF52AE0E097CBAC85BD85D896DB
:108870002D913D914D915C91DB972E5F3F4F4F4F76
:108880005F4FCB01A0E0B0E0880F991FAA1FBB1F6C
:10889000280F391F4A1F5B1FEC85FD8524AF35AFBC
:1088A00046AF57AF01E010E020E030E0C02AD12A07
:1088B000E22AF32AC0AED1AEE2AEF3AE6DC9CB016F
:1088C000A0E0B0E052FF02C0986FAF600CE0880FEC
:1088D000991FAA1FBB1F0A95D1F78C0D9D1DAE1DB8
:1088E000BF1DEC85FD8580AF91AFA2AFB3AF54C97A
:1088F0004070577042955295507F5427407F5427BF
:10890000CA01A0E0B0E0C82AD92AEA2AFB2A80E0FE
:1089100090E0A0E9B2E027CE079709F08ECD6A017A
:10892000EE24FF248FE090E0A0E0B0E0C822D9223E
:10893000EA22FB2200E710E020E231EEC02AD12A31
:10894000E22AF32A407F507091CD50FF05C08C0180
:108950009D0110642D60306EC12CD12CF0E2EF2E01
:10896000F9E0FF2EC02AD12AE22AF32AE0E014CB54
:1089700000E010E020E530E02DCE0230110509F4D2
:1089800040C00330110529F1C12CD12CE12CB0EEEF
:10899000FB2EE0E001CB80E090E0A0E4B0E034CD3D
:1089A000CE2EDD24EE24FF2480E090E0A0E5B1EEA1
:1089B000C82AD92AEA2AFB2A822F90E0A0E0B0E058
:1089C000DC0199278827C82AD92AEA2AFB2AE0E06D
:1089D000E3CA4857574491F16C01EE24FF240FE09D
:1089E00010E020E030E0C022D122E222F32220E198
:1089F0003FEF4FE251EEC22AD32AE42AF52AE0E003
:108A0000CBCACE2EDD24EE24FF2480E090E0A0EA45
:108A1000B1EEC82AD92AEA2AFB2A822F90E0A0E0E8
:108A2000B0E0ECE0880F991FAA1FBB1FEA95D1F7B1
:108A3000C82AD92AEA2AFB2AE0E0AECA02E010E0FE
:108A400020E030E0C00ED11EE21EF31E2CEF3FEFFF
:108A50004FEF5FEFC222D322E422F522AC85BD8521
:108A6000DC96CD92DD92ED92FC92DF97EE85FF854C
:108A700080819181A281B3818F7D80839183A28344
:108A8000B3838AC86F927F928F929F92AF92BF9268
:108A9000CF92DF92EF92FF920F931F93CF93DF93CA
:108AA000EC014A015B0139016CE97FE10E94240A73
:108AB000FE01E05CFF4FD501C4018E7F8CAF9DAFFE
:108AC000AEAFBFAF83ED90E0A0E0B0E080839183D4
:108AD000A283B383C40181709070892B69F581FCF6
:108AE0003AC080E5A82E81E0B82EAC0EBD1EC25B58
:108AF000DE4F79826882F501118300832496E99222
:108B0000F992D982C882C455D140CE018A5A9E4F6B
:108B1000BE01A3010E94955580E0DF91CF911F9186
:108B20000F91FF90EF90DF90CF90BF90AF909F900C
:108B30008F907F906F90089583EF90E0A0E0B0E079
:108B400080839183A283B38390E5A92E91E0B92E0F
:108B5000AC0EBD1ECCCFB0E5AB2EB1E0BB2EAC0E43
:108B6000BD1ED501ED91FC91CE0163E371E0099545
:108B7000BECFDC01159640E050E0FA01EE0FFF1F7A
:108B8000E40FF51FEE0FFF1FEE0FFF1FE40FF51FA1
:108B9000EE0FFF1FEE0FFF1FEE0FFF1FE35BFF4FF8
:108BA000E80FF91F20E010821182128213822F5FDA
:108BB0003D962830C1F790961C9290971D924F5F7A
:108BC0005F4F40325105C9F608950F931F93CF931D
:108BD000DF938C01EC012596DE0120E030E0F90105
:108BE000EE0FFF1FE20FF31FEE0FFF1FEE0FFF1F31
:108BF000E20FF31FEE0FFF1FEE0FFF1FEE0FFF1F21
:108C0000E35BFF4FE00FF11F80E0108211821282C0
:108C100013828F5F3D968830C1F790961C92909793
:108C20001D922F5F3F4F20323105C9F680E018A218
:108C300019928F5F8032D9F7F801408351836283A4
:108C40007383DF91CF911F910F910895FC016170A3
:108C500084818E7F862B84830895FC016170660F6A
:108C600084818D7F862B84830895FC01EB5BF24F1A
:108C700060817181828193810895FC01EB5BF24FE9
:108C8000408351836283738308952F923F924F9262
:108C90005F926F927F928F929F92AF92BF92CF928C
:108CA000DF92EF92FF920F931F93DF93CF93CDB795
:108CB000DEB7A3970FB6F894DEBF0FBECDBF1C0181
:108CC000488B598B6A8B7B8B2C8B0D8BFF8AEE8AA2
:108CD000D98EC88EDC014D905D906D907C9048A23D
:108CE00059A26AA27BA2A30192012F5F3F4F4F4F6F
:108CF0005F4F09F443C188899989AA89BB892AE011
:108D0000B695A795979587952A95D1F78A879B87DA
:108D1000AC87BD8788899989AA89BB890FE0B695F8
:108D2000A795979587950A95D1F7288939894A8912
:108D30005B8914E156954795379527951A95D1F794
:108D400082279327A427B5274A845B846C847D847B
:108D500084259525A625B7258F71082F10E03101B0
:108D6000600E711E7B8E6A8ED30115963C9120E0B9
:108D700088E690E0089FA001099F500D189F500DB4
:108D8000112436C0832F90E0FC01EE0FFF1FE80F87
:108D9000F91FEE0FFF1FEE0FFF1FE80FF91FE40F83
:108DA000F51FE20DF31DE75BFF4F81909190A190BD
:108DB000B190C080D180E280F380ED54F0404888CB
:108DC00059886A887B88481459046A047B0460F0D7
:108DD000D701C601880D991DAA1DBB1D481659064D
:108DE0006A067B0608F4EBC02F5F283039F031505B
:108DF0003F3F41F637E087E090E0C6CF88A199A1D8
:108E0000AAA1BBA183709070A070B0700097A1055B
:108E1000B105F1F081E0E88DF98D808380E0A396C3
:108E20000FB6F894DEBF0FBECDBFCF91DF911F917B
:108E30000F91FF90EF90DF90CF90BF90AF909F90F9
:108E40008F907F906F905F904F903F902F900895FC
:108E5000288939894A895B8920703070407F2E8348
:108E60003F8348875987A101475B524F5D8F4C8FE5
:108E7000C101855B924F9F8F8E8F2E813F814885E8
:108E80005985E2E15695479537952795EA95D1F7AB
:108E900048A059A06AA07BA0240D351D461D571D72
:108EA000AC8DBD8DED91FC91DC018D919C913E01CD
:108EB0000894611C711CB3010995882309F479C0D9
:108EC00029813A814B815C81DA01C90175E0B6954F
:108ED000A795979587957A95D1F7F82FFF70FF871B
:108EE000DA01C90183709070A070B0708130910573
:108EF000A105B10509F4ADC181309105A105B10508
:108F000008F4C5C082309105A105B10509F4EDC092
:108F10000397A105B10509F4CEC055245394AC8D37
:108F2000BD8DED91FC91AE8DBF8D8D919C91B30166
:108F30000995882309F4B7C029813A814B815C8166
:108F4000DA01C90183709070A070B0708130910512
:108F5000A105B10509F436C281309105A105B1051D
:108F600008F09CC15F84550C550C550C550C252DF3
:108F70002760A88DB98D2C9380E051CF8824992447
:108F80005401442455243201288939894A895B894E
:108F9000420E531E641E751E481859086A087B0845
:108FA000AE89BF894D925D926D927C92139781E05C
:108FB00036CF8CE0E88DF98D808380E030CFEB5B9D
:108FC000FF4F40805180628073803C968081282FC3
:108FD00023702E87869586958F708F87AA8DBB8D7F
:108FE00015963C93A0E0FF856F2F70E025E43DE0EF
:108FF000220E331ECB01880F991FF1012081318190
:1090000042815381EBEBF2EF2E0E3F1E04C05695CA
:109010004795379527958A95D2F723703070407021
:109020005070223031054105510559F0233031058A
:109030004105510509F4A8CF211531054105510518
:1090400021F4AA2351F58BE016C0BE85B13039F169
:10905000B13008F01CC1ED89EE2349F4F10184819F
:1090600081FD92CFFC89FF2311F080FD8DCFAA23D3
:1090700009F09DC18FE062957295707F7627607FC1
:109080007627862BA88DB98D8C9380E0C8CE85E09D
:10909000A88DB98D8C9380E0C2CE88E0ECCF2C896E
:1090A000222329F371CFBF85B295B07FBE60E88DD2
:1090B000F98DB083B4CE2070307F88899989AA89D0
:1090C000BB8980709C7FAF70B070892F9A2FAB2FB7
:1090D000BB27820F931FA41FB51F89839A83AB837D
:1090E000BC8355249C01AD011ACF412C512CB0EF0B
:1090F0006B2EBFEF7B2E4222532264227522AAE000
:109100005695479537952795AA95D1F7B22FB37005
:10911000BE878E809F80A884B984C12CD12CF0E1B9
:10912000EF2EF12CA1E0EA8DFB8D85A190E0FC01F2
:10913000EE0FFF1FE80FF91FEE0FFF1FEE0FFF1FCF
:10914000E80FF91F88E690E0089F9001099F300D15
:10915000189F300D1124E20FF31FE20DF31DEB5B9E
:10916000FF4F4082518262827382EA8DFB8D85A11E
:1091700090E0FC01EE0FFF1FE80FF91FEE0FFF1F3D
:10918000EE0FFF1FE80FF91FE20FF31FE20DF31DB3
:10919000E35BFF4FC082D182E282F382EA8DFB8DD6
:1091A00085A190E0FC01EE0FFF1FE80FF91FEE0F05
:1091B000FF1FEE0FFF1FE80FF91FE20FF31FE20D75
:1091C000F31DE75BFF4F80829182A282B382EA8D1A
:1091D000FB8D85A190E0FC01EE0FFF1FE80FF91F4A
:1091E000EE0FFF1FEE0FFF1FE80FF91FE20FF31F37
:1091F000E20DF31DEF5AFF4F80818C7F4E85842B4B
:109200008083EA8DFB8D85A190E0FC01EE0FFF1FAE
:10921000E80FF91FEE0FFF1FEE0FFF1FE80FF91FFA
:10922000E20FF31FE20DF31DEF5AFF4F9F859F7072
:10923000990F990F8081837C892B8083EA8DFB8D28
:1092400085A185838F5F85A3883009F0CCCE15A2D8
:10925000CACE20703C7F88899989AA89BB89807091
:10926000907FAF70B0706AE0B695A7959795879597
:109270006A95D1F7820F931FA41FB51F89839A8324
:10928000AB83BC83552453949C01AD0148CEB230CE
:1092900009F48FC0B33009F0EACE76CE8230910562
:1092A000A105B10509F4E3C00397A105B10509F4CF
:1092B000B3C04424552432011D82E4E056954795FD
:1092C00037952795EA95D1F7622FE62FF0E09F01B9
:1092D0002F703070862F82958F7090E02817390795
:1092E00059F4862F8695869590E08E279F27837068
:1092F0009070892B09F457C082E792E00E945B08C6
:10930000AD812A2F30E02E5F3F4F220F331F89811E
:109310009A81AB81BC8104C0B695A7959795879536
:109320002A95D2F7E82FE370EE87F694E794D79466
:10933000C794F694E794D794C7946E2F70E080E0BA
:1093400090E0A70196010E94156B460E571E681EFD
:10935000791E860E971EA81EB91EA0E0E4CE412CF1
:1093600070EF572E7FEF672E7FEF772E422253222A
:109370006422752288889988AA88BB8880E090EF4B
:10938000AFEFBFEF88229922AA22BB2264E0569554
:109390004795379527956A95D1F7622FC12C90E1B3
:1093A000D92EE12CF12C63706E87A0E0BCCE8DE04D
:1093B00062CE3C89332309F0E7CD4D89442309F47B
:1093C000E3CD55CE412C512C7FEF672E7FEF772ECA
:1093D000422253226422752288889988AA88BB88F1
:1093E00080E090E0AFEFBFEF88229922AA22BB2253
:1093F00088899989AA89BB896EE0B695A7959795C2
:1094000087956A95D1F7E82FE370ED83C12CD12CB5
:1094100081E0E82EF12C51CF552009F0A0CF412C4E
:10942000ECEF5E2EEFEF6E2EEFEF7E2E42225322F8
:109430006422752288889988AA88BB8880E09CEF7E
:10944000AFEFBFEF88229922AA22BB2274E0569583
:109450004795379527957A95D1F7922F93709E87E8
:10946000C12C64E0D62EE12CF12CA0E05CCE412C86
:10947000B0EF5B2EBFEF6B2EBFEF7B2E422253224D
:109480006422752288889988AA88BB8880E090EF3A
:10949000AFEFBFEF88229922AA22BB229A85937050
:1094A0009D83A4E05695479537952795AA95D1F7C2
:1094B000622FC12CF0E1DF2EE12CF12C06CFEF92D0
:1094C000FF920F931F93CF93DF93EC018B017A01EF
:1094D0006DE47DE00E94240AC75BD24F0993199383
:1094E000F982E882CB54DD408FEF9FEFAFEFBFEF03
:1094F00088839983AA83BB83CB5BD24F188219825E
:109500001A821B82C554DD40DE01159620E030E052
:10951000F901EE0FFF1FE20FF31FEE0FFF1FEE0F1B
:10952000FF1FE20FF31FEE0FFF1FEE0FFF1FEE0FE7
:10953000FF1FE35BFF4FEC0FFD1F80E010821182E5
:10954000128213828F5F3D968830C1F790961C92ED
:1095500090971D922F5F3F4F20323105C9F6DF9162
:10956000CF911F910F91FF90EF900895FC01408BD8
:10957000518B628B738B30E040E050E0248735875D
:10958000468757870895CF92DF92EF92FF920F930D
:109590001F93DF93CF93CDB7DEB72A970FB6F8941A
:1095A000DEBF0FBECDBF8C017B016A018AE09BE468
:1095B0009A8389831C821B821E821D8218861F82C9
:1095C0001A870987C8016CE170E00E94240AF8013B
:1095D000F182E082D382C28282E790E4A0E0B0E030
:1095E00084839583A683B783C7016FE0AE014F5F85
:1095F0005F4F0E94BF0D2A960FB6F894DEBF0FBED4
:10960000CDBFCF91DF911F910F91FF90EF90DF9031
:10961000CF9008952F923F924F925F926F927F92D8
:109620008F929F92AF92BF92CF92DF92EF92FF9272
:109630000F931F93DF93CF93CDB7DEB71C01962E08
:10964000772EF42E522E4E2C1C2D6A2C2223E9F15B
:10965000AA24BB246501002321F5FF2011F5E92C84
:10966000F72C163009F4DEC01730A8F1193009F4D0
:109670005CC01A3070F4173009F49BC0183089F4BC
:10968000F701828193810E94B9455520C9F581E097
:1096900009C01D3009F4C0C01F3009F4AAC01A3037
:1096A000A1F380E0CF91DF911F910F91FF90EF9098
:1096B000DF90CF90BF90AF909F908F907F906F90F2
:1096C0005F904F903F902F9008956E2D0E94EA0A70
:1096D0005B016C01C0CF123009F462C01330C0F4DA
:1096E000112309F44BC01130E1F6882009F0B0C015
:1096F000552009F4E9C0F701A480B580C680D78061
:10970000C101642DA60195010E943C0B81E0CACFE6
:10971000133049F1153029F6552009F48BC0F701B3
:10972000A484B584C684D784EBCFF1E06F1609F426
:10973000BBC082E0681609F0A8CF882009F0A5CF49
:109740008AED92E00E945B08A114B104C104D10427
:1097500009F07CC186EE92E00E945B0880EF92E007
:109760000E945B0892CF552009F47FC0F7018281E7
:1097700093810E9435465B016C01C2CF552009F4EC
:1097800090CF662009F08DCF882009F049C176E09E
:10979000A72E7DE2B72E75E0C72E79E6D72EB0CF83
:1097A000552009F46BC0F701A084B184C284D3842E
:1097B000A7CFF5E06F1621F087E0681609F065CFB6
:1097C000882009F427C1F5E06F1609F01EC1E1E019
:1097D0008E1609F462C1F5E06F1609F011C1E2E0DE
:1097E0008E1609F052CFF701808191810E94F00D11
:1097F0004CCF882009F055CFE1E06E1609F051CF2B
:10980000552009F41AC1F701808191810E94DF0D72
:109810005C01CC24DD2474CF8DEF92E00E945B08C4
:1098200080E040CF552069F0F701A088B188C28858
:10983000D38866CFF701A486B586C686D78681E031
:1098400031CFF701A08AB18AC28AD38A81E02ACFB8
:10985000F1E08F1609F025CF552009F4FAC0F70181
:10986000A08CB18CC28CD38C4BCFF70182819381B9
:10987000B601A5010E943D4681E014CFF701848125
:1098800080FF0BC082819381B601A5010E94E5454E
:10989000F701828193810E94B945F701A086B186C4
:1098A000C286D38681E0FECE882009F0EECE87EB1B
:1098B00092E00E945B08C601B5010E94B80A8AECDA
:1098C00092E00E945B08E1CEF7016480758086809B
:1098D00097806A247B248C249D24C301807F947804
:1098E000892B09F0BDC075FE1CC0F70180819181F4
:1098F000B5FCCEC040E050E060E070E00E94D70DC3
:10990000F70184819581A681B78120E030E240E0B3
:1099100050E082279327A427B52784839583A683C5
:10992000B78371FE21C0A601950169E05695479560
:10993000379527956A95D1F72170F7018281938138
:10994000622F0E942D46F70184819581A681B781FF
:1099500020E032E040E050E082279327A427B5279B
:1099600084839583A683B78370FE1CC055274D2D35
:109970003C2D2B2D2170F70182819381622F0E9453
:109980002646F70184819581A681B78120E031E0E8
:1099900040E050E082279327A427B527848395834E
:1099A000A683B783C30181709070892B09F46FCEB1
:1099B000F70122813381C50181709070892B09F0F4
:1099C00074C04FEF5FEF6FEF7FEFC9010E94E54575
:1099D000F701828193810E94B945F70184819581C5
:1099E000A681B78121E030E040E050E08227932754
:1099F000A427B52784839583A683B78381E052CEBD
:109A000087E0681609F4EBCE40CE87E0681609F4CB
:109A1000DECE3BCEF701808191810E94F00DD3CE46
:109A200081E0881609F03DCE8AE6A82E81EAB82E9C
:109A300086E1C82E8BE0D82E63CEB5017F73F70187
:109A4000808191810E94E50D81E02CCE8DEE92E027
:109A500083CEF701A08EB18EC28ED38E81E022CE4E
:109A600088E892E00E945B08F70164817581868135
:109A700097810E94B80A86EA92E00E945B08C601BC
:109A8000B5010E94B80A8BEA92E00E945B08FFCF02
:109A900040E050E06FEF7FEF31CFF701808191819F
:109AA000B601A5010E94EB0D96CEF70140855185C8
:109AB000628573858ACFFC0180E01482158216824C
:109AC00017828F5F3C968031C1F708952F923F92A5
:109AD0004F925F926F927F928F929F92AF92BF92BE
:109AE000CF92DF92EF92FF920F931F93DF93CF936A
:109AF00000D000D0CDB7DEB73C014A015B011801B0
:109B00002901FA82E9829C838B83FC0160E0780161
:109B10008901E80CF91C0A1D1B1D84819581A68111
:109B2000B7810097A105B105E1F020813181428123
:109B3000538182169306A406B50648F0820F931F40
:109B4000A41FB51F88169906AA06BB0620F1281582
:109B500039054A055B0528F02E153F0540075107DA
:109B6000D0F06F5F3C966031C1F620E030E0EB81D1
:109B7000FC8184819581A681B7810097A105B105FB
:109B800011F12F5F3F4FEB81FC813C96FC83EB830F
:109B90002031310561F780E00F900F900F900F900A
:109BA000CF91DF911F910F91FF90EF90DF90CF90B9
:109BB000BF90AF909F908F907F906F905F904F90ED
:109BC0003F902F900895F901EE0FFF1FE20FF31F52
:109BD000DF01AA0FBB1FAA0FBB1FA60DB71D8D92D9
:109BE0009D92AD92BC9213973196EE0FFF1FEE0F30
:109BF000FF1FE60DF71D2082318242825382898148
:109C00009A8119969C938E9318971B96DC92CE920C
:109C10001A9781E0C1CFAF92BF92CF92DF92EF92BD
:109C2000FF920F931F93CF93DF93EC015A016B01C7
:109C3000122FFC0160E070E020813181428153816C
:109C4000A216B306C406D50668F084819581A68164
:109C5000B781280F391F4A1F5B1FA216B306C4061F
:109C6000D506C0F16F5F7F4F3C966031710521F7DB
:109C700007FD24C081E193E00E945B080023D9F432
:109C800089E193E00E945B0884E293E00E945B0814
:109C9000612F70E080E090E00E945F0A89E293E02B
:109CA0000E945B08C601B5010E94B80A84E493E0F3
:109CB0000E945B08FFCF8EE193E0E4CF80E0DF916C
:109CC000CF911F910F91FF90EF90DF90CF90BF90B9
:109CD000AF900895FB01EE0FFF1FE60FF71FEE0F89
:109CE000FF1FEE0FFF1FEC0FFD1F0F77A085B18543
:109CF00082859385B601A501212FFD010995DFCF4E
:109D0000EF92FF920F93CF93DF93E701FC01308531
:109D1000F18480819181A281B381481B590B6A0B28
:109D20007B0B84819581A681B781481759076A0703
:109D30007B0780F4832F9F2DFC01E40FF51F002388
:109D400081F0223009F4ABC0233008F0B2C02130DA
:109D500009F4ABC080E0DF91CF910F91FF90EF90BD
:109D60000895283009F484C0293060F4223009F4C1
:109D7000CFC0243009F4C2C0213061F780818883CC
:109D800081E0E9CF203209F443C0203409F0B2C0A9
:109D900080A191A1A2A1B3A188A399A3AAA3BBA3C7
:109DA00084A195A1A6A1B7A18CA39DA3AEA3BFA397
:109DB00080A591A5A2A5B3A588A799A7AAA7BBA787
:109DC00084A595A5A6A5B7A58CA79DA7AEA7BFA757
:109DD00080A991A9A2A9B3A988AB99ABAAABBBAB47
:109DE00084A995A9A6A9B7A98CAB9DABAEABBFAB17
:109DF00080AD91ADA2ADB3AD88AF99AFAAAFBBAF07
:109E000084AD95ADA6ADB7AD8CAF9DAFAEAFBFAFD6
:109E100080899189A289B389888B998BAA8BBB8B06
:109E200084899589A689B7898C8B9D8BAE8BBF8BD6
:109E3000808D918DA28DB38D888F998FAA8FBB8FC6
:109E4000848D958DA68DB78D8C8F9D8FAE8FBF8F96
:109E500080859185A285B38588879987AA87BB87E6
:109E600084859585A685B7858C879D87AE87BF87B6
:109E700080819181A281B38188839983AA83BB83E6
:109E800084819581A681B7818C839D83AE83BF83B6
:109E900081E0DF91CF910F91FF90EF90089588813D
:109EA00099819183808381E056CF8881808381E08E
:109EB00052CF2430A9F0283009F04CCF8881998105
:109EC000AA81BB8180839183A283B3838C819D818E
:109ED000AE81BF8184839583A683B78381E03BCF26
:109EE00088819981AA81BB8180839183A283B38376
:109EF00081E031CF203109F02DCFAACF808191812F
:109F0000A281B38188839983AA83BB8381E023CF15
:109F1000808191819983888381E01DCFCF92DF92E8
:109F2000EF92FF920F931F93FC01CB0120833183AB
:109F300042835383E482F58206831783D186C086E9
:109F4000BA01A90198018701A0E8EA2EAEE4FA2E31
:109F50006F010E94664D1F910F91FF90EF90DF906F
:109F6000CF900895CF92DF92EF92FF920F931F93BD
:109F7000FC01CB012083318342835383E482F58249
:109F800006831783BA01A9019801870176016F0141
:109F90000E94664D1F910F91FF90EF90DF90CF9040
:109FA0000895FC010190F081E02D09952FEF8F3F7E
:109FB000920779F02FEF8E3F920739F08F3F91058E
:109FC00009F01CF49C01C901089520E031E0C901A9
:109FD000089520E038E0C9010895FB0121E08030B8
:109FE000920721F00280F381E02D09950895EF9208
:109FF000FF920F931F93DF93CF9300D0CDB7DEB7BF
:10A000008C010656104ED801ED90FC900A591F4164
:10A01000F80180A991A9A2A9B3A90097A105B1054A
:10A0200029F181309105A105B10509F462C08230A2
:10A030009105A105B10509F465C083309105A1051D
:10A04000B10501F184309105A105B10509F466C09F
:10A050000597A105B10509F181E00F900F90CF910F
:10A06000DF911F910F91FF90EF90089586E593E0A7
:10A070000E945B08F701E55FF94C80818E7F808349
:10A0800081E0EBCF80E090E0A0E0B1E0F8018083D8
:10A090009183A283B38381E0E0CFF801848195812D
:10A0A000A681B78180389105A105B105A8F5208565
:10A0B000318542855385211531054105510509F446
:10A0C00046C0213031054105510531F50296880F12
:10A0D000991F880F991FE80EF91EF8018081918160
:10A0E000A281B381F70180839183A283B38381E04E
:10A0F000B4CFD8016D917D918D919C910E945F0AA2
:10A1000081E0ABCF1A82F80180818983CE0101966C
:10A110000E945B0881E0A1CF80E09FCFD801149618
:10A120004D915D916D917C911797D7011496ED91AA
:10A13000FC91159716968D919C91179728E030E029
:10A14000E20EF31E9701D8010C91099586CF029675
:10A15000880F991F880F991FE80EF91EF70180815B
:10A160009181A281B381F80180839183A283B3831B
:10A1700073CF0F931F938B018BE693E00E945B08D4
:10A18000C8010E945B088FE793E00E945B08FFCF45
:10A190002F923F924F925F926F927F928F929F92F7
:10A1A000AF92BF92CF92DF92EF92FF920F931F93E5
:10A1B000DF93CF93CDB7DEB728970FB6F894DEBF05
:10A1C0000FBECDBF9C015BE0452E56E3552E480ED9
:10A1D000591EF201808180FFAAC0C9018B50904DA9
:10A1E0009E838D83F901E35DFF4CFC83EB83C90102
:10A1F000895E9F4C9A8389834AEB242E45E3342E53
:10A20000220E331EF901E45EFD4FF887EF8320E054
:10A2100030E040E050E0662477244301AA24BB24C8
:10A2200065010894A11CB11CC11CD11C4C994FC0E4
:10A23000211531054105510509F04CC0E090C13BA5
:10A24000F090C23B0091C33B1091C43B8091C13B55
:10A250009091C23BA091C33BB091C43BE816F90674
:10A260000A071B0759F7662477244301D601C50165
:10A270008F709070A070B0700097A105B10509F4BF
:10A2800079C0AA2009F471C0D601C5019F70A070E1
:10A29000B0700097A105B10509F462C0D601C501EF
:10A2A000A170B0700097A105B105B1F18F819885BB
:10A2B0000E94493DF201808180FF39C0A8019701C9
:10A2C0000894A11CB11CC11CD11C4C9BB1CF7901BD
:10A2D0008A01CCCF8091C13B9091C23BA091C33BFE
:10A2E000B091C43BE090C13BF090C23B0091C33BB6
:10A2F0001091C43B8E159F05A007B10759F7E216D0
:10A30000F3060407150719F361147104810491041D
:10A31000B1F535014601AACFC1010E94CF698F81F5
:10A3200098850E94493DF201808180FDC7CF289623
:10A330000FB6F894DEBF0FBECDBFCF91DF911F9156
:10A340000F91FF90EF90DF90CF90BF90AF909F90D4
:10A350008F907F906F905F904F903F902F900895D7
:10A3600089819A810E94D45999CF8B819C810E94C6
:10A37000BE5C8ACF8D819E810E942D5882CFC601FE
:10A38000B50166197709880999090E945F0A8CE866
:10A3900093E00E945B08EE24FF24870164CF2F9294
:10A3A0003F924F925F926F927F928F929F92AF9265
:10A3B000BF92CF92DF92EF92FF920F931F93CF93B2
:10A3C000DF93EC014B011A01398328831B830A8335
:10A3D000FD82EC82DF82CE82FC01E55FF94C808158
:10A3E00081608083ACE14A2EA2E05A2E4C0E5D1EA5
:10A3F000C20140E050E060E070E023E433E509EBA7
:10A4000010E5F7EFEF2EFFE4FF2EE9E3CE2EE3E5B4
:10A41000DE2E0E944245882329F082E993E00E94C3
:10A420005B08FFCFFE01EA54FE4DD183C083B5E047
:10A43000AB2EBFE2BB2EAC0EBD1EC5010E945B4D14
:10A44000A8EB6A2EA1E27A2E6C0E7D1EC3016BE290
:10A4500073E5A5010E945F4ACE01B101F40109959F
:10A46000FCE08F2EF6E39F2E8C0E9D1ECE018E5E9D
:10A470009D4FB50120E030E040E050E0E2E3EE2EF9
:10A48000F12C012D112D64010E948E4F882329F497
:10A4900087EA93E00E945B08FFCFCE018B53904D7B
:10A4A000B201A3010E94C34AC40162E174E022E345
:10A4B00030E040E050E00E942D0A11EEC12E1FE274
:10A4C000D12ECC0EDD1EC601B201A5010E94695439
:10A4D000882329F487EA93E00E945B08FFCFCE012E
:10A4E0008B50904DB501A6010E944558882329F450
:10A4F00087EA93E00E945B08FFCFCE01895E9F4C04
:10A50000B501A6010E943059882329F487EA93E017
:10A510000E945B08FFCFBDE28B2EB0E39B2E8C0E1A
:10A520009D1EC401B501A60100E010E020E130E469
:10A53000A6E1EA2E0E94B35D882329F487EA93E01E
:10A540000E945B08FFCFCE01815B9E4CB501A60146
:10A5500000E010E020E230E4F5E1EF2E0E94B35D70
:10A56000882329F487EA93E00E945B08FFCFCE019D
:10A570008F589D4CB501A60100E010E020E730E4C3
:10A58000E4E1EE2E0E94B35D882329F487EA93E08C
:10A590000E945B08FFCFCE018D569C4CB201A501F5
:10A5A0000E941B60882329F487EA93E00E945B08DD
:10A5B000FFCFCE018A529C4CB501A6010E94476391
:10A5C000882329F487EA93E00E945B08FFCFCE013D
:10A5D0008C5B9B4CB501A6010E94EE64882329F494
:10A5E00087EA93E00E945B08FFCFCE018E549A4C1D
:10A5F000B2010E94AB65882329F487EA93E00E94A8
:10A600005B08FFCFCE0186549A4CB501A6010E948B
:10A61000EE67882329F487EA93E00E945B08FFCF66
:10A62000C40161ED7FE44DEE5FE49E010E94005B9A
:10A63000DF91CF911F910F91FF90EF90DF90CF901E
:10A64000BF90AF909F908F907F906F905F904F9052
:10A650003F902F900895EF92FF920F937B01BA01E4
:10A66000A90124E000E00E940B4E0F91FF90EF90B3
:10A670000895FC01E656F04E808191818B53904DF8
:10A680000E94B64A08957F928F929F92AF92BF9296
:10A69000CF92DF92EF92FF920F931F93DF93CF93AE
:10A6A00000D000D0CDB7DEB74B01102F7E2C0C2D83
:10A6B0006501FC01E656F04E60817181812F90E0CA
:10A6C000FC0131978E239F23892B69F4CF01AA27A0
:10A6D00097FDA095BA2F82239323A423B523009737
:10A6E000A105B105A1F090E0892F0F900F900F9078
:10A6F0000F90CF91DF911F910F91FF90EF90DF901E
:10A70000CF90BF90AF909F908F907F9008955B0106
:10A71000C50188549E4DBA01A901202F0E2D7E013E
:10A720000894E11CF11C0E9445468823E1F249810E
:10A730005A816B817C81C5018B5F904D212F072D44
:10A7400074010E940B4E90E0882319F081E0982755
:10A75000CBCF91E0FBCFCF92DF92EF92FF920F939E
:10A760001F93CF93DF93EC016B01BC016B5F704DC6
:10A77000885F9D4F20E030E040E050EAE12CF12C72
:10A78000012DB1E01B2F0E94B24F882379F0FE010A
:10A79000E55FF94C808182608083DF91CF911F91CA
:10A7A0000F91FF90EF90DF90CF90089587EB93E0AB
:10A7B0000E945B08FFCFCF92DF92EF92FF920F9340
:10A7C0001F93CF93DF93EC01EA80FB800C811D8106
:10A7D0008E859F85A889B989E822F9220A231B233F
:10A7E0002E813F8148855985CC24D801C701822319
:10A7F0009323A423B5230097A105B10511F0CC2420
:10A80000C394DD2420953095409550952E213F210D
:10A8100040235123211531054105510511F0DD2457
:10A82000D3948B898C1531F08881998161E04C2D0E
:10A830000E947C0D8A898D1531F08881998160E0B4
:10A840004D2D0E947C0DCB8ADA8ADF91CF911F912A
:10A850000F91FF90EF90DF90CF9008950F931F938B
:10A86000FC0106851785208931894423F1F081E0B8
:10A8700090E0A0E0B0E004C0880F991FAA1FBB1FA2
:10A880006A95D2F7802B912BA22BB32B80179107BF
:10A89000A207B30739F086879787A08BB18BCF01CA
:10A8A0000E94DB531F910F91089581E090E0A0E09A
:10A8B000B0E004C0880F991FAA1FBB1F6A95D2F78A
:10A8C00080959095A095B09580239123A223B323E2
:10A8D000DDCFCF92DF92EF92FF920F931F936C0127
:10A8E0008B017A0164E170E00E94240AF601118371
:10A8F0000083C70140E050E060ED70E400E010E04C
:10A9000021E030E0EFE8EE2EE4E5FE2E0E94664DF9
:10A910001F910F91FF90EF90DF90CF900895EF92ED
:10A92000FF920F93CF93DF93E701243009F044C0E7
:10A93000FC0140505040604D7044769567955795A6
:10A94000479576956795579547950023C9F041300F
:10A95000510561057105D9F1423051056105710557
:10A9600009F45CC0453051056105710549F58881E0
:10A970009981AA81BB8182879387A487B5872FC0DD
:10A98000423051056105710509F451C0433051054C
:10A990006105710570F5411551056105710509F4F1
:10A9A00055C0413051056105710509F482C020E0B0
:10A9B00030E040E050E03FC084E494E00E945B0857
:10A9C00081E0DF91CF910F91FF90EF900895888102
:10A9D0009981AA81BB8182839383A483B583CF01AC
:10A9E0000E94DB5381E0DF91CF910F91FF90EF90B8
:10A9F0000895443051056105710509F455C044308E
:10AA0000510561057105D8F14530510561057105A4
:10AA100071F622853385448555850DC088819981DD
:10AA2000AA81BB8186839783A087B187D8CF2681EF
:10AA3000378140855185288339834A835B8381E050
:10AA4000DF91CF910F91FF90EF9008952281338194
:10AA50004481558186859785A089B189282339232A
:10AA60004A235B2386819781A085B1858095909547
:10AA7000A095B095282339234A235B23DCCF22817C
:10AA800033814481558186859785A089B1892823A2
:10AA900039234A235B2386819781A085B1852823AA
:10AAA00039234A235B23C7CF2685378540895189BF
:10AAB000C2CF2281338144815581BDCFCF93DF93B3
:10AAC000FC01EC01AC96AC014C5A5F4F9C012C5F31
:10AAD000314E80E01482158216821782108E118EFC
:10AAE000128E138E188219821A821B821C8A1D8A6A
:10AAF0001E8A1F8ADA011D921D921D921C921397C5
:10AB000054961D921D921D921C925797D9011D9229
:10AB10009D018F5FE858FF4FC858DF4F48585F4F7F
:10AB20008034C1F6DF91CF910895CF93DF93FC017C
:10AB30007183608353834283EC01AC96AC014C5A21
:10AB40005F4F9C012C5F314E80E01482158216828B
:10AB50001782108E118E128E138E188219821A820D
:10AB60001B821C8A1D8A1E8A1F8ADA011D921D9271
:10AB70001D921C92139754961D921D921D921C9229
:10AB80005797D9011D929D018F5FE858FF4FC85814
:10AB9000DF4F48585F4F8034C1F6DF91CF91089561
:10ABA0001F93CF93DF93FC01407FDB01CA0124E0B8
:10ABB000B695A795979587952A95D1F78F73349673
:10ABC00028E78202E0011124CE0FDF1F3497E80F3F
:10ABD000F11DEC5FF14E2081416030E014E113C0C3
:10ABE0002102C0011124FE01E80FF91F808191812B
:10ABF000A281B381817F84179507A607B70749F023
:10AC00003F5F363069F0215058F725E084E690E048
:10AC1000EACF10821182128213823F5F363099F799
:10AC2000DF91CF911F9108952F923F924F925F92A3
:10AC30006F927F928F929F92AF92BF92CF92DF924C
:10AC4000EF92FF920F931F93DF93CF93CDB7DEB7B1
:10AC50002C970FB6F894DEBF0FBECDBF5C012983E1
:10AC60000A83FC82EB82DE82CD82EFE02E2E312C35
:10AC7000412C512C24223522462257223A014B01E5
:10AC80006218730884089508D401C30174E0B6956E
:10AC9000A795979587957A95D1F78F7324E030E043
:10ACA000A20EB31E28E78202A00111244A0D5B1DEB
:10ACB0006CEF7FEFA60EB71ED501A80FB11DAC5FDC
:10ACC000B14E3C91A450BE41BC87AB8761E0C62E1B
:10ACD000D12CE12CF12CC628D728E828F928232FDD
:10ACE00000E014E121502F3F09F491C02102B0018E
:10ACF0001124FA01E60FF71FF887EF838081918115
:10AD0000A281B381817F8C159D05AE05BF0509F435
:10AD100089C00F5F063031F7832F8F5FAB85BC850D
:10AD2000AC5FB14E8C93863009F47AC084E138026E
:10AD3000B0011124640F751F78876F837A817723A0
:10AD400009F069C080E090E0A0E0B0E08629972992
:10AD5000A829B929EF81F88581939193A193B193A3
:10AD6000D50112960D90BC91A02DBA87A987D50167
:10AD70008D919C91BF01A401930100E1EE24CA8052
:10AD8000AB80BC80E985FA850995882339F1EF818C
:10AD9000F88580819181A281B381816080839183D4
:10ADA000A283B383F981F43009F47BC0F981F230D6
:10ADB00009F459C0C10104962F813885280F391F25
:10ADC00038872F836981262F30E040E050E08D8165
:10ADD0009E816F8178850E942D0A81E02C960FB6A6
:10ADE000F894DEBF0FBECDBFCF91DF911F910F91C1
:10ADF000FF90EF90DF90CF90BF90AF909F908F909B
:10AE00007F906F905F904F903F902F90089525E036
:10AE100064E670E06ECF82E090E0A0E0B0E096CF14
:10AE20001C9284CFF981F43069F1F981F23009F094
:10AE300049C0EF81F885E20DF31D84819581AD81D4
:10AE4000BE818D939C932A81222339F6EF81F88568
:10AE500080819181A281B381B695A79597958795B9
:10AE600080958170BBCF2F813885220D331DD9018C
:10AE700014968D919C911597ED81FE81918380832D
:10AE800081E0ACCFEF81F885E20DF31D84819581DF
:10AE9000A681B781ED81FE8180839183A283B383F4
:10AEA000D2CF2F813885220D331DF9018481958100
:10AEB000A681B781ED81FE8180839183A283B383D4
:10AEC00081E08CCFB1016C5F7F4FEF81F8856E0F11
:10AED0007F1FF9812F2F30E040E050E08D819E816F
:10AEE0000E942D0AB0CFAF92BF92CF92DF92EF9225
:10AEF000FF920F931F93FC01A28CB38CC48CD58C52
:10AF000082819381A481B581A816B906CA06DB06A1
:10AF100009F451C026813781408551852A153B05AA
:10AF20004C055D05D9F1A6019501E284F384048501
:10AF30001585E216F3060407150709F179018A0160
:10AF400086859785A089B1898E159F05A007B107D1
:10AF500049F01F910F91FF90EF90DF90CF90BF903D
:10AF6000AF900895828983FFF4CF868D978DA0A13D
:10AF7000B1A18860868F978FA0A3B1A3EACF828901
:10AF800082FFDECF868D978DA0A1B1A18460868FD0
:10AF9000978FA0A3B1A386017501D2CF828981FFCB
:10AFA000C4CF868D978DA0A1B1A18260868F978F27
:10AFB000A0A3B1A3B8CF828980FFACCF868D978D37
:10AFC000A0A1B1A18160868F978FA0A3B1A3A2CFCA
:10AFD0000F931F938C01FC01468D417080819181FC
:10AFE0006AE10E942E54F801268D378D40A151A1AF
:10AFF00056954795379527952170808191816BE112
:10B00000422F0E942E54F801268D378D40A151A168
:10B010005695479537952795569547953795279592
:10B020002170808191816CE1422F0E942E54F801A1
:10B03000268D378D40A151A183E0569547953795D0
:10B0400027958A95D1F72170808191816DE1422FFA
:10B050000E942E541F910F9108950F931F938C01FE
:10B06000FC01828D938DA48DB58D0196A11DB11D1E
:10B07000828F938FA48FB58FC8010E947357C80128
:10B080000E94E8571F910F910895CF92DF92EF929F
:10B09000FF920F931F936C017B018A0162E270E0C3
:10B0A0000E94240AF60111830083C70140E050E0AA
:10B0B00060EA70E400E010E021E030E0EBE6EE2E24
:10B0C000E8E5FE2E0E94664D1F910F91FF90EF90D4
:10B0D000DF90CF900895EF92FF920F931F93CF933D
:10B0E000DF93D701243009F04EC0EC0140505040AE
:10B0F000604A70447695679557954795769567951C
:10B10000579547950023D9F0ED90FD900D911C9136
:10B11000443051056105710509F470C04430510592
:10B1200061057105E0F5FA01EE0FFF1FEE0FFF1F3D
:10B13000EC0FFD1FE282F3820483158328C04430A4
:10B1400051056105710509F45EC044305105610582
:10B15000710508F03FC0FA01EE0FFF1FEE0FFF1F51
:10B16000EC0FFD1F42815381648175814D935D9386
:10B170006D937C93139781E0DF91CF911F910F9195
:10B18000FF90EF9008958DE594E00E945B0881E0C8
:10B19000DF91CF911F910F91FF90EF90089546306E
:10B1A00051056105710509F451C04630510561052D
:10B1B000710598F1473051056105710541F7EA8A3B
:10B1C000FB8A0C8B1D8BCE010E947357CE010E940F
:10B1D000E857DDCF463051056105710591F14630E4
:10B1E000510561057105A0F04730510561057105F4
:10B1F00091F140E050E060E070E0B8CFEA8EFB8E65
:10B200000C8F1D8FC4CF4A8D5B8D6C8D7D8DAECF25
:10B210004E8D5F8D68A179A1A9CFE094F09400953F
:10B2200010958E8D9F8DA8A1B9A18E219F21A0235D
:10B23000B1238E8F9F8FA8A3B9A3CE010E94E85798
:10B24000A6CF4E895F89688D798D90CFEE8AFF8A6F
:10B25000088F198F9CCF4A895B896C897D8986CF3D
:10B26000CF92DF92EF92FF920F931F936C017B01BD
:10B270008A0166E170E00E94240AF60111830083CE
:10B2800012821382148215828FEF9FE7A0E0B0E054
:10B2900086879787A08BB18B0E946E08F601628B20
:10B2A000738B848B958BC70140E050E060E970E4BC
:10B2B00000E010E120E030E0E7EDEE2EE9E5FE2EC3
:10B2C0000E94664D1F910F91FF90EF90DF90CF90FD
:10B2D0000895EF92FF920F931F93CF93DF93EC01AA
:10B2E0000E946E089B01AC018A899B89AC89BD894B
:10B2F000281739074A075B0709F442C0EA84FB8430
:10B300000C851D85E2FE11C08A819B81AC81BD81C7
:10B31000820F931FA41FB51F2E813F814885598539
:10B3200082179307A407B50781F1E3FE0CC082E002
:10B3300090E0A0E0B0E0E82AF92A0A2B1B2BEA866D
:10B34000FB860C871D874E2D4170888199816FE1A6
:10B350000E942E542A853B854C855D8556954795E0
:10B36000379527952170888199816EE1422F0E943F
:10B370002E54DF91CF911F910F91FF90EF90089580
:10B38000EA84FB840C851D85DECF81E090E0A0E09F
:10B39000B0E0E82AF92A0A2B1B2BEA86FB860C87E9
:10B3A0001D87E3FCC4CFCFCF0E9469590895EF9267
:10B3B000FF920F931F93CF93DF93243009F04EC079
:10B3C000EC01405050406049704476956795579520
:10B3D000479576956795579547950023E1F0F701D6
:10B3E000E080F180028113814130510561057105D2
:10B3F00009F440C0413051056105710508F05BC09A
:10B400000E946E086E197F09800B910B6A837B8303
:10B410008C839D8327C0413051056105710589F1F9
:10B42000413051056105710588F50E946E089B0148
:10B43000AC018A819B81AC81BD81281B390B4A0BF1
:10B440005B0BF701208331834283538381E0DF91DB
:10B45000CF911F910F91FF90EF90089588E794E0AE
:10B460000E945B0881E0DF91CF911F910F91FF90C7
:10B47000EF900895EE82FF82088719870E9469592C
:10B48000F1CF2E813F8148855985DBCF4230510570
:10B490006105710509F44AC0433051056105710524
:10B4A00029F020E030E040E050E0CBCF2E853F8512
:10B4B00048895989C6CF423051056105710581F02F
:10B4C000433051056105710569F68E859F85A88910
:10B4D000B989B7FDC7CFEE86FF86088B198BC2CF1F
:10B4E0008A859B85AC85BD8583709070A070B07097
:10B4F000A80197012095309540955095822393237C
:10B50000A423B5232CEF3FEF4FEF5FEFE222F322AE
:10B51000042315238E299F29A02BB12B8A879B8773
:10B52000AC87BD87CE010E9469599CCF2A853B8597
:10B530004C855D8586CF80E091E008950895CF9396
:10B54000DF93DC01EC01C55EDE4F988196FD3EC0C5
:10B55000A75EBE4F8C91A951B14080FF2CC01C96B4
:10B560002C911C972F3FD9F11D969C911D9729175F
:10B5700089F0E92FF0E03796EE0FFF1FEA0FFB1F6F
:10B5800071836083892F8F5F1D968C931D97803404
:10B5900099F1922F9F3F61F01D968C91805C891BE1
:10B5A000813408F08054813218F088818F7D88833F
:10B5B000DF91CF91089595FFFBCFAE5EBE4F6D93A7
:10B5C0007C939F7D9883DF91CF910895A05FBE4FBC
:10B5D0006D937C939F7B9883DF91CF9108951C9608
:10B5E0001C921C9781E01D968C931D971F967C934F
:10B5F0006E931E9790E0D0CF1D961C921D97C9CFD9
:10B60000FC016115710599F04115510539F07783F9
:10B610006683518740873387228708954EE95AE52C
:10B6200077836683518740873387228708956BE944
:10B630007AE5EACF6F927F928F929F92AF92BF92FC
:10B64000CF92DF92EF92FF920F931F93CF93DF93EE
:10B65000DC018C01055E1E4FE801788158E1E52E82
:10B6600051E0F52EE80EF91EF7018081807C808381
:10B670007376788349E1A42E41E0B42EAA0EBB1E56
:10B68000E501888190E080FF39C03EE8832E912C4F
:10B690008A0E9B1EF401D080FFEFDF1609F429C14A
:10B6A0002FE8622E712C6A0E7B1EE3016881605CBC
:10B6B0006D194D2D51E090ECC92EC60EED01C95EFD
:10B6C000DE4F16C0862F981708F056C1403408F098
:10B6D00007C1E42FF0E0E85BFF4FEE0FFF1FEA0F1A
:10B6E000FB1F218130E0232B09F070C05F5F4F5FAB
:10B6F000952F9150613430F38C2DE5CFAC5EBE4F69
:10B700002D913C911197A451B14070FD39C050E08A
:10B71000FD01EA5EFE4FE801888185FFE6C0552302
:10B7200059F4A95EBE4F8C91A751B14081FD03C170
:10B73000E7018881816088832D913C911197608118
:10B740006F71A45EBE4F8C9184FDCDC083FFCBC0D2
:10B7500040E0552309F4EDC081E04827C9010E946B
:10B760002E54DF91CF911F910F91FF90EF90DF90BA
:10B77000CF90BF90AF909F908F907F906F900895E3
:10B7800033FF03C07061F801708332FF04C0E80129
:10B7900088818860888331FF04C0F80180818460DB
:10B7A0008083832F9927892B09F0B3C0A95EBE4FF0
:10B7B0008C91A751B14080FFAACFF70180818460AE
:10B7C000808351E0FD01EA5EFE4FA5CF888182FFB4
:10B7D0008DCF7068F8017083E70188818660888367
:10B7E000F401D080FFEFDF1609F4C0C0E3016881E7
:10B7F000605C6D1951E0613408F06054662309F40F
:10B80000B1C0EFE3ED1510F4F0ECDF0EED2DF0E03C
:10B81000E85BFF4FEE0FFF1FEA0FFB1F0190F08167
:10B82000E02DF3FF04C0E801888180618883F2FF86
:10B8300004C0E801888188608883F1FF04C0E801C2
:10B84000888184608883F501808190E0807C90709D
:10B850008034910509F455C0813491050CF071C014
:10B86000892B09F052C0662309F44FC0A95EBE4F70
:10B870008C91A751B14080FF07C0552321F4E70107
:10B8800088818460888351E0F40190819F3F09F4AE
:10B890003FCFA157BF4F8C91AF58B040805C891B00
:10B8A000813408F08054882309F432CFFD01EA5E28
:10B8B000FE4F808182958695877090E004970CF406
:10B8C0002ACFA95EBE4F8C91A751B14080FF23CFF4
:10B8D000552321F4E70188818C60888351E01BCFD8
:10B8E000E42FE054F7CE40E039CF552309F420CFC0
:10B8F00023CF50E060E0807C90708034910509F0A7
:10B90000ABCF80E0683030F5682F662309F4BCCFF8
:10B91000ADCFA95EBE4F8C91A751B14082FF4BCFF6
:10B92000E70188818660888351E0FD01EA5EFE4F71
:10B93000F2CE41E011CFE70188818260888351E037
:10B94000FBCE8038910549F0803C9105F1F680E00E
:10B950006032D0F281E0682FD8CF80E06031D0F73C
:10B96000682FD3CFE501888190E070CFF501808109
:10B9700090E051E060E0BFCF50E03DCFEF92FF920A
:10B980000F931F93CF93DF93EC018C01055E1E4F45
:10B99000D8018C9186FD46C0E0E1EE2EE1E0FE2E5E
:10B9A000EC0EFD1EF70180819181E885F9852AE57D
:10B9B000EE39F20709F4C1C06A857B850995C75E37
:10B9C000DE4F8881C951D14080FF8FC08C858F3F69
:10B9D00009F4AEC02D85205C922F981B2054913421
:10B9E00008F09054992309F4A3C0E82FF0E03796AB
:10B9F000EE0FFF1FEC0FFD1F0190F081E02D8F5F18
:10BA00008C87803409F4A9C08C85821709F4A7C0FB
:10BA1000D701ED93FC939150913220F4F80180818D
:10BA200080628083EE81FF812AE5EB39F20709F419
:10BA300069C08A859B850995AC0181E04030580733
:10BA400009F43FC0FE01EA5EFE4F80818F71808362
:10BA5000D8012C91922F91609C93C75EDE4F888114
:10BA6000C951D14080FF27C0FE01E257FF4F9081AE
:10BA70009F3F09F468C0DE01A157BF4F8C91981712
:10BA800009F45DC0E82FF0E0E85BFF4FEE0FFF1F09
:10BA9000EC0FFD1F518340838F5F8C93803409F43A
:10BAA0001C92CE010E941A5BDF91CF911F910F91E2
:10BAB000FF90EF90089590FF27C02360F801208346
:10BAC000F0CFFE01EA5EFE4F3081232F22952695AE
:10BAD0002770822F90E0059724F72F5F2295220F81
:10BAE000207E3F71322B3083DCCFF801208125FF8F
:10BAF00012C020642083EE81FF812AE5EB39F20732
:10BB000009F097CFCE0197CFCC5EDE4F59834883A3
:10BB1000C451D140C6CFCE5EDE4F88819981C251DB
:10BB2000D140D7018D939C932062F80120837ACF76
:10BB3000D8018C9180648C9375CFBE013FCF236078
:10BB4000D8012C93AECF1082C157DF4F81E089938B
:10BB500059834883C059D040A4CF1C8655CF8FEF5E
:10BB60008C878D8755CF4F925F926F927F928F9285
:10BB70009F92AF92BF92CF92DF92EF92FF920F937C
:10BB80001F936C012B015A01380149011E2D62E2FD
:10BB900071E00E94240AF601B182A082EA5EFE4FA3
:10BBA0001F718081807E812B8083F6016282738287
:10BBB0008482958228E131E0C20ED31E81E0F60135
:10BBC000808380E682936F0124E030E0C20ED31EB2
:10BBD000F601808322E030E0C20ED31E80E1F60140
:10BBE000808323EE3EEFC20ED31E8FEFF6018487D3
:10BBF00085872EE830E0C20ED31EF60181936F01D7
:10BC0000808321E73FEFC20ED31E8BE99AE5F60150
:10BC1000978386838EE99AE59187808713861286BB
:10BC2000C201B401A30100E010E021E030E0FCE239
:10BC3000EF2EFEE5FF2E0E94664D1F910F91FF90A3
:10BC4000EF90DF90CF90BF90AF909F908F907F90BC
:10BC50006F905F904F900895CF92DF92EF92FF9296
:10BC60000F931F93CF93DF93302FEC018C01065E6F
:10BC70001E4FD801EC91243019F0213009F06FC02B
:10BC8000FE2FFF1FFF27FF1F8A819B81AC81BD8193
:10BC9000481B590B6A0B7B0B769567955795479513
:10BCA0007695679557954795332321F1D701EC9009
:10BCB000433051056105710509F4E2C04430510576
:10BCC0006105710508F459C04730510561057105DA
:10BCD00009F4BFC0483051056105710509F4BFC0C2
:10BCE000443051056105710509F4AAC0CE010E94D6
:10BCF0001A5B39C0443051056105710509F4FBC078
:10BD0000453051056105710508F469C0463051059B
:10BD10006105710509F4D1C0463051056105710511
:10BD200008F487C0473051056105710509F4D3C097
:10BD3000483051056105710509F4C6C030E0E0E006
:10BD4000213009F483C08E2F90E0A0E0B0E0F7012D
:10BD500080839183A283B383332329F0C7CF82E901
:10BD600094E00E945B0881E0DF91CF911F910F91D9
:10BD7000FF90EF90DF90CF9008954130510561051D
:10BD8000710509F48DC0423051056105710508F453
:10BD900049C0FE01E75EFE4F80818E2580FF1DC0F9
:10BDA0009E2DE0FE1DC1E1FE07C0C257DF4F8FEFA1
:10BDB00089938883CF58D04092FF09C08FEF8C873A
:10BDC0008D87C55EDE4F80E68883CB51D140C85E4B
:10BDD000DE4F81EC8883C851D140E08287CF41306B
:10BDE00051056105710509F47DC0413051056105BA
:10BDF000710550F4FF2309F4A9C0C15EDE4FE8814C
:10BE0000CF51D14030E09CCF4230510561057105E2
:10BE100009F44CC0433051056105710509F08ECF1E
:10BE200030E08ECFFF2309F4D5C0C15EDE4FE8823B
:10BE30009ACFC55EDE4FE881CB51D14030E080CF54
:10BE4000C45EDE4FE882CC51D14050CFD701EC9395
:10BE500083CFC25EDE4FE882CE51D14047CFCF5D67
:10BE6000DE4FE882C152D1408E2D90E083709070F9
:10BE7000892B09F43BCF84ED94E00E945B0836CF18
:10BE80008E2D8E2786FF02C0E6FE03C0F801E082F9
:10BE90002DCFCE0160E078E00E949F5AF801F7CFE5
:10BEA000FF2381F1C05EDE4FE8825DCFC85EDE4FCA
:10BEB000E881C851D14030E043CFC35EDE4FE88116
:10BEC000CD51D14030E03CCFCF5DDE4FE881C15253
:10BED000D14030E035CFC25EDE4FE881CE51D14057
:10BEE00030E02ECFFF2359F1C05EDE4FE881C05213
:10BEF000D14030E025CFC45EDE4FE881CC51D14047
:10BF000030E01ECFB7E1CB2EB1E0DB2ECC0EDD1E34
:10BF1000F60110811E2517FD7FC016FF0BC0E6FE3F
:10BF200009C0C55EDE4F80E68883229680E1888363
:10BF3000CD51D140D6018C9118271C93D7CEC95E24
:10BF4000DE4FE881C751D14030E0FACE8E01055E68
:10BF50001E4FD8019C9190FFF1CEC75EDE4F8881C5
:10BF6000C951D14080FF4EC0AE0142575F4FFA0128
:10BF700080818F3F09F456C0E82FF0E0E85BFF4F67
:10BF8000EE0FFF1FEC0FFD1F90818F5FDA018C9386
:10BF9000803409F44EC0FA013081BE0161577F4FF1
:10BFA000DB018C91381709F43FC0E92F3F3F59F06E
:10BFB000DB018C91805C831B813408F080548823E2
:10BFC00011F031E0BDCED8019C919E7FD8019C93A9
:10BFD00031E0B6CECE016E2D70E00E949F5A86CE23
:10BFE0008FEF8C878D87C257DF4F89938883C45723
:10BFF000DF4F80E68883239781E08883C851D14052
:10C00000E08274CECC5EDE4FE881C451D1409E7F89
:10C01000D8019C9330E094CE8DEA94E00E945B08B6
:10C020001F777BCFEFEFD1CF8FEF80838C933FEFE4
:10C03000BCCF1C92B0CF8F929F92AF92BF92CF9203
:10C04000DF92EF92FF920F931F93DF93CF93CDB7C1
:10C05000DEB72A970FB6F894DEBF0FBECDBF5C01E6
:10C060008B014A0163E470E00E94240AF501118308
:10C07000008382E291E0A0E0B0E082839383A48316
:10C08000B5838FEE99E7A1E0B0E086839783A08720
:10C09000B18723E030E040E050E0228733874487D7
:10C0A000558780E290E0A0E0B0E0828B938BA48B78
:10C0B000B58B228F338F448F558F268F378F40A3B8
:10C0C00051A322A333A344A355A38EE390E0A80E6B
:10C0D000B91E81E090E0A0E0B0E0F501808391839B
:10C0E000A283B38382EC9FEFA80EB91E81EA91E68A
:10C0F0009A8389831C821B821E821D8218861F825E
:10C10000BA86A986C8016EE0AE014F5F5F4F0E94FC
:10C11000BF0DC40140E050E060E371E400E010E1D5
:10C1200020E030E0F5E3EF2EF1E6FF2E65010E94FE
:10C13000664D8823A9F490E0892F2A960FB6F894CB
:10C14000DEBF0FBECDBFCF91DF911F910F91FF904A
:10C15000EF90DF90CF90BF90AF909F908F90089519
:10C16000C40140E050E060EF70E400E010E120E046
:10C1700030E0EAECEE2EE0E6FE2E65010E94664D10
:10C1800090E0882319F081E09827D6CF91E081E0F4
:10C190009827D2CFEF92FF920F931F93CF93DF9305
:10C1A000A02FE701243009F044C040505040604FB8
:10C1B0007044769567955795479576956795579509
:10C1C00047950023F9F400E010E020E030E04D3026
:10C1D000510561057105F8F4FC01AA23B1F1CA010A
:10C1E000880F991F880F991FE80FF91F0687178777
:10C1F000208B318B81E0DF91CF911F910F91FF90C8
:10C20000EF900895088119812A813B814D305105B5
:10C210006105710508F3AA2381F4088319832A8331
:10C220003B8381E0DF91CF911F910F91FF90EF90C1
:10C23000089581EF94E00E945B0881E0DF91CF9147
:10C240001F910F91FF90EF900895CA01880F991FD9
:10C25000880F991FE80FF91F0685178520893189F6
:10C26000088319832A833B83DCCFEF92FF920F93DD
:10C270001F93CF93DF93382F192FE7012430B1F5A7
:10C28000002379F580E090E0A0E0B0E0E32FF12F0B
:10C290004050504060437144769567955795479557
:10C2A000769567955795479541305105610571051C
:10C2B00081F1413051056105710520F14230510590
:10C2C0006105710569F10023A9F488839983AA8324
:10C2D000BB8381E0DF91CF911F910F91FF90EF9091
:10C2E000089588819981AA81BB81D0CF81EF94E0A4
:10C2F0000E945B0881E0DF91CF911F910F91FF9029
:10C30000EF900895002399F082839383A483B583EB
:10C31000F1CF002389F086839783A087B187EACF86
:10C32000002341F782859385A485B585CECF828190
:10C330009381A481B581C9CF86819781A085B1857C
:10C34000C4CF6F927F928F92AF92BF92CF92DF92C3
:10C35000EF92FF920F931F93DF93CF93CDB7DEB78A
:10C360003C01D62EB72EF42E122F222319F120E0F5
:10C3700030E040E050E0AA2071F4882061F400230E
:10C3800051F4FF2041F4ED2DFB2D86E0C81689F114
:10C3900087E0C816A9F080E0CF91DF911F910F913F
:10C3A000FF90EF90DF90CF90BF90AF908F907F90F5
:10C3B0006F9008956E2D0E94EA0A9B01AC01DBCFBD
:10C3C0001123A9F0EE5BFF4F8081112381F020E063
:10C3D00030E040E050E0882321F021E030E040E010
:10C3E00050E0C3016E2D0E943C0B81E0D5CF81E06F
:10C3F000D3CF112339F7EE5BFF4F822F81708083FB
:10C4000021FFF5CF8EE095E00E945B0881E0C4CF6C
:10C410002F923F924F925F926F927F929F92AF9234
:10C42000BF92CF92DF92EF92FF920F931F93DF9311
:10C43000CF9300D000D000D0CDB7DEB71C01498328
:10C440005A836B837C83E981FA81EE0FFF1FEE0F25
:10C45000FF1FB1016E0F7F1FDB019696ED90FD90DF
:10C460000D911C919997A8019701209530954095C1
:10C4700050951E96AD90BD90CD90DC9051972A219D
:10C480003B214C215D21E20DF31D82819381A4812A
:10C49000B581E822F9220A231B232E293F29402BAC
:10C4A000512BFB01228F338F448F558F49805A8047
:10C4B0006B807C80440C551C661C771C9924A3E07F
:10C4C000EA2EF12C012D112DF1E0AF2EB12CC12C53
:10C4D000D12CC201880F991F880F991F820D931DBF
:10C4E0008A5A9F4F9E838D83665E7F4FED81FE81CA
:10C4F00080819181A281B3818E219F21A023B123CC
:10C500000097A105B10599F0D601C50180959095D8
:10C51000A095B095FB012081318142815381822316
:10C520009323A423B52380839183A283B38393941D
:10C53000EE0CFF1C001F111FEE0CFF1C001F111F33
:10C54000AA0CBB1CCC1CDD1CF0E19F1679F60894EC
:10C55000411C511C611C711CB201660F771F660FD4
:10C56000771F620D731D6A5A7F4F69807A80660C4F
:10C57000771C660C771C620C731C8AE190E0680ED5
:10C58000791E0CC0EE0CFF1C001F111FEE0CFF1CCF
:10C59000001F111FAA0CBB1CCC1CDD1CFB018081E1
:10C5A0009181A281B3818E219F21A023B123009785
:10C5B000A105B10599F0D601C50180959095A0958A
:10C5C000B095F301208131814281538182239323ED
:10C5D000A423B52380839183A283B3839394F0E251
:10C5E0009F1681F626960FB6F894DEBF0FBECDBF1C
:10C5F000CF91DF911F910F91FF90EF90DF90CF903F
:10C60000BF90AF909F907F906F905F904F903F90C2
:10C610002F900895CF93DF93EC01288139818E8D7F
:10C620009F8DA8A1B9A10097A105B10591F48AA198
:10C630009BA1ACA1BDA10097A105B10551F440E0BB
:10C640008A8D9B8DAC8DBD8D8C7F0097A105B1052A
:10C6500009F041E0C9016AE00E942E542A8D3B8D09
:10C660004C8D5D8D5695479537952795217088811E
:10C67000998169E0422F0E942E544A8D4170888131
:10C68000998168E00E942E54DF91CF910895CF9256
:10C69000DF92EF92FF920F931F936C017B018A014F
:10C6A0006EE670E00E94240AF60111830083C70140
:10C6B00040E050E060EE70E400E010E120E030E0A7
:10C6C000EDE6EE2EE3E6FE2E0E94664D1F910F91E1
:10C6D000FF90EF90DF90CF900895EF92FF920F932D
:10C6E0001F93CF93DF93F701243009F072C0EC0160
:10C6F00040505040604E70447695679557954795E9
:10C7000076956795579547950023A1F1E080F180D4
:10C71000028113814F3051056105710508F465C030
:10C72000453151056105710508F0B9C04231510527
:10C730006105710508F429C14251504060407040C4
:10C74000FA01EE0FFF1FEE0FFF1FEC0FFD1FE65B60
:10C75000FF4FE094F0940095109580819181A28123
:10C76000B381E822F9220A231B23E082F1820283AB
:10C7700013838AC04F3051056105710508F44AC022
:10C78000453151056105710508F0AAC042315105D6
:10C790006105710508F4CCC04251504060407040C2
:10C7A000CA01880F991F880F991FC80FD91FC65B30
:10C7B000DF4F88819981AA81BB8180839183A28385
:10C7C000B38381E0DF91CF911F910F91FF90EF90A4
:10C7D00008958DE195E00E945B0881E0DF91CF91A3
:10C7E0001F910F91FF90EF9008954C305105610516
:10C7F000710530F14C50504060407040CA01880FC4
:10C80000991F880F991FC80FD91FEAAAFBAA0CAB62
:10C810001DABE3CF4C3051056105710508F446C0EE
:10C820004C50504060407040CA01880F991F880FDB
:10C83000991FC80FD91F8AA99BA9ACA9BDA9BDCFB3
:10C84000493051056105710508F083C04630510536
:10C850006105710508F0AAC04330510561057105F5
:10C8600008F4BBCF4350504060407040FA01EE0FD7
:10C87000FF1FEE0FFF1FEC0FFD1FE6A2F7A200A7A0
:10C8800011A7CE010E940862CE010E940A6381E0D6
:10C89000DF91CF911F910F91FF90EF9008954B3151
:10C8A00051056105710508F098CFEBCF4330510574
:10C8B0006105710588F14630510561057105A8F4DF
:10C8C0004350504060407040CA01880F991F880F44
:10C8D000991FC80FD91F8EA19FA1A8A5B9A56DCF7B
:10C8E0004B3151056105710528F080E090E0A0E032
:10C8F000B0E063CF4551504060407040CA01880F9E
:10C90000991F880F991FC80FD91FCA5ADF4F8881F6
:10C910009981AA81BB8151CFCA01880F991F880FC5
:10C92000991FC80FD91F8A8D9B8DAC8DBD8D45CFAA
:10C930004F50504060407040CA01880F991F880FC7
:10C94000991FC80FD91FEE9688819981AA81BB8152
:10C9500034CF4950504060407040FA01EE0FFF1F45
:10C96000EE0FFF1FEC0FFD1FE094F0940095109563
:10C97000828D938DA48DB58DE822F9220A231B2385
:10C98000E28EF38E048F158F7CCF4F505040604065
:10C990007040CA01880F991F880F991FC80FD91FAF
:10C9A000EE96E882F9820A831B8317CF46505040E7
:10C9B00060407040FA01EE0FFF1FEE0FFF1FEC0FFB
:10C9C000FD1F828D938DA48DB58DE82AF92A0A2B3F
:10C9D0001B2BE28EF38E048F158F53CFCF92DF92F5
:10C9E000EF92FF920F931F936C017B018A016EE619
:10C9F00071E00E94240AF60111830083F382E2822F
:10CA0000C70140E050E060E070E400E010E120E0A9
:10CA100030E0E6E1EE2EE5E6FE2E0E94664D1F9127
:10CA20000F91FF90EF90DF90CF900895CF92DF921B
:10CA3000EF92FF920F931F93CF93DF93A02FE70105
:10CA4000243009F04DC0FC0140505040604070441B
:10CA50008A019B0136952795179507953695279559
:10CA600017950795AA23D9F4BB27A72F962F852FB3
:10CA70000197A105B10509F447C080E090E0A0E06E
:10CA8000B0E088839983AA83BB8381E0DF91CF9153
:10CA90001F910F91FF90EF90DF90CF900895C88085
:10CAA000D980EA80FB80452F562F672F77274130AA
:10CAB000510561057105E9F14130510561057105C7
:10CAC000A0F40031110521053105F8F6C114D10497
:10CAD000E104F104D1F282E595E00E945B08FFCF0A
:10CAE00088E395E00E945B08D0CF42305105610594
:10CAF000710559F6C114D104E104F10431F282E563
:10CB000095E00E945B08FFCFD901C8018054904096
:10CB1000A040B04088329105A105B10508F0ADCF25
:10CB2000E80FF91FEA5BFE4F808190E0A0E0B0E0E3
:10CB3000A8CFD901C80180549040A040B0408832AD
:10CB40009105A105B10508F0A0CFE80FF91FEA5B38
:10CB5000FE4FC0829ACFEF92FF920F931F93DF9305
:10CB6000CF93CDB7DEB72A970FB6F894DEBF0FBECE
:10CB7000CDBF8C017B0168E070E00E94240A82EE48
:10CB800095E69A8389831C821B821E821D828BE715
:10CB900097E698878F831A870987C70160E0AE01FF
:10CBA0004F5F5F4F0E94BF0D81E02A960FB6F89449
:10CBB000DEBF0FBECDBFCF91DF911F910F91FF90D0
:10CBC000EF9008952F923F924F925F926F927F92D3
:10CBD0008F929F92AF92BF92CF92DF92EF92FF928D
:10CBE0000F931F93DF93CF93CDB7DEB72B970FB67D
:10CBF000F894DEBF0FBECDBF3C0169877A87013054
:10CC0000D1F080E02B960FB6F894DEBF0FBECDBFFB
:10CC1000CF91DF911F910F91FF90EF90DF90CF9018
:10CC2000BF90AF909F908F907F906F905F904F904C
:10CC30003F902F900895442321F7222311F7882055
:10CC400001F76E2D0E94EA0A6D837E838F83988799
:10CC5000C3016A2D0E94EA0A69837A838B839C83CD
:10CC60008C2D86958695813061F2813008F05FC009
:10CC7000ED80FE800F811885110FEE08FE2C8701D4
:10CC800069807A808B809C80990C6608762C4301A1
:10CC90002D813E814F8158856E2D7E2D8E2D9E2DAE
:10CCA000A980BA80CB80DC80E62CF62C062D162DD0
:10CCB0000E945001E985FA85A0818181128103815A
:10CCC000B481A20F71E0A21708F070E0830F91E029
:10CCD000831708F090E0780F21E0781708F020E043
:10CCE000922B842F810F21E0841708F020E0492F38
:10CCF000480F91E0481708F090E0292B852F800F0E
:10CD000091E0851708F090E0322F380F21E03817B6
:10CD100008F020E0922BB60F9B0FA0837183428313
:10CD20003383948315821682178281E06BCF823021
:10CD300049F0833009F49CC020E030E040E050E04E
:10CD400060E0B8CF2D813E81C901AA2797FDA0954B
:10CD5000BA2F7C018D01110FEE08FE2C870149814D
:10CD60005A813A01882477FC8094982C130124017D
:10CD7000550C2208322C21019C01AD016E2D7E2D17
:10CD80008E2D9E2D53016401E22CF22C022D122DCA
:10CD90000E945001522E232E442E352E6B872D815A
:10CDA0003E814F815885CA01AA27BB27AA2797FD34
:10CDB000A095BA2F5C016D01DD0CAA08BA2C6501A3
:10CDC00029813A814B815C817A0100271127002754
:10CDD000F7FC0095102F37014801990C6608762C56
:10CDE00043019C01AD016A2D7A2D8A2D9A2D5701A0
:10CDF0006801E62CF62C062D162D0E945001732F8B
:10CE0000F42FB52FE62F122F150D91E0121708F011
:10CE100090E0372F320D81E0371708F080E0A92F1E
:10CE2000A30F91E0A31708F090E0892B4F2F440D3A
:10CE300091E04F1708F090E0782F740F81E074179D
:10CE400008F080E0982B5B2F530D21E05B1708F072
:10CE500020E0892F850F61E0851708F060E0622BE4
:10CE60003B85E30F212F3A2F472F582F6E0F22CFEC
:10CE7000C1FE0BC089819A81AB81BC81CD01AA27FB
:10CE8000BB2789839A83AB83BC83C0FE0BC02D81F3
:10CE90003E814F8158859A01442755272D833E8333
:10CEA0004F8358874D815E81CA01AA2797FDA095BF
:10CEB000BA2F7C018D01110FEE08FE2C870129810C
:10CEC0003A813901882477FC8094982C130124013D
:10CED000550C2208322C21019C01AD016E2D7E2DB6
:10CEE0008E2D9E2D53016401E22CF22C022D122D69
:10CEF0000E945001DFCE2F923F924F925F926F922D
:10CF00007F928F929F92AF92BF92CF92DF92EF92D9
:10CF1000FF920F931F93CF93DF934C01CC2079F5B1
:10CF2000222369F5EB014423F1F56E2D0E94EA0AF4
:10CF30005B016C01C401602F0E94EA0A1B012C01F5
:10CF40008FEF90E0A0E0B0E0A822B922CA22DB2255
:10CF50009501A60160E070E080E090E000E20E94B0
:10CF6000CA022229332944295529288339834A832F
:10CF70005B836C837D838E839F8381E001C080E02F
:10CF8000DF91CF911F910F91FF90EF90DF90CF90A5
:10CF9000BF90AF909F908F907F906F905F904F90D9
:10CFA0003F902F900895288139814A815B81602FBD
:10CFB0000E943C0B288139814A815B816C817D8193
:10CFC0008E819F8100E20E944B0230E040E050E001
:10CFD000C4016E2D0E943C0B81E0D2CFCF92DF9234
:10CFE000EF92FF920F931F936C017B018A0161E521
:10CFF00070E00E94240AF60111830083F382E2822A
:10D000008AE490E0C80ED91E8EE89CE7F601918371
:10D01000808386EB9FEFC80ED91EC70140E050E029
:10D0200060E074E400E010E120E030E0EEE5EE2E98
:10D03000E8E6FE2E0E94664D1F910F91FF90EF9043
:10D04000DF90CF900895CF93DF93DC01FC01E65B86
:10D05000FF4FA85BBF4F0190F081E02D8D919C9117
:10D060001197A854B040E823F9233097F1F4ED016B
:10D07000C45BDF4F888186FF15C090E0309709F0D0
:10D0800091E09295990F990F907C88818F7B892BE5
:10D0900088838D919C9140E0EF2B09F041E061E1A4
:10D0A0000E942E54DF91CF910895ED01C45BDF4FB4
:10D0B000888186FFE2CFDF91CF910895EF92FF92B2
:10D0C0000F931F93CF93DF93D701243009F050C003
:10D0D000EC014050504060407444769567955795F8
:10D0E00047957695679557954795002361F1ED90A3
:10D0F000FD900D911C91493051056105710509F4B0
:10D100006CC04A3051056105710508F045C04230D8
:10D1100051056105710509F40CC1433051056105E4
:10D12000710508F470C0433051056105710509F4BB
:10D13000F1C04830510561057105F1F4EC8AFD8AB2
:10D140000E8B1F8B19C0FA0148385105E8F020E01A
:10D1500030E040E050E02D933D934D935C93139766
:10D1600081E0DF91CF911F910F91FF90EF90089593
:10D1700086E695E00E945B0881E0DF91CF911F91E8
:10D180000F91FF90EF900895EA5BFF4FEE0FFF1FA6
:10D190000590F491E02D0994403151056105710528
:10D1A00009F4B3C04131510561057105D8F040382B
:10D1B00051056105710509F4B7C044385105610591
:10D1C000710509F4ACC04131510561057105A1F645
:10D1D000ECA2FDA20EA31FA3CFCFE88EF98E0A8F7B
:10D1E0001B8FCACF4E3051056105710509F47DC012
:10D1F0004F3051056105710509F0BECFEC8EFD8EF3
:10D200000E8F1F8FB9CF411551056105710509F4C6
:10D2100095C0413051056105710509F0ADCFE88633
:10D22000F9860A871B87A8CFCC5BDF4F288139811D
:10D230004A815B8190CF2C813D814E815F818BCF74
:10D24000C05CDF4F288139814A815B8184CF2CAD5E
:10D250003DAD4EAD5FAD7FCF28AD39AD4AAD5BADD5
:10D260007ACF2CA93DA94EA95FA975CF28A939A9C4
:10D270004AA95BA970CF2CA53DA54EA55FA56BCF94
:10D2800028A539A54AA55BA566CF2CA13DA14EA135
:10D290005FA161CF28A139A14AA15BA15CCF2C8DF0
:10D2A0003D8D4E8D5F8D57CFC85BDF4F8881998153
:10D2B0009C0140E050E04FCF288D398D4A8D5B8D29
:10D2C0004ACF2C893D894E895F8945CF2889398984
:10D2D0004A895B8940CF2C853D854E855F853BCF54
:10D2E000288539854A855B8536CFFC01E85BFF4F91
:10D2F000C70180959095208131818223932391836A
:10D300008083CE010E94236837CFE8A2F9A20AA346
:10D310001BA332CFE88AF98A0A8B1B8B2DCFE8AE8C
:10D32000F9AE0AAF1BAF28CFE8A6F9A60AA71BA73C
:10D3300023CFEC86FD860E871F871ECF8C819D81B3
:10D34000AE81BF818E259F25A027B1278170907067
:10D35000892B31F0FE01E45BFF4F80818068808380
:10D36000EC82FD820E831F8305FD16C08EE89CE7CC
:10D3700004FD9260F2FC8160E6FC8068E5FC80635D
:10D38000E4FC8260C65BDF4F99838883CA54D04037
:10D39000CE010E942368F0CE8EEC9CE7E9CF4F923D
:10D3A0005F926F927F928F929F92AF92BF92CF9235
:10D3B000DF92EF92FF920F93DF93CF9300D000D0D4
:10D3C000CDB7DEB76C01ACE46A2E712C680E791E05
:10D3D000D3018C9187FF08C0F601848180FFBFC014
:10D3E000D3018C918F778C93F601848180FFA0C04C
:10D3F000D3018C918F7390E08130910509F4BAC00C
:10D400008230910509F4DAC0892B09F091C0F60148
:10D410002489358946895789C90181709070892B83
:10D4200009F4DFC0DA01C9018E7F848B958BA68B4E
:10D43000B78B21FDF2C0D60154968D909D90AD9092
:10D44000BC90579780EF9FEFAFEFBFEF88229922F4
:10D45000AA22BB22F60182819381B501A40124E0B6
:10D4600000E02E010894411C511C72010E940B4ED9
:10D47000882309F0C8C080E090E0A0E0B0E0F601A9
:10D4800080A791A7A2A7B3A7B501A4014C5F5F4FE6
:10D490006F4F7F4F8281938124E000E072010E94F0
:10D4A0000B4E882309F0AAC080E090E0A0E0B0E035
:10D4B000F60184A795A7A6A7B7A7B501A401485F61
:10D4C0005F4F6F4F7F4F8281938124E000E07201B4
:10D4D0000E940B4E882309F08CC080E090E0A0E011
:10D4E000B0E0F60180AB91ABA2ABB3AB8CE090E0C7
:10D4F000A0E0B0E0880E991EAA1EBB1E8281938117
:10D50000B501A40124E000E072010E940B4E8823C3
:10D5100009F47EC089819A81AB81BC81F60184AB1C
:10D5200095ABA6ABB7ABD3018C91807C81608C931B
:10D53000C6010E9423680F900F900F900F90CF911B
:10D54000DF910F91FF90EF90DF90CF90BF90AF9061
:10D550009F908F907F906F905F904F900895E85BC1
:10D56000FF4F808191818068918380838C91807C42
:10D570008C9336CFF60124A935A946A957A946FFB1
:10D5800007C0E85BFF4F8081918182609183808337
:10D5900052FD0EC0F601E35BFF4F80819181A281B5
:10D5A000B3810196A11DB11D80839183A283B383B2
:10D5B000D3018C91807C82608C93BACFF60184A9D0
:10D5C00095A9A6A9B7A9A5FF07C0E85BFF4F808171
:10D5D0009181916091838083D3018C91807C8C9325
:10D5E000A7CFD60198968D909D90AD90BC909B97BB
:10D5F00031CF89819A81AB81BC8173CF89819A8136
:10D60000AB81BC8155CF89819A81AB81BC8137CFF9
:10D6100080E090E0A0E0B0E081CFE85BFF4F808148
:10D62000918192609183808306CF629FD001739F26
:10D63000F001829FE00DF11D649FE00DF11D929FAE
:10D64000F00D839FF00D749FF00D659FF00D9927ED
:10D65000729FB00DE11DF91F639FB00DE11DF91F11
:10D66000BD01CF0111240895A1E21A2EAA1BBB1BF4
:10D67000FD010DC0AA1FBB1FEE1FFF1FA217B3079E
:10D68000E407F50720F0A21BB30BE40BF50B661FB4
:10D69000771F881F991F1A9469F760957095809578
:10D6A00090959B01AC01BD01CF0108952F923F924F
:10D6B0004F925F926F927F928F929F92AF92BF92A2
:10D6C000CF92DF92EF92FF920F931F93CF93DF934E
:10D6D000CDB7DEB7CA1BDB0B0FB6F894DEBF0FBEAB
:10D6E000CDBF09942A88398848885F846E847D84F8
:10D6F0008C849B84AA84B984C884DF80EE80FD80FA
:10D700000C811B81AA81B981CE0FD11D0FB6F8946F
:0ED71000DEBF0FBECDBFED010895F894FFCF30
:10D71E00014E6F20616C6C6F636174696F6E732064
:10D72E00696E20617672206D6F646520706C656124
:10D73E0073652100736420696E6974206661696C7B
:10D74E00656400417474656D707420746F2062722C
:10D75E00616E636820746F206E6F6E2D776F7264CA
:10D76E002D616C69676E65642041524D2061646461
:10D77E007265737300496E76616C6964206D6F64B7
:10D78E00652070617373656420746F2063707550CB
:10D79E0072764D6F6465546F42616E6B656452654F
:10D7AE00677350747228290043616E6E6F74207512
:10D7BE006E726169736520464951207768656E20E7
:10D7CE006E6F6E65207261697365640043616E6E83
:10D7DE006F7420756E72616973652049525120779E
:10D7EE0068656E206E6F6E65207261697365640088
:10D7FE00496E76616C696420696E7374722030783C
:10D80E0000207365656E206174203078002E2043F1
:10D81E005053523D3078000D0A0000008007B000D2
:10D82E0080010000C007D000900100009007B000FA
:10D83E0090010000D007F0009001000010000000E1
:10D84E0030001000B0013000B0015000B0010000F7
:10D85E00B0000000D0007000B00100001001000008
:10D86E007002000050010000700100009001900055
:10D87E0010000000D0010000F001000000000000C8
:10D88E000000717561727465722070616765206643
:10D89E006F756E64210D0A00637031353A20756E16
:10D8AE006B6E6F776E2062697473206368616E674A
:10D8BE006564203078002D3E3078002C2068616C35
:10D8CE0074696E670D0A00417474656D707420740E
:10D8DE006F206C6F636B203078002B333220696EB3
:10D8EE00206963616368650D0A004463616368655E
:10D8FE00206E6F7720006F7574206F6600696E0062
:10D90E00206C6F636B206D6F64650D0A0046435388
:10D91E0045206E6F7420737570706F727465640A33
:10D92E00004D656D6F7279200072656164007772CB
:10D93E0069746500206F662000206279746573201B
:10D94E00617420706879736963616C2061646472BC
:10D95E0020307800206661696C732C2068616C74CD
:10D96E00696E670D0A00487970657263616C6C2090
:10D97E0030206361756768740D0A00456D756C61C2
:10D98E0074696F6E206572726F723A203C3C003E75
:10D99E003E2068616C74696E670D0A0020487A0D2E
:10D9AE000A004661696C656420746F20696E697443
:10D9BE00204350553A20006572726F722048616C98
:10D9CE0074696E670D0A0043616E6E6F7420696E26
:10D9DE00697420636F52414D2048616C74696E67A3
:10D9EE000D0A0043616E6E6F7420616C6C6F636123
:10D9FE0074652052414D20627566666572204861DD
:10DA0E006C74696E670D0A0043616E6E6F742069E7
:10DA1E006E69742052414D2048616C74696E670DB9
:10DA2E000A0001008FE210FF2FE1042701200021E0
:10DA3E0000F00DF80A242407651C0527002200F0CB
:10DA4E0006F82060241D491C8029F8D12847BC46C1
:10DA5E00BBBB70477078613235355F49432E633AF0
:10DA6E0020556E657870656374656420007078610A
:10DA7E003235355F54494D522E633A20556E6578D6
:10DA8E0070656374656420007078613235355F525D
:10DA9E0054432E633A20556E6578706563746564E1
:10DAAE0020007078613235355F554152542E633AFD
:10DABE0020556E65787065637465642000707861BA
:10DACE00323535554152543A20444D41206D6F64E4
:10DADE00652063616E6E6F7420626520656E616293
:10DAEE006C656400554152543A2049724441206D90
:10DAFE006F646520736574206F6E20554152540A11
:10DB0E00007078613235355F507772436C6B2E63DF
:10DB1E003A20556E657870656374656420005365B0
:10DB2E0074207370656564206D6F64650070786134
:10DB3E003235355F4750494F2E633A20556E657822
:10DB4E0070656374656420007078613235355F44AA
:10DB5E004D412E633A20556E657870656374656429
:10DB6E002000646D613A2077726974657320756E5A
:10DB7E00696D706C21007078613235355F4C4344AD
:10DB8E002E633A20556E6578706563746564200067
:00000001FF
